:020000040800F2
:1000000000000220C9F40008A1870008A3870008A7
:10001000A5870008A7870008A9870008000000003E
:10002000000000000000000000000000AB87000896
:10003000AD87000800000000AF870008B187000806
:100040000DF500080DF500080DF500080DF5000888
:100050000DF500080DF500080DF50008B58700083E
:100060000DF500080DF500080DF500082D5C0008E1
:100070000DF500080DF500080DF500080DF5000858
:100080000DF500080DF500080DF500080DF5000848
:100090000DF500080DF500080DF50008858900082C
:1000A0000DF500080DF500080DF500080DF5000828
:1000B000D9870008E98700080DF500080DF500084C
:1000C0000DF500080DF500080DF500080DF5000808
:1000D0000DF500080DF50008998A00080DF50008D7
:1000E0000DF500080DF500080DF500080DF50008E8
:1000F0000DF500080DF500080DF500080DF50008D8
:100100000DF500080DF500080DF500080DF50008C7
:100110000DF500080DF500080DF500080DF50008B7
:100120000DF500080DF500080DF500080DF50008A7
:100130000DF500080DF500080DF500080DF5000897
:100140000DF500080DF500080DF50008DD87000825
:100150000DF500080DF500080DF500080DF5000877
:100160000DF500080DF500080DF500080DF5000867
:100170000DF500080DF500080DF500080DF5000857
:080180000DF500080DF5000863
:1001880024A60508000000200C0B0020100B0020FE
:10019800E4610020064B07481A68074B1A60074BB2
:1001A80000221A70064B01221A7001F070B800BFC5
:1001B80078400020100D00208C4000206440002072
:1001C8008C3A002008B5034801F061F8024B002280
:1001D8001A7008BDA00F00208C3A002008B5054B06
:1001E800012200201A7004F04DF80348BDE80840C9
:1001F80001F04DB824410020441000202DE9F041C1
:10020800144C204602F083FB00201349134A02F0E5
:1002180035F91349134A0746002002F02FF912490D
:10022800124A0646002002F029F9D22105463A462C
:1002380023460A2002F03AFAD22132462346FA200F
:1002480002F034FA5A20D2212A462346BDE8F0416A
:1002580002F02CBA580E00204A960508CD01000875
:1002680053960508E50100085B9605089D010008FE
:1002780008B5054B012200201A7004F003F8034862
:10028800BDE8084001F003B82441002044100020D4
:10029800044B054800221A70044B02221A7000F021
:1002A800F6BF00BF64400020580E00208C3A0020A2
:1002B80008B5034800F0EBFF024B00221A7008BD96
:1002C800A00F00208C3A00202DE9F041144C204664
:1002D80002F01DFB00201349134A02F0CFF813491E
:1002E800134A0746002002F0C9F81249124A064686
:1002F800002002F0C3F8D22105463A4623460A20D8
:1003080002F0D4F9D221324623465A2002F0CEF91F
:10031800AA20D2212A462346BDE8F04102F0C6B9F8
:10032800100D00204A960508B902000864960508D1
:10033800990200086D96050879020008002008B5A2
:1003480003F0A0FF064B00221A70064B1B78022B05
:100358000CBF05480548BDE8084000F098BF00BF3D
:10036800244100208C3A0020580E0020100D002057
:1003780010B5084C204602F0CAFA00200649074A80
:1003880002F07CF8D22102462346E620BDE8104060
:1003980002F08CB98C1100207696050845030008F8
:1003A80010B5074C4FF6E071206801F0BBFB2068E0
:1003B800044901F065FBBDE8104002F0E1BC00BF54
:1003C800100B00207F96050810B5074C4FF6E0711A
:1003D800206801F0A7FB2068044901F051FBBDE843
:1003E800104002F0CDBC00BF100B00209496050809
:1003F80070B5514C2DED028B20684FF6E07101F07D
:1004080091FB20684D4901F03BFB02F0B9FC00204C
:1004180003F038FF23790BB9FFF7C2FF6379464D24
:1004280053B928684FF6E07101F07CFB286844490D
:1004380001F026FB02F0A4FCA3790BB9FFF7C4FF77
:100448003D4C6379002B69D02379002B66D094ED5D
:10045800038AD4ED048A78EE687A88EE288AA2683E
:10046800384B394D1A6017EE900A0EF0B1F9002298
:10047800364B0EF001FA02460B46002034490EF0C6
:1004880025FB0EF0DBFC334B0646186018EE100A0D
:100498000EF09EF90022304B0EF03AF802460B4659
:1004A80000202B490EF012FB21A3D3E900230EF004
:1004B8002FF80EF0C3FCA279286000232371637122
:1004C80002B1A371254A1F4C137031464FF4967040
:1004D80005F01DFC29684FF4987005F018FC216898
:1004E8004FF49A7005F013FC1A4B94ED001A124C55
:1004F80093ED000AD5ED000A07F090F820684FF652
:10050800E07101F00FFB2068154901F0B9FA07F016
:10051800B8F802F035FC134802F076FC1248BDEC3E
:10052800028BBDE8704000F0B2BE00BFAFF30080A0
:100538000000000000805140100B0020A99605081B
:10054800BE960508040D0020080D002000005E403E
:10055800000049400C0D00200000F03F8C3A0020BC
:10056800D396050880969800A00F0020014800F057
:100578008EBE00BFA00F00202DE9F047384C394D42
:10058800A3686068AB600EF023F9064620680F4642
:100598000EF01EF90022344B0EF06EF90022804650
:1005A800894630463946304B0DF0B4FF42464B463B
:1005B8000EF08CFA0EF042FC25A3D3E90023686103
:1005C800394630460DF0A6FF42464B460EF07EFAFD
:1005D8000EF034FCA8614FF6E07003F027FE68695E
:1005E800224E0EF0F5F805F11C0402460B46204693
:1005F800314612F0B7FD224600236E203A2103F05F
:1006080043FFA8690EF0E4F802460B46204631463F
:1006180012F0A8FD224600236E206C2103F034FF5F
:10062800A8680EF0D5F80CA3D3E900230EF024F93E
:1006380002460B4620460E4912F094FD6E209E217C
:1006480022460023BDE8F04703F01EBFAFF3008049
:100658000000000000805140000000A2941A6D4282
:10066800D45E0020100B002000005E40E7960508CD
:10067800ED96050870B506F0CBFF10EE104A06F0AF
:10068800DDFF064620460EF0A3F807EE106AF8EEE6
:10069800C77A044617EE900A0D460EF099F81AA389
:1006A800D3E900230EF0E8F802460B462046294617
:1006B8000EF00CFA0EF0C2FB114CA0600EF088F898
:1006C8000DA3D3E900230EF0D7F804F11C05024668
:1006D8000B4628460B4912F045FD4FF6E07003F033
:1006E800A5FD00236E209E212A4603F0CDFE01239E
:1006F800A37170BDAFF30080000000A2941A6D4290
:10070800100B0020ED9605081F85EB51B81E194007
:1007180038B506F077FF0F4C10EE100A84ED030A87
:100728000EF056F804F11C0502460B4628460A4905
:1007380012F018FD4FF6E07003F078FD00236E20EC
:100748003A212A4603F0A0FE01236371BDE8384030
:1007580026E600BF100B0020E796050838B506F01E
:1007680051FF0F4C10EE100A84ED040A0EF030F819
:1007780004F11C0502460B4628460A4912F0F2FC11
:100788004FF6E07003F052FD00236E206C212A46DC
:1007980003F07AFE01232371BDE8384014E600BF58
:1007A800100B0020E79605082DE9F04F4F4D504EED
:1007B80085B000244FF6FF78284602F0A8F8414695
:1007C800224623464B480094019401F06FF9042710
:1007D8007062224623464FF6E0714748009701941D
:1007E80001F064F9414630602246234643480097A9
:1007F800019401F05BF94146B06222462346404825
:100808000097019401F052F92346F06241462246CE
:100818003C480097019401F049F93B4930633B4A51
:10082800204601F02BFE3A493A4A0746204601F095
:1008380025FE3949394A8046204601F01FFE3849CD
:10084800384A8146204601F019FE3749374A824620
:10085800204601F013FE3649364A84462046CDF834
:100868000CC001F00BFE21468346726A2B462046D7
:1008780001F01CFF214632682B467D2001F016FF4F
:100888006E21F26A2B460A2001F010FF3C21326BE0
:100898002B460A2001F00AFF69213A462B46E6203A
:1008A80001F004FF372142462B46E62001F0FEFE08
:1008B8004A462B46E6209B2101F0F8FE52462B467D
:1008C8006E20C82101F0F2FEC8215A462B46AA2004
:1008D80001F0ECFEDDF80CC0E620C82162462B468C
:1008E80005B0BDE8F04F01F0E1BE00BFFC0E0020EE
:1008F800100B0020F6960508BE960508AA9605086E
:10090800FE9605081797050831970508650700083A
:100918003897050819070008409705087D0600085C
:1009280048970508810500084E97050875050008D1
:1009380055970508F9030008014B93ED000A704725
:100948000C0D0020014B93ED000A7047080D0020A4
:10095800014B93ED000A7047040D0020AFF30080AF
:10096800294B2A48062210B51A704FF6E07400F099
:100978008EFC0020214607F055F83120214607F06B
:1009880051F86320214607F04DF89520214607F0DD
:1009980049F81F34C7204FF4FC6107F043F820469C
:1009A80003F044FC052001210023194A03F06CFDE3
:1009B800052020210023174A03F066FD0520522157
:1009C8000023154A03F060FD84210520134A002303
:1009D80003F05AFD4FF4FC6003F028FCB621052013
:1009E8000F4A002303F050FD204603F01FFC0D4A78
:1009F80000238720DC2103F047FD0B4B00221A60FF
:100A08000A4B01221A7010BD24410020D412002084
:100A18005C970508939705088B9705086097050864
:100A2800A09C0508629705087C40002064400020CF
:100A38003B4B3C48072270B51A704FF6E07400F043
:100A480026FC0020214606F0EDFF3120214606F065
:100A5800E9FF6320214606F0E5FF9520214606F0D0
:100A6800E1FF4FF6FF752146C72006F0DBFF284659
:100A780003F0DCFB0520012100232B4A2B4E03F059
:100A880003FD052020210023294A03F0FDFC052051
:100A980052210023274A03F0F7FC05208421002374
:100AA800254A03F0F1FC0520B6213246002303F065
:100AB800EBFC40F213144FF4FC6003F0B7FB204644
:100AC80001211E4A002303F0DFFC204620211C4A96
:100AD800002303F0D9FC204652213246002303F0BC
:100AE800D3FC20468421174A002303F0CDFCB6210D
:100AF800154A0023204603F0C7FC284603F096FB5E
:100B0800124A00237D20DC2103F0BEFC104B00229A
:100B18001A60104A012313700F4A137070BD00BF8A
:100B280024410020D412002067970508899B0508F6
:100B38006B9705086F970508729705087B97050856
:100B480077970508769705087A9705087F97050827
:100B58007C40002064400020604D002038B52D4BBB
:100B68002D4805241C704FF6E07500F090FB00201E
:100B7800294606F057FF2720294606F053FF4F2045
:100B8800294606F04FFF7720294606F04BFF9F20A5
:100B9800294606F047FF2946C7201F3506F042FFC1
:100BA800284603F043FB0121002320461B4A03F09B
:100BB8006BFC162100232046194A03F065FC3E21F0
:100BC80000232046174A03F05FFC662100232046D5
:100BD800154A03F059FC8E2100232046134A03F0DE
:100BE80053FCB621124A0023204603F04DFC284648
:100BF80003F01CFB0F4A00237D20DC2103F044FC9A
:100C08000D4B00221A600D4A012313700C4A137011
:100C180038BD00BF24410020D4120020899B05085C
:100C28008A9705088E9705089297050896970508EC
:100C38009A9705089E9705087C400020644000208C
:100C4800604D0020F8B53B4B3B483C4F3C4E0422DE
:100C58001A704FF6E07400F01AFB0020214606F0E7
:100C6800E1FE3120214606F0DDFE6320214606F034
:100C7800D9FE9520214606F0D5FE4FF6FF75214690
:100C8800C72006F0CFFE284603F0D0FA0520012140
:100C980000233A4603F0F8FB052020210023294AC7
:100CA80003F0F2FB052052210023274A03F0ECFB56
:100CB800052084210023254A03F0E6FB0520B62100
:100CC8003246002303F0E0FB40F213144FF4FC60BB
:100CD80003F0ACFA204601213A46002303F0D4FB86
:100CE800204620211A4A002303F0CEFB2046522139
:100CF8003246002303F0C8FB20468421154A00230E
:100D080003F0C2FBB621144A0023204603F0BCFBC3
:100D1800284603F08BFA114A00237D20DC2103F0DA
:100D2800B3FB0F4B00221A600E4A012313700E4AC0
:100D38001370F8BD24410020D4120020BF97050885
:100D4800899B0508AA970508BA970508AF9705086B
:100D5800B4970508B9970508BE970508C29705080E
:100D68007C40002064400020604D0020F8B5324BE4
:100D78003248334F334E03221A704FF6E07400F0B6
:100D880086FA0020214606F04DFE6320214606F033
:100D980049FEB3204FF4FC6106F044FE2146C7200B
:100DA8001F3406F03FFE204603F040FADC21002302
:100DB8007D20254A03F068FB204603F037FA05201A
:100DC800012100233A4603F05FFB0520522100234E
:100DD8001E4A03F059FBB62100230520324603F0D2
:100DE80053FB40F213154FF4FC6003F01FFA002385
:100DF800284601213A4603F047FB5221284632464D
:100E0800002303F041FBB621114A0023284603F0D2
:100E18003BFB204603F00AFA0E4A00230520A221D4
:100E280003F032FB0C4B00221A600C4A01231370AA
:100E38000B4A1370F8BD00BF24410020D4120020D3
:100E4800DC970508899B0508CD970508D7970508FD
:100E5800DB9705089B9705087C400020644000202C
:100E6800604D002008B5074B074802221A7000F0B1
:100E78000EFA06F0CFFC054B00221A60044B012243
:100E88001A7008BD24410020D41200207C400020A4
:100E980064400020002008B503F0F4F9064B002256
:100EA8001A70064B1B78022B0CBF05480548BDE895
:100EB800084000F0ECB900BF244100208C3A002023
:100EC800580E0020100D00202DE9F14F2D4C204622
:100ED80001F01DFD00202C492C4A01F0CFFA2C49C5
:100EE8002C4A8146002001F0C9FA2B492B4A0746B3
:100EF800002001F0C3FA2A492A4A0646002001F0D8
:100F0800BDFA2949294A0546002001F0B7FA2849BF
:100F1800284A8046002001F0B1FA2749274A82462C
:100F2800002001F0ABFAD22183464A462346E62048
:100F380001F0BCFB28203A462346014601F0B6FBE7
:100F4800462132462346282001F0B0FB64212A4678
:100F58002346282001F0AAFB822142462346282066
:100F680001F0A4FB524623462820A02101F09EFB55
:100F780028205A46BE21234601B0BDE8F04F01F0B3
:100F880095BB00BF44100020769605089D0E00080A
:100F9800E09705086D0E0008CD970508750D000847
:100FA800C29705084D0C0008EB970508650B00086B
:100FB800F6970508390A00086297050869090008C4
:100FC80008B5002003F05EF906F0EEFA06F06AF8BC
:100FD800064B00221A70064B01221A7006F080FD9B
:100FE8000448BDE8084000F052B900BF2441002081
:100FF8008C3A0020100D002008B5002003F042F9BB
:1010080006F0D2FA064B00221A70064B02221A701A
:1010180006F066FD0448BDE8084000F038B900BF96
:10102800244100208C3A0020580E002008B50020EA
:1010380003F028F9034B044803221A70BDE808405E
:1010480000F025B98C3A0020FC0E002010B50B4C9E
:1010580006F0AAFA04F0A4F806F019FB06F040FD21
:1010680020684FF6E07100F05DFD2068044900F04B
:1010780007FDBDE8104001F083BE00BF440B00200F
:10108800009805080088C83880B2042810B505D92A
:101098000A480B4A0B4B7F2102F09AF80A4CC0B25F
:1010A80004F006F920684FF6E07100F03BFD206877
:1010B8000649BDE8104000F0E3BC00BF14980508DD
:1010C80034D0030834980508440B002065980508B7
:1010D8002DE9F04F5248534D85B0002401F017FC1C
:1010E8004FF6FF71224623464F480094019400F0C2
:1010F800DDFC042607464FF6E071224623464B489E
:101108000096019400F0D2FC4FF6E071804622462A
:10111800234647480096019400F0C8FC4FF6FF713B
:1011280081462246234643480096019400F0BEFCBF
:10113800234628604FF6FF7122463F4800960194E7
:1011480000F0B4FC3D4968603D4A204601F096F93C
:101158003C493D4A8246204601F090F93B493C4AC9
:101168008346204601F08AF93A4902903A4A2046D5
:1011780001F084F93A4603902146294B204601F0B4
:1011880095FA21464246264BC82001F08FFA0A21DB
:101198004A46234BC82001F089FA2A68204B64216B
:1011A800782001F083FA78206A681D4B014601F027
:1011B8007DFAC82505262827E0B203F0ABFF274AA9
:1011C8000146284601F05AF994FBF6F106FB114155
:1011D80079431E31024689B20020114B0134013592
:1011E80001F064FA042CADB2E6D1D22152460520B2
:1011F8000B4B01F05BFAD2215A464C20084B01F008
:1012080055FAD221029A064B9C2001F04FFA039A14
:10121800034BEC20D22105B0BDE8F04F01F046BAEF
:10122800A00F0020440B0020759805087F9805083A
:101238008C98050897980508AA960508AB9805089C
:1012480055100008B398050835100008BC98050823
:1012580001100008C5980508C90F00088D1000087E
:1012680008B500F005FAFEF7C9FFFFF79DFAFFF78A
:101278002BF8FFF729FEFFF72BFFFFF779F800F0AF
:101288008BFA00F0D9F8BDE8084000F0A1B910B514
:10129800044628B90F48104A104B452101F098FF21
:1012A8000F4B1868844213D010B1C36900219847C6
:1012B800002002F0E7FF002002F0CEFF4FF6FF709B
:1012C80002F0B4FFE369204601219847044B1C60F3
:1012D80010BD00BFCE98050843D00308EA9805085A
:1012E8004C0B00200048D2E7A00F00204FF6FF70FB
:1012F80070474FF6FF70704713B5002944D04FF27E
:10130800DE7002F0BFFF002003F086F80F2002F025
:101318008DFF1E4C1E4A412101230A2003F0B4F818
:10132800042003F079F8236828209621042B21DC77
:101338000123184A03F0A8F801A90DF10602206854
:1013480003F02AFB0F2002F071FFBDF80400BDF87E
:10135800061014382822002380B202F097FFBDF847
:101368000610BDF80400143989B22822012302F0BE
:101378008DFF09E0084A012303F086F81E20A52105
:10138800064A012303F080F81CBD00BF500B002063
:10139800FA9805080D990508299905083F9905083F
:1013A80037B51E4C2368042B05462BDC01A80DF12C
:1013B800060103F0EFFABDF80630BDF8042018491D
:1013C800042007F02BFD2368002B04DA1548164A81
:1013D800164B592105E0042B05DD1248124A144B1F
:1013E8005A2101F0F5FE04EB8302BDF80410013325
:1013F8009180BDF806102360052BD18008D1201DEF
:1014080003F04AFB00230B482360FFF740FF03E08B
:1014180028460121FFF770FF3EBD00BF500B00209A
:10142800569905089B99050855D00308BD990508E4
:10143800D4990508E810002037B50B4C204601F078
:1014480066FA0A4B0A49009300250120094A0A4B0B
:10145800019501F004F9294602462346284603B0BF
:10146800BDE8304001F022B9B40D00200113000896
:10147800F5120008FB120008A91300084FF6FF70C8
:1014880070474FF6FF7070471FB54FF6E07002F0D7
:10149800F9FE002002F0C0FF0F2002F0C7FE002175
:1014A800294A2A4C01230A2002F0EEFF002002F00C
:1014B800BDFE042002F0B0FF0A201921244A0123AE
:1014C80002F0E2FF2521234A01230A2002F0DCFF73
:1014D8001F2002F0ABFE01230A2037211E4A02F02A
:1014E800D3FF237873B301231E2096211B4A02F0F1
:1014F800CBFF62881A49684611F034FE01231E208A
:10150800A2216A4602F0C0FFA2881649684611F077
:1015180029FEAE216A4601231E2002F0B5FF0F20E6
:1015280002F084FE6088A188143880B22822002343
:1015380002F0ACFEA1886088143989B22822012300
:1015480002F0A4FE1FBD00BF029A0508680B002028
:10155800149A0508349A0508549A0508779A0508D4
:10156800899A0508969A050801B18DE7704713B561
:101578000DF1060101A803F0C1F9144B01221A70FC
:101588005988BDF80420891A0E311C2919460AD831
:101598009C88BDF80600201A0E301C2803D89968CC
:1015A8000131996001E000238B60084B996801299B
:1015B80005DD00229A601A70FFF794FE05E05A8054
:1015C800BDF806209A80FFF75FFF1CBD680B00205E
:1015D80037B50B4C204601F09AF90A4B0A4900939B
:1015E80000250120094A0A4B019501F038F82946DF
:1015F80002462346284603B0BDE8304001F056B8FD
:10160800E810002071150008851400088B140008E4
:101618007715000838B50D4B0D4D00241C700D4B87
:101628001C700D4B4FF0FF321A600C4B1A680C4BB4
:1016380020461A6002F026FE0A4B1B78022B0CBFCC
:1016480009480A48FFF723FE2C7038BD24410020C2
:10165800604D0020644000207C400020784000203D
:101668008C4000208C3A0020580E0020100D0020DD
:1016780010B50B4C204601F04AF9002001462246DD
:1016880000F074FA00200749074A00F0F7FED2215B
:10169800024623464FF48270BDE8104001F006B8B8
:1016A800D41200204E9705081D16000810B5064CE8
:1016B8004FF6FF71206800F035FA044B206819686E
:1016C800BDE8104000F0DCB9740B00209801002040
:1016D80008B5002002F0D6FD054B1868054B1968BF
:1016E80000F0CEF90448BDE80840FFF7D0BD00BFC0
:1016F800740B002094010020A00F002008B5FFF70C
:10170800D5FF0020014605F043FEBDE8084001F082
:1017180037BB0088A0F5C87080B2092808B505D97C
:101728000748084A084B8F2101F052FD074B1880E3
:10173800074BFF21197005F02BFEBDE80840B5E7FF
:10174800A39A050867D00308C69A050878130020ED
:101758007A1300200088A0F5967080B2092808B591
:1017680005D90848084A094B832101F031FD084B87
:101778001880084B0121197005F00AFEBDE80840E1
:1017880094E700BFA39A05087CD00308C69A050809
:10179800781300207A1300202DE9F34100243A48F9
:1017A8003A4D01F0B4F8224623464FF6FF71384807
:1017B8000094019400F07AF904262246234607464D
:1017C8004FF6FF7133480096019400F06FF92346F5
:1017D800286022464FF6FF712E480096019400F0CB
:1017E80065F92D4968602D4A204600F047FE2C49CE
:1017F8002C4A0646204600F041FE214680463A46DD
:101808002046214B00F052FF2A681F4B2046282112
:1018180000F04CFF3246D2211B4B5A2000F046FF05
:10182800AA20D2214246184B00F040FF0F254FF462
:10183800967440F2351620461B491C4A00F01EFEDD
:1018480001340246782128460F4BA4B2233500F014
:101858002DFFB442ADB2EED10F254FF4C87440F25B
:10186800991620461249134A00F008FE0134024630
:101878009B212846044BA4B2233500F017FFB4423D
:10188800ADB2EED1BDE8FC8130120020740B00200F
:10189800F79A0508BB960508039B05080517000875
:1018A8000C9B0508D9160008159B05085D1700084C
:1018B800179B05081B17000808B508B143682BB922
:1018C8000348044A044B9B2101F082FC586908BD77
:1018D800199B050890D003083B9B050808B5FFF73E
:1018E800EBFF8068123080B208BD08B5FFF7E4FF4F
:1018F8004068063080B208BD2DE9F84F0446884696
:10190800FFF7DAFF6689E589074606F1030905F15D
:101918000F0AB8F1000F1FD01F2002F087FC2046E5
:10192800FFF7DCFF83462046FFF7DFFF2946034623
:101938005FFA8BF2F0B202F0ADFC042002F06CFD0D
:101948000B364FF6FF70033502F070FCB0B2A9B247
:101958003A68012302F098FD3D69204641464A460F
:101968005346A847BDE8F88F13B504460DF10601A4
:1019780001A802F0C3FF2046FFF79EFF6389BDF868
:101988000410BDF80620C91AE389D21A0339C368BE
:101998000F3A204698471CBDF7B5044614200D465B
:1019A80016461F4611F06CF8089BC7600361064B8A
:1019B8000649074A80E8700000930190054B002013
:1019C80000F04DFEFEBD00BF01190008F318000825
:1019D800E518000871190008704708B508B1436890
:1019E8002BB90448044A054BAD2101F0F1FB5869B5
:1019F80008BD00BF5A9B0508A8D003083B9B0508F3
:101A0800F8B505460E46FFF7E8FF836B04461BB1A1
:101A180028463146984700E018466F8994F83C30CC
:101A2800ED890EB9034310D0208E02F0FFFB608EC3
:101A380002F012FC94F8350002F0EEFC94F8343011
:101A480038462946224602F01FFD002384F83C3020
:101A5800F8BD08B5FFF7C1FF90F83500BDE80840AC
:101A680002F0EFBC38B5FFF7B8FF044611F000FCF0
:101A7800054694F8350002F0DFFC684380B238BDB3
:101A880038B50D46FFF7A9FF29462E22044611F066
:101A98001FFC50B1204629462E2211F06BFC002372
:101AA80084F82E30012384F83C3038BD2DE9F74303
:101AB800074640200E461546984610F0E1FF0446BA
:101AC80028B91148114A124B4E2101F081FB114BE4
:101AD800114A12498DE818000020114B00F0BFFD93
:101AE80039468146FFF7CCFF9DF82830268684F8D2
:101AF80035300B9B6586A363002384F8348084F813
:101B08003C304846BDE8FE835A9B0508C0D0030810
:101B1800789B0508091A00085B1A00086D1A000866
:101B2800E119000810B50C46FFF757FF012304869A
:101B380080F83C3010BD00BF4FF4A0707047C8203B
:101B480070477047074B1B78022B07B508D1064B27
:101B58001B78022B04D001A80DF1060102F0CEFE7D
:101B68000EBD00BF604D00202441002073B50A4B14
:101B780006460D461446009300200849084A094BBA
:101B8800019000F06CFD294602462346304602B01B
:101B9800BDE8704000F08ABD4B1B0008411B0008DF
:101BA800471B00084D1B000813B502AB03E90600EC
:101BB800436843B1027C0124082A9C7004D11B6944
:101BC8002146984700E01C4620461CBD30B5002839
:101BD8002BD0058B002425E0036A1A7C012A05D145
:101BE8005B681A888A421BD1187F30BD052A06D146
:101BF8005B681A888A4213D193F82C0030BD032AF7
:101C080006D15B681A888A420AD193F8250030BD4C
:101C1800062A05D15B681A888A4201D1D87A30BD74
:101C280001340430AC42D7D3002030BD08B18175EF
:101C380001207047F8B504460D46D0B1E175D0F8DB
:101C480098309847012D0DD12746002606E0F869FF
:101C580000F10802436906CA98470136238B043706
:101C68009E42F4D3D4F8983020462946984701205C
:101C7800F8BDF8BDF8B50546084617460E4611F0FA
:101C8800F7FA013FB84234BF04463C463CB1284607
:101C98003146224611F06EFB00232B55F8BD2C70FF
:101CA800F8BDF7B5044600200090019000296CD0DB
:101CB8000E8B68E000F1080351F823301D7C042DD9
:101CC80004D15D682D88954247D0013000F10803A2
:101CD80051F823301D7C012D04D15D682D88954273
:101CE8003BD0013000F1080351F823301D7C052D4D
:101CF80004D15D682D8895422FD0013000F108038A
:101D080051F823301D7C032D04D15D682D88954240
:101D180023D0013000F1080351F823301D7C022D37
:101D280004D15D682D88954217D0013000F1080371
:101D380051F823301D7C072D04D15D682D8A95420A
:101D48000BD0013000F1080351F823301D7C062D1B
:101D580008D15D682D88954203D103F1080120461A
:101D680015E0013000F1080351F823502B7C082BB3
:101D780009D16F683F88974204D105F108012046D0
:101D88001A4605E00130B04294D32046694608223D
:101D980011F026F92046FEBDF8B505460F46164651
:101DA800002830D04388032B2FD0202010F068FE65
:101DB800044600282BD040F80C5B39460C22FFF76C
:101DC80059FF1820E66110F05BFE0646B8B1022301
:101DD8000374012363760F4B446063600E4BA3606A
:101DE800002323766B8805EB830201339BB2012B1A
:101DF80050606B800CD16A685268137608E0204600
:101E080010F046FE04E0064602E0002600E0064622
:101E18003046F8BD30500408CE4C040837B5456844
:101E280002AB03E906003DB3037C0124042B85F8CB
:101E3800314022D1688E02F0F9F995F8300002F0AD
:101E4800EBFA95F8343043B9BDF80200BDF8061036
:101E5800AA1C234602F018FB0FE0012B03D1084807
:101E680040F2395104E0022B07D1054840F24151B4
:101E7800044A054B01F0ACF92C4620463EBD00BF94
:101E88008B9B0508801B0408899B0508F8B5044648
:101E98000F46164610B3838A0A2B20D0202010F054
:101EA800EFFD0546E8B14460102200F1080039460C
:101EB800FFF7E0FE4FF6FF73A08A2B801F236B808D
:101EC80000232B76831D013080B20128EE6144F88F
:101ED8002350A08207D1A3691876F8BDF8BD002069
:101EE800F8BD0120F8BD0120F8BD2DE9F0411D46DF
:101EF8004B1C984280460C4617460CDD95420ADC7E
:101F0800013208F101035B1A521BC8B2D2B29BB26C
:101F1800294602F0BDF9A8F10208BDF81800C4EB83
:101F2800080802F083F901261FFA88F808E0A919C1
:101F3800601C80B289B24246002302F0A7F901363C
:101F48007B1B9E42F3D3BDE8F081F8B5C7B21446B7
:101F580038461E460D4602F09FF9621E92B2384678
:101F6800294602F099F9304602F060F9022606E0A7
:101F7800A21B92B23846294602F08EF90136A642D3
:101F8800F6D3F8BD70B5044600F11E003C220023CC
:101F980080B20D4602F07AF91E3DA9B220463C22D5
:101FA8000123BDE8704002F071B970B504460138EC
:101FB8000322002380B20D4602F068F9013DA9B260
:101FC800204603220123BDE8704002F05FB9F7B54F
:101FD800089D2E7BEF7A1C463604AB7A06EB072663
:101FE800F618431A687B06EB00602D180020019054
:101FF800121B08462146009501F098FEFEBD30B53B
:10200800456885B004AB03E906007DB101242C7353
:102018006D68BDF80800BDF80A109DF80C209DF801
:102028000E300095FFF7D3FF204600E0284605B0A4
:1020380030BD2DE9F04385B004AB03E906004468E0
:10204800BDF80860BDF80C70002C41D0012384F85D
:10205800263094F825300BB9A26800E06268FFB218
:10206800BDF80A109DF80E30009230463A46FFF748
:10207800AEFF04F10C08022002F0CEF9404611F040
:10208800F7F8054600B1451E0F3F0024153E1FFA1C
:1020980087F90DE002F0CAF902F0CEF904FB1061ED
:1020A80089B248462022002302F008FA0134E4B23B
:1020B800AC42EFD3002002F0B9F8B8B2B1B2424650
:1020C800012302F0FBF9002002F0A6F9012000E04C
:1020D800204605B0BDE8F0832DE9F04385B004AB98
:1020E80003E906004568BDF80860BDF80C70002DCE
:1020F8003CD001236B762B7EBDF80A10012B0CBF58
:102108006A68AA689DF80E300092FFB23A463046D7
:10211800FFF75DFF0C35022002F07EF9284611F02A
:10212800A7F80E3F81460024163E1FFA87F80DE0F7
:1021380002F07CF902F080F904FB106189B2404694
:102148002022002302F0BAF90134E4B24C45EFD959
:10215800002002F06BF8B8B2B1B22A46012302F0AF
:10216800ADF9002002F058F9012000E0284605B03A
:10217800BDE8F0832DE9F04F85B00546DDF84090C5
:10218800029148469046039311F072F8DDF838A0A2
:10219800DDF83CB00646294600242F4611E024B15C
:1021A800B4420CBF5B46534600E0039B01F10805AF
:1021B800ADB200932846029A4346FFF708FF013460
:1021C8002946B442EBDD002002F030F8022002F08C
:1021D80023F97D1D08F10508A8B21FFA88F14A46BF
:1021E800012305B0BDE8F04F02F04EB970B5406864
:1021F80086B006AB03E9060000282ED0012380F83C
:102208002D308668164BF21A534243EB020390F8BE
:102218002C205AB1002B134D134B144A08BF1D46EE
:10222800134B00F11C0418BF13460AE0002B0D4D98
:102238000D4B0E4A18BF1D460D4B00F10C0408BF8C
:102248001346BDF81200BDF81410BDF8162000960C
:1022580001950294FFF78EFF012006B070BD00BF04
:10226800F02404082C210408D22604080E230408AC
:10227800B428040870B5446886B006AB03E90600C4
:1022880004B301236377A668104B227FF11A4B42EF
:1022980043EB01030AB10BB904E01BB966680C4DA6
:1022A8000C4B01E00C4D0D4BBDF81200BDF814109D
:1022B800BDF8162000960C3401950294FFF75AFFDA
:1022C800012000E0204606B070BD00BF3C30040885
:1022D800782C04085A2E04081E3204080034040816
:1022E8002DE9F04385B004AB03E906004468BDF866
:1022F8000860BDF80A90BDF80C50BDF80E80002C9F
:1023080000F08C800123A3740220676802F084F82F
:102318004FF6FF7001F0A0FF002001F087FFEDB23B
:102328005FFA88F8A6F1160189B230462A46434674
:102338000097FFF74CFE277A002F2ED1A28A23465A
:1023480000E00137974204D29969097E04330029D5
:10235800F7D002F06BF802F06FF8A9F116091FFA2E
:1023680089F90E2101FB10914FF6FF7208F101085F
:102378005FFA88F389B2009248462A46FFF7B5FD0E
:10238800022002F049F81F2001F050FFA38A002B19
:1023980038D0103DE8B2303E2CE0E3685C68A28A91
:1023A8002346013A002700E00137974204D2996991
:1023B800097E04330029F7D002F038F802F03CF81F
:1023C8000E2101FB10914FF6FF7208F101085FFA28
:1023D80088F389B2009248462A46FFF786FD022014
:1023E80002F01AF81F2001F021FFA38A53B1103D13
:1023F800E8B21A3E0637B1B254F827200123083252
:1024080002F05CF8002002F007F84FF6FF7001F0C8
:1024180023FF1F2001F00AFF012000E0204605B03D
:10242800BDE8F0832DE9F04105463620884614467C
:102438001F4610F025FB0646E0B120F8025B414636
:102448002E22FFF717FCBDF8183086F83440738643
:102458001820012386F8307086F8313010F010FB10
:10246800044618B104234660037404E0304610F0B3
:102478000FFB00E004462046BDE8F081F8B50646AB
:1024880024200F46154610F0FBFA0446D8B10F4B2E
:10249800068083600E4B39464360102200F10C0021
:1024A800FFF7E8FB012600231820256223776677CB
:1024B80010F0E6FA054610B14460067404E02046C0
:1024C80010F0E6FA00E005462846F8BD3C3004085E
:1024D800962A0408F8B506462C200F46154610F033
:1024E800CFFA0446E8B120F80C6B39461922FFF7F9
:1024F800C1FB0D4BA562A3600C4B6360002384F8FD
:1025080025301820012384F8263010F0B9FA054642
:1025180018B103234460037404E0204610F0B8FAAD
:1025280000E005462846F8BD6C4904080A46040838
:1025380010B50446142010F0A3FA20B100234380FC
:10254800014B0480036110BDA11D000838B5054684
:10255800442010F095FA0446C0B10E4B0582436042
:102568000D4B0360012383740023037283820B4B9A
:102578000364182010F084FA054618B10723446054
:10258800037404E0204610F083FA00E0054628466C
:1025980038BD00BF00420408F63D0408951E000837
:1025A8002DE9F04105463420884614461F4610F0B0
:1025B80067FA064620B3144B05808360134B4146E7
:1025C8004360102200F10C00FFF754FB214606F18E
:1025D8001C001022FFF74EFB002386F82C30182031
:1025E8000123376386F82D3010F04AFA044618B1F3
:1025F80005234660037404E0304610F049FA00E011
:1026080004462046BDE8F081F02404084A1F040867
:102618002DE9F041044614200D461646984610F060
:102628002FFA0746B8B1069B048003610023C372E2
:1026380001234560068180F80A800373182010F092
:102648001FFA044618B106234760037404E03846AD
:1026580010F01EFA00E004462046BDE8F0812DE99E
:10266800F041044618200D461646984610F008FA20
:102678000746B8B101238370069B04800361079B5A
:1026880045608660C0F80C804361182010F0F8F9A6
:10269800044618B108234760037404E0384610F074
:1026A800F7F900E004462046BDE8F0812DE9F34142
:1026B80098461B8B1D2B05460C4617464FF000000D
:1026C80000F2B480B5F5A07F0090019000F2AE80D2
:1026D800F02900F2AB80127CADF80610511EADF85F
:1026E8000250072900F28A80DFE801F045595E04AC
:1026F800456A14767B684E4A7A611A8893F83430B2
:102708003A80013BDBB2012B7FD8ADF80240ADF82F
:1027180006507AE005F11602ADF8002004F1160221
:10272800ADF8042002AE434A16E903007A6107F1C6
:10273800080282E8030003F10802013348F8227016
:10274800A8F818307B681A8A187A3A8000286CD161
:10275800FFF7FCFE3849436859603849DF600126B5
:10276800163D196002461E72A8B2E1B24346FFF751
:102778009DFF30465AE0012A0CBF314B314B786837
:102788007B6130F80C3B3B8010F072FD431CDB0092
:102798001A34ED18ADF80440ADF8005035E07B6808
:1027A800294A1B687A6102E0284A7B687A611B889B
:1027B80014353B80ADF800501434ADF8044024E0E3
:1027C8007B68234A7A611A883A801A899B7AAD18FD
:1027D800ADF80050E418F0E77E681E4B7B61338843
:1027E80038463B8073689847013D4519ADF800505D
:1027F800B36838469847013C0419DEE71648174A7B
:10280800174B40F21A3100F0E3FC02AA12E9030068
:1028180007F1080383E80300B8F8183003F1080249
:10282800013348F82270A8F818300120BDE8FC816F
:10283800251E0008E9220008EC390408E2350408DE
:102848007D220008F5210008E12000083B2000084F
:1028580007200008B11B00088B9B0508901B040883
:10286800899B0508F8B51646002834D01378002B44
:102878002ED0028B002327E0046A257C042D21D169
:1028880065682F888F421DD195F8313053B16F8E0E
:1028980001F0F2FC04F1080268866369204606CA62
:1028A80098476F86A81C31462E22FFF7E3F995F862
:1028B80031307BB104F108026369204606CA9847A3
:1028C8000120F8BD013304309342D5D30020F8BD70
:1028D8001846F8BD0120F8BD70B5B8B1068B04469E
:1028E800002310E0256A287C04280AD16D6828880E
:1028F800884206D11046A91C2E22FFF7BBF90120F9
:1029080070BD01330434B342ECD3002070BD38B538
:10291800044620B3134BC361134BC0F89830134BD4
:10292800C0F89C30124B00257822C0F8A03085757D
:10293800C5750583294600F1200010F093FBD4F8F3
:1029480098302046294698470A4A1388312B07D8D9
:10295800094941F8234001331380012038BD38BDAF
:10296800284638BD3D1C0008351C0008D51B00084A
:10297800AB1C00087C0B00207C1300202DE9F041E3
:102988000446002800F0B380078B02460025A8E023
:10299800136A1E7C042E00F08780012E23D158680C
:1029A80003888B4240F09B8005F1080710F070F80F
:1029B80054F827004FF00008C0F8048010F068F8B9
:1029C800228B531E9D4208D00732238354F82210CD
:1029D80044F8271044F8228002E044F82780258331
:1029E8003046BDE8F081052E5ED0032E5CD0022E65
:1029F80013D15B68186803888B4270D14388013B08
:102A08009BB243800BB910F043F805F1080654F85F
:102A18002630586810F03CF84EE0072E21D15E6849
:102A2800338A8B425BD1002706E0BB1D013756F87D
:102A3800230010F02DF8FFB2B38ABB42F5D8002767
:102A4800B78205F1080654F82630586810F020F8C7
:102A580054F8260033E044F8267025830120BDE8A9
:102A6800F081062E1ED1586803888B4237D105F1B4
:102A7800080610F00DF854F826000027476010F0FB
:102A880007F8228B531E9D4209D00833013A54F8A7
:102A98002310228344F8261044F82370DEE744F814
:102AA80026701AE0082E1AD1586803888B4216D16E
:102AB8000FF0EEFF05F1080654F8260000274760DE
:102AC8000FF0E6FF228B531E9D42C4D0073254F804
:102AD800221044F8261044F822702383BEE70135FB
:102AE8000432BD42FFF454AF0020BDE8F081BDE8D8
:102AF800F08170B5044600282AD0068B751E08366A
:102B080000EB86061EE056F8043D1A7C042A13D012
:102B1800012A11D0052A0FD0032A0DD0022A02D18A
:102B28005B681B6809E0072A02D15B68198A05E01F
:102B3800062A01D0082A04D15B6819882046FFF7C5
:102B48001DFF013D681CDED100232383012070BDD9
:102B580070BDF0B528B30023068B1A461EE0046A40
:102B6800257C072D18D16468258A8D4214D1A78A3F
:102B7800002504EB83040DE004EB050C0435DCF8B8
:102B880018C09CF818C0BCF1010F03F1010301D172
:102B9800D8B2F0BDBB42EFD301320430B242DED32B
:102BA8000020F0BD70B508B3048B00231BE0026A57
:102BB800157C072D15D15268158A8D4211D1002335
:102BC800958A11461C46012007E013B996693076AC
:102BD80001E08E69347601330431AB42F5D301202C
:102BE80070BD01330430A342E1D3002070BD2DE94C
:102BF800F04128B30023078B1A461EE0046A257C9F
:102C0800072D18D16468258A8D4214D1B4F814C0F0
:102C1800002504EB83040CE066190435B66996F8C0
:102C28001880B8F1010F03D106F10800BDE8F08162
:102C380001336345F0D301320430BA42DED30020B9
:102C4800BDE8F0812DE9F04700282FD00023B0F827
:102C580018C01D4627E0046A267C072E21D1646827
:102C6800268A8E421DD1B4F81480002604EB83090D
:102C780015E009EB0604A7693C7E012C0DD192F8FA
:102C880000A0BAF1000F08D007F108001146102281
:102C9800FEF7F0FF2046BDE8F087013304364345D0
:102CA800E7D3013504306545D5D30020BDE8F0876A
:102CB800F0B5B0B1068B002510E0046A277C062F1A
:102CC8000AD1646827888F4206D123819DF8143081
:102CD8006260A3720120F0BD01350430B542ECD327
:102CE8000020F0BD10B500210446FEF7A3FF2046E2
:102CF8000121BDE81040FEF79DBF38B598B1048B9F
:102D0800024600230CE0106A058804328D4206D181
:102D180000F10802436906CA9847012038BD01330B
:102D2800A342F0D3002038BD10B50C460021FEF7B1
:102D380081FF20460121BDE81040FEF77BBF13B597
:102D480002AC04E90C00BDF80230834206D8BDF895
:102D58000030834234BF0020012000E00020BDF88D
:102D680006308B4206D8BDF804308B4234BF0021B0
:102D7800012100E00021002818BF0846C0B21CBD90
:102D880038B5114B114A1988002319E052F8045F2D
:102D9800A87D012812D100240CE004F1080355F89D
:102DA8002300037C082B03D1436800211B69984743
:102DB8000134A4B22B8BA342EFD838BD01339BB2A8
:102DC8008B42E3D138BD00BF7C0B00207813002074
:102DD800704770B5094CA5787DB9094B1E78012E4E
:102DE8000BD16368013363606268064B9A4204D969
:102DF800284601F0D3FAA670656070BD7C0B0020F0
:102E08003000002040420F00054A9060134602E05F
:102E180099680139996091680029F9D1704700BF14
:102E28007C0B0020F0B585B001F066FD002800F0AD
:102E38004981002502A80DF10A01ADF80850ADF846
:102E48000A5001F05BFD03A80DF10E01ADF80C501E
:102E5800ADF80E5001F09EFDBDF80C10BDF808202D
:102E68000091BDF80E10BDF80A3001912C46964D20
:102E78009649082005F0D2FFA878012803D101F06F
:102E88008DFAAC7019E1924B5B78012B40F01581FB
:102E9800AB78002B40F011816B6029888D4A09E1DD
:102EA80052F8046FB07D012840F002810025FAE055
:102EB80005F10803BDF8080056F82340BDF80A10CC
:102EC80004F108030CCBFFF73AFF002800F0E98073
:102ED800237C013B062B00F29F80DFE803F00429E6
:102EE800159D1F9D4C006668012304F10805337782
:102EF80095E8060063692046984700233377204603
:102F0800636995E8060086E0636893F8252012F166
:102F1800FF3218BF012283F8252077E0636893F811
:102F28002C2012F1FF3218BF012283F82C206DE00B
:102F38006268137E1568002B6ED16E882F4629466D
:102F4800184606E051F804EFDEF804E001338EF885
:102F58001800B342F6D301231376002607E057F88A
:102F6800040F00F10802436906CA984701366B88C6
:102F78009E42F4D350E0656820892E68A37B227BAB
:102F88000096A0F1160189B2FFF721F81420FFF787
:102F98003BFF2B7AC3B9AF8A29461A461E4609E079
:102FA800886990F818E00676BEF1010F08BF13464D
:102FB80004310132BA42F3D301220BB9AB6924E0E0
:102FC800053355F8233020E06368DB685A6800232E
:102FD800908A154619461F4609E0AE6996F818E02A
:102FE8003776BEF1010F08BF0B4604350131814227
:102FF800F3D3411E8B4203D1053052F8203003E051
:1030080004D2073352F8233001221A7604F1080259
:1030180006CA636920469847237C013B072B4CD896
:10302800DFE803F00410074B0A0D123A63681B6AC5
:1030380034E063689B6A2DE063681B6B2AE0636871
:103048001B6927E0636824E063681A7A7AB9988A6A
:103058001946013800E00132824204D28C69247E8C
:103068000431002CF7D0063253F8223011E0DB6827
:103078005A68908A11460138002300E001338342E0
:1030880004D28C69247E0431002CF7D0063352F820
:103098002330DB69984710E06368DB68204698476F
:1030A8000BE00135ADB2338BAB423FF601AF04E024
:1030B80001339BB28B427FF4F3AE01F063FC0F2027
:1030C800FFF7A2FE05B0F0BD7C0B0020B19B050800
:1030D8003000002078130020034B9A6812B19A68D8
:1030E800013A9A60704700BF7C0B00202DE9F34736
:1030F8000120DFF8D080DFF8D090014609F0B6FF54
:103108000025012403234FF48076022740466946B0
:103118008DF8053000968DF804708DF806508DF8FE
:10312800074009F0FBFB40460821224609F076FCDF
:10313800234BDFF898801A6844F2A243B2FBF3FAF3
:103148000AF1FF3A204621461FFA8AFA09F0BEFF23
:10315800C8F804A048464146A8F80050A8F802500C
:10316800A8F8085088F80A500AF04CFB7023A8F811
:103178000C300423A8F810300AF1FF3A63236422C4
:1031880003FB0AF3B3FBF2F39BB2C8F8143008F15F
:103198000C014846A8F80E40A8F81870A8F81A506C
:1031A800A8F81C60A8F81E500AF04AFC48462146B8
:1031B8000AF0BDFB484621460AF0C3FEBDE8FC877D
:1031C800A401002000000240000001408C0B0020F8
:1031D80083B50E460746154910201C46154605F0CE
:1031E8001DFE1020124905F019FE1020114905F0A6
:1031F80015FE10200E4905F011FE002310200E497F
:10320800019305F00BFE334610200C493A4605F0B1
:1032180005FE10200A492A4605F000FE102009493B
:10322800224605F0FBFD019B0133E7E7EB9B050810
:10323800F09B0508109C0508209C0508309C050893
:10324800459C0508569C050808B5164B1A6A0132B4
:103258001A621A6A012A1A4603D013484FF4A07159
:103268000FE05862194602E04B6A013B4B62506A14
:103278000C4B0028F8D11A6A012A06D00A4840F2F5
:103288004B110A4A0A4BFFF7A3FF1A6A013A1A625E
:103298001B6A2BB10448054A064B40F24D11F2E770
:1032A80008BD00BF8C0B0020679C050892530408DA
:1032B800919C0508A29C05080C4B0D491A6844F21C
:1032C800A2436428B2FBF3F3D4BF20EAE070642081
:1032D800013B9BB24B60013B58436422B0FBF2F0C8
:1032E80080B2486103480C310AF02DBBA4010020CC
:1032F8008C0B00200000014010B5134B93F82820D8
:103308002AB11248124A134B4FF40A710EE00122F7
:1033180083F8282066234FF0C042013BDBB21080BF
:1033280033B90A480A4A0C4B40F23221FFF750FFE2
:103338001488A4B28442F0D1084B1980024B0022B1
:1033480083F8282010BD00BF8C0B0020679C05085F
:103358009C530408B39C0508899B0508000002607B
:1033680010B5FFF7C3FE6420FFF7A6FFE5204FF472
:103378000041FFF7C1FF00200121FFF7BDFF012039
:103388004FF48071FFF7B8FF02204FF4E061FFF7B8
:10339800B3FF032041F23001FFF7AEFF0420002104
:1033A800FFF7AAFF082040F20221FFF7A5FF092036
:1033B8000021FFF7A1FF0A200021FFF79DFF0C2045
:1033C8000021FFF799FF0D200021FFF795FF0F203F
:1033D8000021FFF791FF10200021FFF78DFF11203A
:1033E8000021FFF789FF12200021FFF785FF132036
:1033F8000021FFF781FF102041F2B071FFF77CFF39
:1034080037211120FFF778FF3220FFF71DFF122028
:1034180040F23B11FFF770FF3220FFF715FF132032
:103428004FF4C051FFF768FF0F212920FFF764FF11
:103438003220FFF709FF20200021FFF75DFF212040
:103448000021FFF759FF30200021FFF755FF3120F9
:103458000721FFF751FF322040F20311FFF74CFF1D
:10346800352040F20741FFF747FF40F20444362079
:1034780040F60F11FFF740FF37202146FFF73CFFCA
:1034880038204FF48061FFF737FF39202146FFF7D6
:1034980033FF3C200021FFF72FFF3D204FF48061D0
:1034A800FFF72AFF50200021FFF726FFEF215120C8
:1034B800FFF722FF52200021FFF71EFF532040F2A2
:1034C8003F11FFF719FF60204FF41C51FFF714FF5D
:1034D80061200121FFF710FF6A200021FFF70CFF90
:1034E80080200021FFF708FF81200021FFF704FF5B
:1034F80082200021FFF700FF83200021FFF7FCFE58
:1035080084200021FFF7F8FE85200021FFF7F4FE54
:1035180090201021FFF7F0FE92200021FFF7ECFE2B
:1035280093200321FFF7E8FE95204FF48871FFF7F9
:10353800E3FE97200021FFF7DFFE98200021FFF728
:10354800DBFE072040F27311BDE81040D4E610B549
:10355800FFF7CCFD6420FFF7AFFE21210720FFF71E
:10356800CBFE3220FFF770FE01210020FFF7C4FEDA
:103578003220FFF769FE23210720FFF7BDFE322026
:10358800FFF762FE00211020FFF7B6FE40F6B830C4
:10359800FFF75AFE33210720FFF7AEFE3220FFF770
:1035A80053FE112046F63001FFF7A6FE3220FFF742
:1035B8004BFE4FF4C0610220FFF79EFE3220FFF75A
:1035C80043FE122046F6EB41FFF796FE3220FFF746
:1035D8003BFE03204AF6A401FFF78EFE3220FFF7D8
:1035E80033FE00210C20FFF787FE3220FFF72CFE68
:1035F8000D2040F60C01FFF77FFE3220FFF724FE76
:103608000E204FF42C51FFF777FE3220FFF71CFEF7
:10361800B0211E20FFF770FE3220FFF715FE0120B3
:1036280042F63F31FFF768FE3220FFF70DFE052016
:103638000021FFF761FE3220FFF706FE0021062079
:10364800FFF75AFE3220FFF7FFFD16204EF61C71D9
:10365800FFF752FE3220FFF7F7FD172040F2031163
:10366800FFF74AFE3220FFF7EFFD00210B20FFF79E
:1036780043FE3220FFF7E8FD00210F20FFF73CFE54
:103688003220FFF7E1FD41200021FFF735FE32200F
:10369800FFF7DAFD42200021FFF72EFE3220FFF768
:1036A800D3FD00214820FFF727FE40F23F143220C7
:1036B800FFF7CAFD21464920FFF71EFE3220FFF71B
:1036C800C3FD00214A20FFF717FE3220FFF7BCFD9B
:1036D80000214B20FFF710FE3220FFF7B5FD4420F4
:1036E8004FF46F41FFF708FE3220FFF7ADFD0021D0
:1036F8004520FFF701FE3220FFF7A6FD21464620B0
:10370800FFF7FAFD3220FFF79FFD302040F20771E6
:10371800FFF7F2FD3220FFF797FD31204FF40171DA
:10372800FFF7EAFD3220FFF78FFD32204FF40171D9
:10373800FFF7E2FD40F202543220FFF785FD2146F3
:103748003320FFF7D9FD3220FFF77EFD342040F209
:103758000751FFF7D1FD3220FFF776FD35204FF4F2
:103768000171FFF7C9FD3220FFF76EFD36204FF4D7
:103778000171FFF7C1FD3220FFF766FD21463720B2
:10378800FFF7BAFDA4F500743220FFF75DFD21466E
:103798003A20FFF7B1FD3220FFF756FD2F2041F206
:1037A800BE21FFF7A9FD3220FFF74EFD21463B2041
:1037B800FFF7A2FD3220FFF747FD00212320FFF786
:1037C8009BFD3220FFF740FD00212420FFF794FDE8
:1037D8003220FFF739FD25204FF40041FFF78CFD1B
:1037E8003220FFF731FD00214F20FFF785FD322001
:1037F800FFF72AFD4E200021FFF77EFD3220BDE8AD
:10380800104021E508B5124B93F829202AB1114838
:10381800114A124B40F242210FE0012283F829207D
:10382800222166234FF0C042013BDBB2118033B93D
:103838000848094A0A4B40F25B21FFF7C9FC108887
:1038480080B22228F0D1024B002283F8292008BD3B
:103858008C0B0020679C0508A9530408B39C050835
:10386800899B050810B5224B49F22032032823D83A
:10387800DFE800F0021A0B111C8846F6280041F216
:103888002801944218BF01461AE01C8841F208003A
:1038980046F6080104E01C8841F2300046F6300183
:1038A800944208BF01460BE0188846F62001904272
:1038B80008BF4FF4815103E00E4840F2792113E02C
:1038C8001B8848F68912934205D049F22032934268
:1038D80007D1032000E01120FFF70EFDBDE81040DE
:1038E80090E7044840F28521034A044BFFF770FC37
:1038F80032000020679C0508BE530408899B050810
:10390800014B18800A209FE4000002604FF0C0437A
:10391800188003F500331A881A88188880B270470F
:103928002DE9F041022098B00121002409F09EFB06
:10393800012502268C488DF85C5016A98DF85E404A
:103948008DF85F4016968DF85D6008F0E7FF182047
:10395800294609F08BFB2846294609F09FFB21469A
:103968000C22824809F05AF829460C227F4809F0AF
:1039780055F804210C227D4809F050F805210C2245
:103988007A4809F04BF807210C22784809F046F8E4
:1039980008210C22754809F041F809210C227348C6
:1039A80009F03CF80A2171480C2209F037F80B217C
:1039B8006E480C2209F032F80E210C226B4809F0EF
:1039C8002DF80F210C22694809F028F807210C224C
:1039D800674809F023F808210C22654809F01EF809
:1039E80009210C22624809F019F80A210C226048C2
:1039F80009F014F80B210C225D4809F00FF80C218E
:103A08000A465B4809F00AF80D210C22584809F0CB
:103A180005F80E210C22564809F000F80C225448EB
:103A28000F2108F0FBFF03274CF6B3734F4816939A
:103A380016A98DF85D708DF85E408DF85F408DF8A1
:103A48005C6008F06BFF4FF6807316A94848169320
:103A58008DF85D708DF85E408DF85F408DF85C6084
:103A680008F05CFF40F6B830FFF7EEFB224631461F
:103A78003D4808F0C8FF44F6FF70FFF7E5FB2A460B
:103A88003146394808F0BFFF40F6B830FFF7DCFB95
:103A98004FF48053102709930DF13C084FF400238D
:103AA80068460F94109412941395149415940094E6
:103AB8000194029404940694079408940A94059433
:103AC8000B940C9311960397CDF8348008F09FFC63
:103AD8000423684611931094129413951494159422
:103AE8000F96CDF8388008F092FC2946204608F059
:103AF8000EFD40F6B830FFF7A7FB2046FFF706FF9C
:103B080004461C491C4D3846224605F087F948F6FC
:103B180089139C421AD049F220339C420DD041F2BD
:103B280089239C4212D03846144905F077F9144885
:103B3800144A154BA621FFF74BFB3846134922467A
:103B480005F06CF92C80FFF70BFC0AE0FFF7FFFC8F
:103B580048F689122A8010200D4941F2892305F080
:103B68005DF918B0BDE8F08100040240000C024085
:103B780000100240C89C050832000020DF9C0508A0
:103B8800679C0508D6530408899B0508169D0508F7
:103B98004B9D05084FF0C04322221A8003F50033DD
:103BA80082B01A8892B2ADF806201B889BB2ADF895
:103BB8000630BDF8060080B202B07047134B1B8870
:103BC80048F68912934210B504460BD049F22032C8
:103BD800934213D1C1F1EF01202089B2FFF78CFB8A
:103BE800212006E0C1F1EF014E2089B2FFF784FBE6
:103BF8004F202146BDE81040FFF77EBB0448054A28
:103C0800054B40F2F321FFF7E3FA00BF3200002032
:103C1800679C0508DF530408899B05082DE9F041D6
:103C28000D46C5F1F008411E5E18C2EB0802C5F149
:103C3800EF039BB292B2B6B29A422CBF9046984616
:103C48009A4234BF11461946864234BF3746074662
:103C580040F23F13864238BF06469E4228BF1E46A2
:103C68001B4B1B8848F68912B8F1EF0F28BF4FF09D
:103C7800EF089342044610D049F2203293421FD1F4
:103C88005020FFF739FB51204146FFF735FB522002
:103C98003946FFF731FB53200AE041EA082189B28F
:103CA8004420FFF729FB45203946FFF725FB46202E
:103CB8003146FFF721FB20462946BDE8F0417DE764
:103CC8000448054A054B40F2DD21FFF781FA00BFA1
:103CD80032000020679C0508ED530408899B0508FD
:103CE80000200146F0224FF4A07397E7072040F226
:103CF8007311FFF701BB07200021FFF7FDBA10B5CC
:103D08001446FFF75BFFFFF77DFD2046BDE8104036
:103D1800F6E508B5FFF752FF4FF0C04322221A809C
:103D280003F500331A88188880B208BDF8B580B248
:103D380002FB03F589B292B29BB2069C9DF81C6007
:103D4800FFF76CFF0020FFF78DFD002709E034F82E
:103D5800020B1EB1030A43EA002080B2FFF7D0FD30
:103D68000137AF42F3DBBDE8F840B9E72DE9F74F7B
:103D780016469DF834200C9F01920546B2B280B2D7
:103D88000C46984689B29BB2FFF748FF4FF0000BEC
:103D98000020FFF767FDDA463DE0002D30DB09EB38
:103DA800050340F23F1293422ADC002C28DB0BEB80
:103DB8000403EF2B24DC19F00F0F04D1B9F1000F25
:103DC800C8BF0AF1010A174B09EA0303002B03DAFB
:103DD800013B63F00F030133019A0AB1C3F10F03EA
:103DE800012202FA03F337F81A2013401BB213B169
:103DF8000D4B588D01E00D4A508880B2FFF780FDC9
:103E080009F1010901E04FF00009C145C5DB0AF1DC
:103E1800010A0BF1010BB345F5DB03B0BDE8F04F28
:103E28005EE700BF0F0000808C0B002032000020EE
:103E38002DE9F04F85B004469DF83C00029200271A
:103E48008A46039088463E4640F23F1C9B463AE02D
:103E5800002C2FDBE1452DDCBAF1000F2ADBB8F18D
:103E6800EF0F27DC2A0702D1002DC8BF01361B49F6
:103E78002940002903DA013961F00F010131039A61
:103E88000AB1C1F10F010E9830F8162003FA01F1BA
:103E98000A4012B272B112494A8D019392B21FFAC6
:103EA80089F01FFA88F1CDF800C0FFF728FFDDF888
:103EB80000C0019B013509F101095D45C8DB0136E8
:103EC800013708F10108029A974203DAA146002552
:103ED8000123F2E705B0BDE8F08F00BF0F000080B6
:103EE8008C0B002082B0044BADF80600BDF806200C
:103EF80092B25A8502B070478C0B002082B0044BF6
:103F0800ADF80600BDF8062092B25A8002B070479C
:103F18003200002070B50646FFF7E2FE0020FFF7EA
:103F2800A1FCF02409E0013D3046ADB2FFF7E8FC02
:103F3800002DF8D1013CA4B214B14FF4A075F2E7FA
:103F480070BD70B51D461446FFF738FE2846FFF7CA
:103F580089FC0025054E05E0708D80B2FFF7D0FC86
:103F68000135ADB2A542F7D170BD00BF8C0B002062
:103F78002DE9F0410C4616461F461A460023054611
:103F8800FFF7DFFF611E711828463A46002389B201
:103F9800FFF7D7FF2846214632460123FFF7D1FF16
:103FA800013D7F19B8B2214632460123BDE8F041F0
:103FB800C7E770B580B202FB03F489B292B29BB234
:103FC800FFF72CFE0020FFF74DFC0025054E04E00E
:103FD800708D80B2FFF794FC0135A542F8DBBDE88F
:103FE80070407DE68C0B0020F8B5561A0C4601315E
:103FF80089B21F460546FFF7E1FD0120FFF732FCB5
:104008004FF0C04322221A800E4A0F491388B6B2D5
:10401800002304E01088013321F8020B9BB2B3425D
:10402800F8D121462846FFF7C9FD0120FFF71AFC01
:10403800002404E03846FFF763FC0134A4B2B4421C
:10404800F8D1F8BD00000260624D002070B5194B30
:10405800194AD98D92F9004064180025A4B2AC42DF
:1040680008BF0124C62C28BFC6240F2615704FF69A
:10407800FF7288B09E85DC855A8519200A222B4656
:104088002146FFF75EFF21463046FFF742FE2246F3
:1040980003460A4968460FF065F86A4604A80849C5
:1040A8000FF060F83220D22104AA2B4600F0ECF978
:1040B80008B070BD8C0B0020282A00208A9D0508B6
:1040C800929D05082DE9F0431F2093B0FFF722FFCA
:1040D8004FF47840FFF71EFF4FF6E0754FF4FC6091
:1040E800FFF718FF2846FFF715FF0020494CFFF798
:1040F80011FF00200146642203464FF6FF79A4F819
:104108002A90FFF71EFF00200A2164220346FFF7CA
:1041180018FF00200146642201234FF47847658583
:10412800FFF70FFF7720EF21C82200234FF4FC662A
:104138006785FFF706FFBD213222012340F23F10B9
:104148006685FFF7FEFEA0203222002378216785CE
:10415800FFF7F7FEA0207821322201234FF01F0835
:104168006685FFF7EEFEA020782132220223A4F80C
:104178002A80FFF7E6FEA0207821322203236585F6
:10418800FFF7DFFE244B2549A3F8028002AD3C224D
:1041980028460EF025FFEB20C32105223023009589
:1041A8000025A4F82A900195FFF7E0FD32210A20A6
:1041B80096220B466785FFF7DBFE32213C209622CC
:1041C8000B466685FFF7D4FE32210B4696226E20F9
:1041D800A4F82A80FFF7CCFEFFF78DFDFFF786FDD8
:1041E8003220FFF769F82846FFF766F86420FFF7E2
:1041F80063F80B4B03F110028DE8240028465A6837
:104208001B682946FFF792FD1195119B0133119305
:10421800FBE700BF8C0B002032000020025404088A
:1042280020780108004870474814002082B0064BE7
:10423800ADF80600BDF8062092B21A80188880B240
:1042480002B0FFF74FBE00BF44140020014B18888E
:1042580080B270474414002082B0064BADF80600C7
:10426800BDF8062092B21A80188880B202B0FFF713
:1042780045BE00BF46140020014B188880B2704725
:1042880046140020FFF746BEFFF7C8BCFFF759BE2B
:10429800FFF76EBEFFF78DBE2DE9F04F4FEA4208DB
:1042A80000253D4C85B082468B46C8F10308174669
:1042B8002E461FFA87F909EB0B0C228805EB0A0337
:1042C8001FFA8CFC9BB26146184692B2CDF804C026
:1042D8000293FFF714FDC9EB0B0292B20392029B03
:1042E80022880399184692B2FFF709FDDDF804C049
:1042F8002288C5EB0A039BB26146184692B2029324
:10430800FFF7FDFC029B22880399184692B2FFF73B
:10431800F6FC05EB0B0292B2039209EB0A03228822
:1043280003999BB2184692B20293FFF7E8FC029BEE
:104338002288C5EB0B0C1FFA8CFC1846614692B21A
:10434800CDF804C0C9EB0A09FFF7D9FC2288039904
:104358001FFA89F992B24846FFF7D1FC2288DDF8A6
:1043680004C092B248466146FFF7C9FCB8F1000F95
:1043780004DA08EB860808F1060805E0F31B08F1E3
:104388000A0808EB8308013F01360135BE42ADB289
:104398008FD905B0BDE8F08F4414002008B9FFF7A5
:1043A800AABC012801D1FFF7A1BC704770470020C3
:1043B8000146F0224FF4A073FFF730BC704708B5F0
:1043C80005280CD8DFE800F012140305070909488E
:1043D80008BD094808BD094808BD094808BD09487D
:1043E800094A0A4B40F24111FEF7F2FE084808BD9F
:1043F800084808BD20000020100000200800002008
:1044080000000020979D05083E540408899B050874
:10441800280000201800002010B50446FFF7CFFF41
:10442800014B18601C7110BD38000020014B187931
:10443800704700BF3800002008B5FFF7C0FF80882C
:1044480008BD08B5FFF7BBFFC08808BDF7B51F4614
:104458000B4B0C4E1D681446EA882B68203C5443CD
:10446800A4B2AE1B03EB440418BF0126AB888DE849
:10447800500017B1FFF7DCFC01E0FFF777FCFEBD49
:1044880038000020280000202DE9F0410F4698460A
:1044980015460446084E08E0204643463946FFF7CD
:1044A800D5FF33689B88E418A4B215F8012B002ABD
:1044B800F2D1BDE8F08100BF3800002010B50446F5
:1044C80008462146BDE81040DEE7094B70B50446B2
:1044D80018790E461546FFF7B4FFC6F1F001091A20
:1044E80089B220462A460023BDE87040CCE700BFC9
:1044F80038000020704700BF044B1A680AB9044A04
:104508001A601A681018186010467047BC0B002013
:10451800E46100204FF0FF30704708B50248034AB5
:10452800034B3721FEF754FEB69D05085454040882
:10453800899B05080120704710B504460A480221E6
:1045480009F01AF80028F9D00748214608F0DDFFDD
:104558000548012109F010F80028F9D00248BDE803
:10456800104008F0CFBF00BF0038004010B5194810
:10457800022109F001F80028F9D01648002108F0B6
:10458800C4FF1448012108F0F7FF0028F9D01148AA
:1045980008F0B8FF0402A4B2002301E001339BB283
:1045A800002BFBD00B48022108F0E6FF0028F9D0C9
:1045B8000848002108F0A9FF0648012108F0DCFF9F
:1045C8000028F9D0034808F09DFF2043C0F3CB0032
:1045D80010BD00BF003800402DE9F0478AB00AAF8F
:1045E8000A20012108F042FD4FF4604347F8143DCA
:1045F800474EDFF824A1012400254FF00208304679
:1046080039468DF81A508DF818808DF819808DF874
:104618001B4008F083F930460D21052208F0FEF909
:1046280030460E21052208F0F9F9052230460F21FF
:1046380008F0F4F921464FF4804008F03BFD50465D
:1046480008F016FE4FF48273ADF802304FF4007391
:10465800ADF80A303823ADF80C30504607236946C8
:10466800ADF81030ADF80050ADF80450ADF8065074
:10467800ADF80850ADF80E5008F02CFE5046214613
:1046880008F0C3FEA9468DF81A5030464FF48055FD
:10469800394605958DF818408DF819808DF81B401E
:1046A80008F03CF93046294608F0A9F94025394672
:1046B80018488DF818908DF819808DF81A908DF893
:1046C8001B40059508F02AF921464FF4804008F070
:1046D800FDFC0621032008F087FF0C2307A88DF8AE
:1046E800213007958DF820908DF8224007F00AFEBA
:1046F80017238DF8243009A80F238DF825308DF85D
:1047080026308DF8274004F017FD0AB0BDE8F08781
:1047180000040240000C024000380040014B1878A9
:10472800704700BFC00B0020024B5A889B8802804C
:104738000B807047C00B0020014B00221A70704795
:10474800C00B0020F0B593B06846002148220EF057
:1047580089FC6D46002464484FF4805108F051F9F3
:10476800002301E001339BB2002BFBD09020FFF720
:10477800E3FE002301E001339BB2002BFBD0FFF7DF
:10478800F5FE4FF480510746574808F038F90023E2
:1047980001E001339BB2002BFBD053484FF480510A
:1047A80008F02FF9002301E001339BB2002BFBD066
:1047B800D020FFF7C1FE002301E001339BB2002B9C
:1047C800FBD0FFF7D3FE4FF480510646464808F069
:1047D80016F945F8047B01342E6244484021E4B2BE
:1047E80008F0FBF810B9092CB5D101E0092C78D1F3
:1047F8009DE80C00D218029B03980699D218049BD6
:10480800C018059BC018079BCB180899032490FB78
:10481800F4F092FBF4F25B1893FBF4F3151AC11A47
:104828009C1A002DB8BF6D420029B8BF4942002C20
:10483800B8BF6442502D03DD502909DD502C50DCEF
:104848008D4205DAAC424FF0020405DB111806E090
:104858008C424FF0020401DAD11800E0C1180A9B1B
:10486800099A0C980F9DD2180B9BD2180D9BC01853
:104878000E9BC018109BEB18119D91FBF4F10324BB
:1048880092FBF4F290FBF4F05B1993FBF4F3161A25
:10489800C41A9D1A002EB8BF7642002CB8BF6442D5
:1048A800002DB8BF6D42502E89B203DD502C09DDB2
:1048B800502D16DCA64205DAB5424FF0020405DB9E
:1048C800131806E0A5424FF0020401DAD31800E0FD
:1048D800C318074A93FBF4F39BB2938001235180DA
:1048E800137013B0F0BD00BF00040240000C02407A
:1048F800C00B002000000000FFF710BFF7B5054609
:104908000C4601A80DF10601FFF70EFF1B4BBDF881
:104918000660BDF8040093E80600724301FB00221C
:1049280099685218164992FBF1F207EE102AF8EE30
:10493800C77A40F23F17FCEEE77A17EE902A92B258
:10494800B2F5207F28BF3A462A801D69DA685B697C
:104958006E4302FB0060C01890FBF1F107EE101ADD
:10496800F8EEC77AFCEEE77A17EE903A9BB2B3F509
:10497800F07F28BFEF232380FEBD00BFC80B0020B7
:1049880040420F00FFF7D8BE014B187E704700BFAA
:10499800C80B0020FFF7C8BE042808B505D907488A
:1049A800074A084B7D21FEF713FC054B03EB8000FB
:1049B800038B0B80438B138008BD00BFD79D050870
:1049C8005A540408F59D050808B5082001F090F927
:1049D80042F69643C31A584240EB030008BD10B58F
:1049E8000A2001F0ADF90C4C20600E2001F0A8F966
:1049F8006060122001F0A4F9A060162001F0A0F96F
:104A0800E0601A2001F09CF920611E2001F098F95D
:104A180001236061237610BDC80B002010B5FFF795
:104A2800DBFD01F02FFA044601F038FA0749034686
:104A38002246202004F0F2F9FFF7C6FF28B101F062
:104A48003BFA10B9BDE81040C9E710BD319E050812
:104A580010B5104C0A20216801F059F961680E2040
:104A680001F055F9A168122001F051F9E16816200A
:104A780001F04DF921691A2001F049F961691E20F8
:104A880001F045F9082042F69641BDE8104001F0D2
:104A980021B900BFC80B00202DE9F04F0346A7B08D
:104AA800B0F800C01C898688DF885D89CDF810C001
:104AB800B249B0F802C0B3F80C90B3F80E80CDF844
:104AC80024C00FFA84FB30B201220FFA87FE0BEBE9
:104AD800000C0A7629B20FFA89FACDF888C001EBE2
:104AE8000E0C0FFA88F2CDF890C00AEB0B0CCDF83B
:104AF80030C002EB010CCDF858C0B3F810C05B8A87
:104B0800CDF800C00FFA8CFC06910CEB00010A915D
:104B180002930CEB0A011BB2239103EB0E010E91D9
:104B280099182591049900FA81F05844504460443A
:104B3800DDF824C006990EFA8CFEDDF810C01FFAC5
:104B480080FB1CFB0CF08E4416FB0600964414FBFD
:104B58000400009A19FB09009E4412FB02001FFA88
:104B68008EFA09F013FEDDF824C0029ACDE912018D
:104B78001CFB0CF017FB070015FB050018FB0800D1
:104B880012FB020009F002FEDDF824C0029ACDE90A
:104B9800140104991CFB01F317FB063615FB046688
:104BA800009B18FB096612FB036009F0EFFDDDE9C5
:104BB8001423CDE90001DDE9120109F05DFE044688
:104BC8000D46DDE9000102460B4609F055FE024696
:104BD8000B462046294609F09BFCCDE918015846AA
:104BE80009F0E4FDCDE91001DDE91023DDE900015C
:104BF80009F042FECDE90601504609F0D7FD80468E
:104C080089464246DDE912014B4609F035FEDDE9E9
:104C18001023CDE91C01DDE9140109F02DFE002265
:104C280006460F46564BDDE9180109F025FE4246B7
:104C380004460D464B46DDE9060109F01DFE024615
:104C48000B4609F067FC02460B462046294609F048
:104C580061FC424604460D464B46DDE91C0109F05D
:104C68000BFE02460B462046294609F051FCDDE9B9
:104C7800102304460D463046394609F0FDFD02462C
:104C88000B462046294609F043FCDDF828C0CDE94B
:104C980002014FEA8C10DDF830C000EB0C20DDF883
:104CA80010C0A0241CFB040009F070FDDDF838C01A
:104CB800CDE90A014FEA8C10DDF858C000EB0C2052
:104CC800DDF824C01CFB040009F060FDCDE90C01EF
:104CD800504609F05BFDDDE91023CDE91601DDE959
:104CE8000C0109F0C9FD4246CDE91E014B46DDE93C
:104CF8000A0109F0C1FD4246CDE920014B46DDE934
:104D0800000109F0B9FD32463B4609F001FCCDE946
:104D18000E01584609F03AFDDDE91C23CDE91A01D8
:104D2800DDE9060109F0F4FBDDF88CC0C024CDE90B
:104D3800060104FB0CF0DDF888C0302505FB0C00EB
:104D4800DDF810C078261CFB060009F01FFDDDF811
:104D580094C0824604FB0CF0DDF890C005FB0C0003
:104D6800DDF824C01CFB06008B4609F00FFDDDE9C9
:104D7800102306460F4609F07FFD03E0C80B00200C
:104D8800000014404246CDE904014B4650465946BE
:104D980009F072FDDDE9142380468946DDE90A0140
:104DA80009F06AFDDDE9002304460D46DDE90C0142
:104DB80009F062FD02460B462046294609F0A8FB89
:104DC8000022A14B09F058FDDDE9202304460D46D9
:104DD800DDE91E0109F09CFB02460B46DDE91601E0
:104DE80009F04AFD02460B462046294609F092FB87
:104DF800002204460D46954BDDE90E0109F03CFD05
:104E080002460B462046294609F084FBDDE90223C9
:104E180009F05CFE88A3D3E9002309F02DFD09F011
:104E2800C5FF8B490860DDE91223DDE90C0109F0B3
:104E380023FDDDE9002304460D46DDE90A0109F0FA
:104E48001BFD02460B462046294609F061FB00225D
:104E58007D4B09F011FDDDE91E2304460D46DDE911
:104E6800200109F055FB02460B46DDE91A0109F05D
:104E780003FD02460B462046294609F04BFB00225B
:104E880004460D46714BDDE9060109F0F5FC0246C2
:104E98000B462046294609F03DFBDDE9022309F0CF
:104EA80015FE65A3D3E9002309F0E6FC09F07EFFAF
:104EB800674A5060DDE90E23DDE90A0109F0DCFCF0
:104EC800DDE9062304460D46DDE90C0109F0D4FCB2
:104ED80002460B462046294609F01CFB00220446E0
:104EE8000D465A4BDDE9180109F0C6FC02460B468F
:104EF8002046294609F00EFBDDE9022309F0E6FD0C
:104F08004DA3D3E9002309F0B7FC09F04FFF504B3C
:104F180059469860DDE91423504609F0ADFCDDE9F7
:104F2800002304460D463046394609F0A5FC0246E2
:104F38000B462046294609F0EBFA0022424B09F0BD
:104F48009BFC424604460D464B46DDE9040109F048
:104F5800DFFA02460B46DDE9160109F08DFC024630
:104F68000B462046294609F0D5FA35A3D3E9002394
:104F780004460D46DDE90E0109F07EFC02460B46AB
:104F88002046294609F0C6FADDE9022309F09EFD0C
:104F980029A3D3E9002309F06FFC09F007FFDFF824
:104FA800B0C0DDE91223CCF80C003946304609F0D0
:104FB80063FCDDE9002304460D465046594609F0D6
:104FC8005BFC02460B462046294609F0A1FA00225E
:104FD8001D4B09F051FCDDE9042304460D4640460B
:104FE800494609F095FA02460B46DDE91A0109F02F
:104FF80043FC02460B462046294609F08BFA10A3CB
:10500800D3E9002304460D46DDE9060109F034FC26
:1050180002460B462046294609F07CFADDE90223C0
:1050280009F054FD04A3D3E9002309F025FC09F095
:10503800BDFE074908610DE00000000080842E4194
:105048000000000000C082400000144000008940B9
:10505800C80B0020DDE90E235046594609F00CFC28
:10506800DDE9062304460D463046394609F004FCBE
:1050780002460B462046294609F04CFA11A3D3E90B
:10508800002304460D46DDE9180109F0F5FB024648
:105098000B462046294609F03DFADDE9022309F0CE
:1050A80015FD0AA3D3E9002309F0E6FB09F07EFE0B
:1050B800034A506127B0BDE8F04FC9E4AFF3008060
:1050C800C80B00200000000000C082400000000063
:1050D80080842E41AFF30080064B074A596811605F
:1050E8001969064A1160D969054A11609A6A054B1F
:1050F8001A607047400000208040002030410020A6
:105108008440002044400020014B1878704700BFBD
:10511800E40B0020032808B505D90548054A064BC5
:105128006E21FEF755F80C235843044B185808BD58
:105138006C9E050886540408869E050840000020D9
:10514800032808B505D90648064A074B7321FEF718
:105158003FF8064B0C2202FB0030406808BD00BF38
:105168006C9E050896540408869E05084000002099
:10517800034B044A1B780C2101FB032398687047F2
:10518800E40B002040000020034B044A1B780C204D
:1051980000FB032399607047E40B002040000020C7
:1051A800144B1B78012B10B5134B144C0ED11968F6
:1051B800C82000F0ACFD2168CC2000F0A8FD104B01
:1051C800D020196800F0A3FDD4200DE01968D8207C
:1051D80000F09DFD2168DC2000F099FD084BE020DF
:1051E800196800F094FDE420064B1968BDE81040EA
:1051F80000F08DBD000D00208040002030410020CF
:105208008440002044400020144B1B78012B10B52B
:10521800134C0FD1C82000F093FD2060CC2000F083
:105228008FFD104B1860D02000F08AFD0E4B1860DF
:10523800D4200EE0D82000F083FD2060DC2000F0B0
:105248007FFD084B1860E02000F07AFD064B1860DF
:10525800E42000F075FD054B186010BD000D00201E
:10526800804000203041002084400020444000203D
:1052780008B502F0FBF910B1BDE80840C4E708BD65
:105288000148FCF704B800BF301200200148FBF7C2
:10529800FEBF00BF301200200148FBF7F8BF00BF77
:1052A800301200200148FBF7F2BF00BF3012002087
:1052B800032808B505D91448144A154B4B21FDF7A6
:1052C80087FF144B1870144B02281870134B0FD01B
:1052D800032813D0012805D0114A12681A60BDE8C6
:1052E8000840CDE70F4A12681A60BDE80840CDE7CC
:1052F8000D4A12681A60BDE80840CDE70B4A1268EB
:105308001A60BDE80840CDE76C9E0508A75404085C
:10531800B09E0508E40B002076400020980100208C
:10532800900100208C0100208801002084010020C9
:10533800064B07495960C021002219721E211A70B4
:10534800D9601A745A611A76DA61704770140020AD
:1053580040787D0110B50321FF22C02001F078F8C4
:105368001F4C102120608022C02001F071F811210B
:1053780020608022C02001F06BF81221206080227A
:10538800C02001F065F8132120608022C02001F0C0
:105398005FF8142120608022C02001F059F81521FF
:1053A80020608022C02001F053F88022206016215E
:1053B800C02001F04DF82060C0201721802201F0A4
:1053C80047F82060074CC020227AB72101F040F846
:1053D8000023237463612376E3610123237010BDE6
:1053E800604000207014002038B5C0200321FF223F
:1053F80001F02EF80B4D00242B19615D5A78C0205E
:10540800023401F025F8C82CF6D1B121AC22C02015
:1054180001F01EF8C0200321002201F019F8002035
:1054280038BD00BFBB5404082DE9F34706460F46B4
:1054380092461D461AB90C1FE401914635E005EE67
:10544800902A06EE903AB8EE657AF8EE667AFC0194
:10545800C7EE277AA4F500749FED5C7A67EE877A29
:1054680017EE900A09F0B4F941EC100B0BF09CF917
:1054780059EC108B4946404609F0C0FC24184FEA05
:10548800CA1009F083F9CDE90001284609F07EF930
:105498004B46424609F0F0F902460B46DDE90001A9
:1054A80009F036F809F0AAFC8146002E14BF4FF027
:1054B80022084FF01A08C5F307224146C02000F021
:1054C800C7FF08F10101EAB2C02000F0C1FFC4F330
:1054D800014208F10201C02000F0BAFFC4F307221C
:1054E80008F10301C02000F0B3FFE2B208F10401A3
:1054F800C02000F0ADFFC9F3034305F4702243EA6E
:10550800123208F10501C02000F0A2FF08F10601DF
:10551800C9F30722C02000F09BFF08F107015FFADA
:1055280089F2C02000F094FFC020B121A02200F031
:105538008FFF07EE107A264CF8EEC77A0EBBD4ED33
:10554800015A06EE90AAB8EE657A05EE905AB8EEC2
:10555800666AF8EE656A0123C6EE266A237477EE5A
:10556800A67A67EE277A17EE900A09F031F941EC2E
:10557800100B0BF019F951EC100B09F03FFC6061AE
:1055880020E005EE90AAD4ED016AB8EE656A05EE52
:10559800905AB8EE667AF8EE656A0123C6EE266A76
:1055A800237677EEA67A67EE277A17EE900A09F047
:1055B8000FF941EC100B0BF0F7F851EC100B09F058
:1055C8001DFCE0610020BDE8FC8700BF000000432F
:1055D800701400200022012326E7012838B50D4663
:1055E80004D002280CBF3C242C2400E0342421469B
:1055F800C02001F029F805F0070200F00F0040EA8A
:1056080002122146C020BDE8384000F021BF2DE934
:10561800F3470A9C1D4607468A461646524B01E048
:105628006D0864089C42FBD82DB906F10076043E4B
:10563800F601A94634E006EE905AB8EE667A06EE10
:10564800904AF8EE667AF601C7EE277AA6F5007654
:105658009FED467A67EE877A17EE900A09F0B8F858
:1056680041EC100B0BF0A0F859EC108B4946404662
:1056780009F0C4FB3618E80109F088F8CDE9000103
:10568800204609F083F84B46424609F0F5F80246F1
:105698000B46DDE9000108F03BFF09F0AFFB81464E
:1056A800022F9BBF324BDB194FF0000893F8C880DC
:1056B800C4F307224146C02000F0CAFE08F10101E8
:1056C800E2B2C9B2C02000F0C3FE08F10201C9B2BB
:1056D800C6F30142C02000F0BBFE08F10301C9B2C5
:1056E800C6F30722C02000F0B3FE08F10401C9B2D6
:1056F800F2B2C02000F0ACFE04F47024C9F30343F6
:1057080008F1050143EA1432C9B2C02000F0A0FE36
:1057180008F10601C9B2C9F30722C02008F1070839
:1057280000F096FE5FFA89F25FFA88F1C02000F077
:105738008FFEBAF1010F0CBF2F220F220DB942F0D4
:105748004002012F06D002D3022F0AD105E0C02063
:10575800102104E0C020112101E0C020122100F036
:1057680077FE0020BDE8FC87FFFF0F000000004324
:10577800BB54040807B5012300930023FFF747FF34
:105788000EBD00280CBFFF22002208B5C02003214F
:1057980000F05EFE002008BD08B5C020B121AC2293
:1057A80000F056FE002008BD704708B500F050F91B
:1057B80000F050F9014B00221A7008BDE80B0020D8
:1057C800024B187880F00100704700BFE80B0020FA
:1057D800014B1878704700BFE80B002008B54FF45C
:1057E80000710F4807F0F9F80E4BD0F101005A7814
:1057F80038BF0020824201460ED05A681D2A0DDCAF
:1058080001321E2A5A6009D15870074800225A608E
:10581800BDE8084003F00CBC00225A6008BD00BF78
:1058280000080240E80B00200C9F0508014B58783F
:10583800704700BFE80B002010B500210446012284
:10584800302000F005FEC0B9012001F0A3F8002CBB
:10585800B8BF4034E4B210212246302000F0F8FDF1
:10586800012001F097F830201121224600F0F0FDC8
:105878000120BDE8104001F08DB810BD10B5002121
:1058880004460122302000F0E3FDC0B9012001F0F8
:1058980081F8002CB8BF4034E4B2122122463020EF
:1058A80000F0D6FD012001F075F8302013212246C2
:1058B80000F0CEFD0120BDE8104001F06BB810BD2E
:1058C800002810B5044603DB5F2CA8BF5F2400E066
:1058D800002430200021012200F0BAFDA8B90120DF
:1058E800E4B201F057F83B212246302000F0B0FD29
:1058F800012001F04FF830203C21224600F0A8FD9D
:105908000120BDE8104001F045B810BD302810B5A1
:1059180004460ADC10F17F0F02DB002802DB05E0F9
:105928006FF07E0404F5807400E0302400213020FC
:105938000A4600F08DFDA8B90120E4B201F02AF86A
:1059480041212246302000F083FD012001F022F899
:1059580030204221224600F07BFD0120BDE81040A6
:1059680001F018B810BD282810B5044609DC10F15C
:10597800180F02DB002802DB04E06FF017047F3405
:1059880000E02824002130200A4600F061FDA8B973
:105998000120E4B200F0FEFF53212246302000F03F
:1059A80057FD012000F0F6FF30205421224600F078
:1059B8004FFD0120BDE8104000F0ECBF10BD08B558
:1059C80030200021012200F043FD60B9012000F0E1
:1059D800E1FF30203321402200F03AFD0120BDE8EC
:1059E800084000F0D7BF08BD10B5302000210122C3
:1059F80000F02EFD044660B9012000F0CBFF3020F6
:105A08003321224600F024FD0120BDE8104000F0BB
:105A1800C1BF10BD10B530200021012200F018FDD3
:105A28000446A0B9012000F0B5FF342122463020F9
:105A380000F00EFD012000F0ADFF30203721224696
:105A480000F006FD0120BDE8104000F0A3BF10BD26
:105A58004020F1E6402011E708B50021012230205E
:105A680000F0F6FC012000F095FF302034210246BA
:105A780000F0EEFC012000F08DFF302037210246B7
:105A880000F0E6FC0120BDE8084000F083BF08B53F
:105A980000210122302000F0DBFC012000F07AFF19
:105AA800302034210C2200F0D3FC0120BDE808404E
:105AB80000F070BF00000000704770477047194B36
:105AC8001949D3ED006A93ED017A00231A469FED38
:105AD800176A03E0F0EE476AB0EE677A505E05EEAB
:105AE800900AF8EEE57A0133C7EE867A9BB218B2CF
:105AF80004327F2877EEE67AECDD27EE077A07EEA8
:105B0800A77A0B49074A0B80BDEEC77A00231360BA
:105B18005360C2ED027A17EE102A064B92001A6003
:105B2800704700BFF00B0020282600200000FA452F
:105B3800583A0020FC1600202DE9F84F2E4B2F4A2A
:105B480019682F4B19B92F4911602F4A02E02F49C4
:105B580011602F4A1A602F4BDFF8BCA0DFF8BC9009
:105B6800DFF8BCB000221A80244A9846176830E053
:105B780007EB84036500B3F9023007EE103AF8EE3C
:105B8800C77A013617EE900A08F022FE18A3D3E967
:105B9800002308F071FE09F009F929F815002AF820
:105BA800140037F9243007EE103AF8EEC77A0135B9
:105BB80017EE900A08F00CFE0DA3D3E9002308F0B5
:105BC8005BFE09F0F3F82BF8140029F81500A8F883
:105BD8000060B8F8006034B2FF2CC9DD00F05EF850
:105BE80000F06AF801F0C0F8BDE8F84F67E700BFB9
:105BF8009A9999999999E93FF0160020E41600209E
:105C0800201500202A2E00202A2A00202A360020CB
:105C18002A320020583A0020282200202826002076
:105C28002824002010B50B4C204606F0C4FA0A4B75
:105C380018600A4806F0BFFA094B1860FFF77CFFA6
:105C4800084B0949012220469A81BDE8104006F018
:105C580033BB00BF10600240F0160020886002408D
:105C680004170020F00B002020800010014B18685A
:105C7800704700BFFC16002008B5054B0548198879
:105C88000022012309F080FD034B187008BD00BFF6
:105C980070000020102200202C1D00200348044919
:105CA800044A4FF4807309F0E7BD00BF7400002078
:105CB800282200200E20002003480449044A4FF4FB
:105CC800807309F0D9BD00BF80000020282400207F
:105CD8004818002038B505460C460135C1F30721A0
:105CE80000F066FEA8B2E1B200F062FE00B238BD74
:105CF80038B5044600F070FD01340546A0B200F046
:105D08006BFDEDB2C0B240EA052000B238BD37B530
:105D18000B0E8DF804300B0C8DF805300B0A8DF83E
:105D280006308DF80710002400E0284601AB451C1A
:105D3800E15C013400F03CFE042CADB2F5D13EBD6F
:105D480037B5002400E02846451C00F045FD01ABAE
:105D5800ADB2E0540134042CF5D19DF805009DF84E
:105D68000430000440EA03609DF8073018439DF8AA
:105D7800063040EA03203EBD38B50446642000F0F2
:105D880009FE25786068AD00EDB2257006F02BFE9F
:105D9800237A40FA03F000F003000543104B257006
:105DA80005F00F055A5D6378D218D2B2D3B201322A
:105DB800D2B2022A637001D80022A2705BB2012B12
:105DC80003DD0123A3700023637094F901300133CC
:105DD80003DAFF23A3700023637094F9020038BD2F
:105DE8008C550408F7B504200121234F07F03EF92C
:105DF80002AD01214FF48040012407F067F9002625
:105E08004FF4B0733846694645F8083D8DF804608C
:105E18008DF8074006F082FD1020214607F026F98C
:105E280078236946154800938DF804608DF807407B
:105E380006F074FD0420214607F018F921464FF4B6
:105E4800804007F043F91E233846694600938DF8D1
:105E580004608DF8074006F061FD0220214607F036
:105E680005F9B02306488DF8046069468DF80740A7
:105E7800009306F053FDFEBD0008024000100240EA
:105E880000040240802108B5034806F0A6FDD0F1C1
:105E9800010038BF002008BD0004024008B54FF4D7
:105EA8008071044806F099FDD0F1010038BF002048
:105EB80008BD00BF0008024008B5FFF7E3FF08B1BE
:105EC800FFF7ECFFC0B208BD10B5642000F062FD1A
:105ED8000F48FFF751FF044610B90E4B187009E040
:105EE800FFF7DCFF30B9002C0A4B01DD012200E08E
:105EF800FF221A700848FFF73FFF0028074B01D11F
:105F0800187010BD01DD012200E0FF221A7010BDDB
:105F1800C000002088400020CC000020282A002053
:105F280007B50220012107F0A1F8012300938DF89D
:105F3800043002238DF805300448002369468DF8A3
:105F480006308DF8073006F0E9FC0EBD000402406B
:105F580010B5084C01210022204606F054FD40F2FD
:105F6800FF4000F017FD012120460A46BDE8104019
:105F780006F049BD0004024008B5FFF7E9FF00211B
:105F88000A46302000F064FA012000F003FD0121E8
:105F98000A46302000F05CFA012000F0FBFC0021EA
:105FA8000122302000F054FA012000F0F3FC012116
:105FB8000822302000F04CFA012000F0EBFC02210E
:105FC8000122302000F044FA012000F0E3FC002117
:105FD8000A46302000F03CFA012000F0DBFC1B21CF
:105FE800CD22302000F034FA012000F0D3FC042147
:105FF8000322302000F02CFA012000F0CBFC06210F
:106008000822302000F024FA012000F0C3FC072108
:106018000A46302000F01CFA012000F0BBFC0821E1
:106028008022302000F014FA012000F0B3FC1E2179
:10603800B022302000F00CFA012000F0ABFC052162
:106048009122302000F004FA012000F0A3FC0D2179
:106058000322302000F0FCF9012000F09BFC0E2107
:106068000022302000F0F4F9012000F093FC142104
:106078008022302000F0ECF9012000F08BFC0B218D
:106088008822302000F0E4F9012000F083FC302061
:106098000C21822200F0DCF9012000F07BFC1221A7
:1060A8008822302000F0D4F9012000F073FC13217D
:1060B8008C22302000F0CCF9012000F06BFC00218C
:1060C8000122302000F0C4F9012000F063FC0C210B
:1060D8000822302000F0BCF9012000F05BFC0D2103
:1060E8000822302000F0B4F9012000F053FC0E2102
:1060F8000822302000F0ACF9012000F04BFC0F2101
:106108000822302000F0A4F9012000F043FC00210F
:106118000A46302000F09CF9012000F03BFC4021A9
:106128000222302000F094F9012000F033FC002214
:106138004121302000F08CF9012000F02BFC3020A8
:106148003F21D42200F084F9012000F023FC002133
:106158000122302000F07CF9012000F01BFC102106
:106168000F22302000F074F9012000F013FC1121F7
:106178000F22302000F06CF9012000F00BFC1221F6
:106188000022302000F064F9012000F003FC132104
:106198000022302000F05CF9012000F0FBFB09210F
:1061A8003C22302000F054F9012000F0F3FB0021DC
:1061B8000122302000F04CF9012000F0EBFB3020E8
:1061C8003421024600F044F9012000F0E3FB3020BE
:1061D8003721024600F03CF9012000F0DBFB3621B4
:1061E8000322302000F034F9012000F0D3FB3921DC
:1061F8000322302000F02CF9012000F0CBFB3B21DA
:106208003C22302000F024F9012000F0C3FB3C219F
:106218000A46302000F01CF9012000F0BBFB0021E9
:106228000A46302000F014F9012000F0B3FB512198
:10623800C022302000F00CF9012000F0ABFB302028
:106248005221002200F004F90120BDE8084000F0C6
:10625800A1BB00BF2DE9F04F454E464D93B001213B
:106268004FF4001006F002FF304605F0A5FE4FF08F
:10627800C0630293404B0393404B002404934FF4B4
:1062880000794FF400334FF480684FF400674FF4FF
:10629800005A4FF4807B304602A90C93019309976A
:1062A800CDF8189005940794CDF82080CDF828A053
:1062B800CDF82CB00D9405F00BFF2246304630493E
:1062C80005F061FF3046012105F067FF01210A460C
:1062D8004FF0402007F038F9284605F06DFE294AAE
:1062E800019B0392284A0C9304922846402202A953
:1062F800059209970294CDF818900794CDF820805C
:10630800CDF828A0CDF82CB00D9405F0E1FE22467A
:1063180028461E4905F037FF2846012105F03DFFB4
:1063280042F2107701220221194807F00DF9384688
:1063380000F030FB3046012105F005FF0121284619
:1063480005F001FF384600F025FB0B238DF844309B
:1063580011A801238DF845408DF846408DF8473047
:1063680002F0EAFE384600F015FB13B0BDE8F08FE6
:1063780010600240886002400C4000402A3600202D
:106388002A2E00200C3C00402A3200202A2A002015
:10639800003C004002481021012205F04BBF00BF1D
:1063A8001060024013B50220012106F05FFE4FF491
:1063B80010730E4C009302238DF804308DF80530CD
:1063C80001238DF806302046002369468DF80730F2
:1063D80006F0A4FA20460621042206F01FFB2046F8
:1063E8000921042206F01AFB1CBD00BF000402406C
:1063F80030B5154D85B001214FF4001006F05AFE56
:10640800284606F021FB0023ADF804304BF6FF7355
:10641800ADF806303323ADF808304FF48063ADF89B
:106428000A304FF48043ADF80C3004AC074B2846D3
:10643800012144F8103D06F0A9FB2846694606F0FC
:1064480031FB05B030BD00BF00540040801A060083
:1064580073B54FF4961306460D461446019304E0AF
:10646800019B5A1E0192002B57D031484FF400313E
:1064780006F0A4FC0028F3D12D48012106F092FB78
:106488004FF48053019304E0019B5A1E0192002BA4
:1064980045D02748274906F07CFC0028F4D024483A
:1064A8003146002206F096FB4FF48053019304E036
:1064B800019B5A1E0192002B33D01D481E4906F03D
:1064C80068FC0028F4D01A48294606F006FC4FF468
:1064D8008053019303E0019B5A1E01921BB3144899
:1064E800164906F056FC0028F5D01148214606F05A
:1064F800F4FB4FF49613019303E0019B5A1E01929B
:106508009BB10B480E4906F059FC0028F5D0084805
:10651800012106F053FB002008E0012006E00220DC
:1065280004E0032002E0042000E005207CBD00BF59
:1065380000540040010003008200070080000700AB
:1065480004000010F7B51F464FF4961306460D4693
:106558001446019304E0019B5A1E0192002B5ED061
:1065680034484FF4003106F029FC0028F3D13148B3
:10657800012106F017FB4FF48053019304E0019BBF
:106588005A1E0192002B4CD02A482B4906F001FCD8
:106598000028F4D027483146002206F01BFB4FF4B0
:1065A8008053019304E0019B5A1E0192002B3AD0BC
:1065B8002048224906F0EDFB0028F4D01D48294662
:1065C80006F08BFB4FF48053019304E0019B5A1EA5
:1065D8000192002B29D01748194906F0DAFB002848
:1065E800F4D000254FF4961610E0615D114806F0CE
:1065F80074FB019603E0019B5A1E0192BBB10D4842
:10660800104906F0DBFB0028F5D00135EBB2BB42A0
:10661800EBD30848012106F0D1FA002008E0012058
:1066280006E0022004E0032002E0042000E0052048
:10663800FEBD00BF005400400100030082000700B7
:10664800800007000400001037B54FF49613044685
:106658000D46019305E0019B5A1E0192002B00F0A4
:106668009B8056484FF4003106F0A8FB0028F2D171
:106678005248012106F096FA4FF48053019305E041
:10668800019B5A1E0192002B00F088804B484C4910
:1066980006F07FFB0028F3D048482146002206F088
:1066A80099FA4FF48053019304E0019B5A1E01921A
:1066B800002B75D04148434906F06BFB0028F4D005
:1066C8003E48294606F009FB4FF48053019304E045
:1066D800019B5A1E0192002B64D038483A4906F0B3
:1066E8006DFB0028F4D03548012106F05BFA4FF421
:1066F8008053019304E0019B5A1E0192002B53D052
:106708002E482F4906F045FB0028F4D02B48214697
:10671800012206F05FFA4FF48053019304E0019BD5
:106728005A1E0192002B41D0244C2849204606F0DD
:1067380045FB0028F3D02046002106F053FA2046F6
:106748000121238B06F03AFA4FF48053019304E0B9
:10675800019B5A1E0192002B2AD018481C4906F0AA
:106768002DFB0028F4D0154806F0B9FA4FF48053F1
:106778000193124A03E0019B591E0191D3B113887A
:106788009B05F8D4012104460C4806F02BFA0B4867
:10679800104906F02DFB0EE001240CE002240AE06B
:1067A800032408E0042406E0052404E0062402E0AB
:1067B800072400E0082420463EBD00BF00540040E6
:1067C800010003008200070004000010020000100E
:1067D800400000100004001013B54FF4961304464F
:1067E800019305E0019B5A1E0192002B00F0B08036
:1067F80061484FF4003106F0E1FA0028F2D15E4812
:10680800012106F0CFF94FF48053019305E0019B75
:106818005A1E0192002B00F09D805748574906F0F8
:10682800B8FA0028F3D05448A021002206F0D2F983
:106838004FF48053019305E0019B5A1E0192002BEF
:1068480000F08A804C484E4906F0A3FA0028F3D09D
:10685800C4F30521484806F040FA4FF480530193E9
:1068680004E0019B5A1E0192002B77D0424845490B
:1068780006F0A4FA0028F4D0E1B23F4806F02DFA59
:106888004FF48053019304E0019B5A1E0192002BA0
:1068980066D039483B4906F091FA0028F4D03648CA
:1068A800012106F07FF94FF48053019304E0019B26
:1068B8005A1E0192002B55D02F48304906F069FA2C
:1068C8000028F4D02C48A121012206F083F94FF4C6
:1068D8008053019304E0019B5A1E0192002B43D080
:1068E800254C2949204606F069FA0028F3D02046AD
:1068F800002106F077F920460121238B06F05EF986
:106908004FF48053019304E0019B5A1E0192002B1F
:106918002CD019481D4906F051FA0028F4D0164821
:1069280006F0DDF94FF480530193134A03E0019B0D
:10693800591E0191E3B113889905F8D40121044641
:106948000D4806F04FF90C48114906F051FA10E0CD
:1069580001240EE002240CE003240AE0042408E0E9
:10696800052406E0062404E0072402E0082400E0E9
:10697800092420461CBD00BF00540040010003004C
:106988008200070004000010020000104000001000
:106998000004001082B0002304E0019B013301933E
:1069A800009B01330093009B8342F6D302B07047EB
:1069B80037B54FF4805304460D46019304E0019B1C
:1069C8005A1E0192002B6ED03D484FF4003106F05C
:1069D800F5F90028F3D13A48012106F0E3F84FF41D
:1069E8008053019304E0019B5A1E0192002B5CD056
:1069F8003348344906F0CDF90028F4D03048A021B6
:106A0800002206F0E7F84FF48053019304E0019B5D
:106A18005A1E0192002B4AD029482B4906F0B9F991
:106A28000028F4D0C4F30521254806F056F94FF4A0
:106A38008053019304E0019B5A1E0192002B38D029
:106A48001F48224906F0A5F90028F4D0E1B21C48F5
:106A580006F043F94FF48053019303E0019B5A1E5B
:106A6800019243B31648194906F093F90028F5D066
:106A78001348294606F031F94FF49613019303E0C1
:106A8800019B5A1E0192C3B10D48114906F096F9AF
:106A98000028F5D00A48012106F090F80D48FFF7C4
:106AA80079FF00200AE0012008E0022006E0032028
:106AB80004E0042002E0052000E006203EBD00BFFF
:106AC8000054004001000300820007008000070016
:106AD80004000010A086010013B50520012106F06E
:106AE800C5FA184C4FF4E053009302238DF8043094
:106AF8008DF805302046002369468DF806308DF85C
:106B0800073005F00BFF20460A21062205F086FF14
:106B180020460C21062205F081FF062220460B2183
:106B2800A4F5006405F07AFF4FF400432046694657
:106B3800009305F0F3FE20460F21062205F06EFFB4
:106B48001CBD00BF000802401FB50446FFF7E8F966
:106B5800FFF74EFCFFF710FAFFF7BEFF01214FF4D5
:106B6800004006F0A7FA02940F4C1023ADF802304B
:106B7800204600236946ADF80430ADF80C30ADF876
:106B88000030ADF8063006F0C4FB69464FF04020EF
:106B980006F093FC2046012106F043FC4FF040200C
:106BA800012106F03EFC1FBD003C0040014B18606F
:106BB800704700BF0C0C0020704710B50A4A1379C3
:106BC800262B04D80949C8540133137110BD074A4C
:106BD8000123591ED45C0133272B5454F9D1034B9C
:106BE80083F8260010BD00BF0C0C00202C3A0020B2
:106BF800704710B504462078FFF7DFFF14F8013F0F
:106C0800002BF8D110BD38B504460D46013D14F8E7
:106C1800010BEDB2FFF7D1FF002DF7D138BD00BF52
:106C2800014B1878704700BF140C0020014B5878AE
:106C3800704700BF140C0020024B187880F0010048
:106C4800704700BF140C0020024B00221A705A70C3
:106C5800704700BF140C0020014B01221A707047C6
:106C6800140C0020014B01225A707047140C0020AC
:106C780082B0002304E0019B01330193009B0133A0
:106C88000093009B8342F6D302B070470148024943
:106C980004F06CBA903A00209040002007B5042018
:106CA800012106F0E3F901214FF4804006F00EFAC5
:106CB8004FF40073009300238DF804300348012338
:106CC80069468DF8073005F029FE0EBD0008024020
:106CD800034A044B1A60044A044B1A60704700BF09
:106CE8000000FA45B04A0020DB0FC93F884A00205F
:106CF800034B00221A60034A034B1A60E8E700BFFF
:106D08003C4100200000FA450016002007EE100A5A
:106D1800024BF8EEC77AC3ED007A704700160020E0
:106D280038B510EE100A07F053FD0DA3D3E9002380
:106D380007F0A2FD084B044618680D4607F048FD09
:106D48000B4602462946204607F0C0FE08F076F8B2
:106D5800024B186038BD00BFB04A0020884A0020A6
:106D6800182D4454FB2119402DE9F04F2DED068BC9
:106D7800734CDFF800A289B00027A34637F80A5001
:106D8800704B2580FE5A704B6680186807F020FD0E
:106D980069A3D3E9002307F06FFD08F007F86368DB
:106DA8006A4AC018011101F580610905090D606082
:106DB800C0F30B100DF1200C32F8203032F82120EE
:106DC800616A238115FB02F0628115FB03F516FB4E
:106DD80002F216FB03F60CEB4103E0602561C0F3F9
:106DE800CF30C5F3CF356261A661C2F3CF32C6F3A7
:106DF800CF3623F8200C23F8105C23F8182C23F83E
:106E0800086C534BA08301310B40002BE58322848F
:106E1800668403DA013B63F003030133CBF82430C3
:106E2800002B7CD14B484C4A6946042308F0E4FF08
:106E38004A484B4A04A9042308F0DEFF49484A4A55
:106E480002A9042308F0D8FF484A494806A90423A0
:106E580008F0D2FFB4F9283007EE903AB4F92A3096
:106E6800B8EEE79A07EE903AB4F92C30B8EEE78A14
:106E780007EE903AB4F92E30F8EEE79A07EE903A1A
:106E8800F8EEE78A68EE087A49EE097A17EE900A72
:106E980007F09EFC41EC100B09F012FE51EC100BB0
:106EA80007F0CCFF68EEA87A49EEA97A0AEE100A34
:106EB800206317EE900A07F08BFC41EC100B09F0E9
:106EC800FFFD51EC100B07F0B9FF68EE897A58EE18
:106ED800297A28EE288A0AEE900A606309EE298A40
:106EE80017EE900A07F074FC804618EE100A8946DF
:106EF80007F06EFC49EC108B41EC110B09F058FDC2
:106F080051EC100B07F09AFF8AEE2A0AA06384ED71
:106F18000F0A01F0D5FB94ED0E0A01F0E1FB0237F0
:106F2800B7F5007F7FF42AAF09B0BDEC068BBDE84A
:106F3800F08F00BFAFF3008039D6C56D305FC44015
:106F4800180C002048180020884A0020A85504087A
:106F580003000080B4000020400C0020A80000209E
:106F6800420C00209C000020440C0020460C00200D
:106F7800900000200E200020014B93ED0F0A70476F
:106F8800180C0020014B93ED0E0A7047180C0020D6
:106F9800014B93ED0C0A7047180C0020014B93ED40
:106FA8000D0A7047180C002010B5FEF7D3F9002021
:106FB800012324210246FEF737FA114B1C780020E2
:106FC800012C05D10146FEF708FB2046002104E00C
:106FD8000721FEF702FB01200721FEF7FEFA6322D4
:106FE8001221C020FFF734FA02200121FEF7F5FA3A
:106FF800FEF7D2FB0120BDE81040FEF7C2BB00BF80
:10700800000D00200D4B1B78012B05D10C4B0D4AB0
:10701800196812688A181A600B4B1B78012B084BE9
:10702800196805D1094A914207DD01321A60704793
:10703800074A914201DD01321A6070478C3A0020FC
:107048008C400020883A0020000D00207FD1F008F5
:107058003F420F000E4B1B78012B05D10D4B0E4AFA
:10706800196812688A1A1A600C4B1B78012B094B95
:1070780005D10B4A1968914208DC1A6070471A68F2
:10708800B2F5FA5FDCBF4FF4FA521A60704700BFDE
:107098008C3A00208C400020883A0020000D002007
:1070A80040420F00024B1A68024B1A60704700BF3B
:1070B800784000208C4000202DE9F04F8246584847
:1070C8008BB0B0FBF1F00C4607F060FB41EC100B05
:1070D80009F06AFB51EC100B07F090FEC307074656
:1070E80048BF471E04FB07F007F050FB46A3D3E94F
:1070F800002307F0EBFC04460D4645EC104B09F065
:1071080053FB59EC108B204642464B46294607F064
:10711800FFF9CDE904014946404607F06FFE3CA35C
:10712800D3E900230990DDE9040107F021FE0028D6
:107138003DD1002401234FF01509224698462046E8
:10714800DFF8E4B003E0234642462C46B04600FB95
:1071580004355D452ED800FB0826DDE904012EA381
:10716800D3E9002307F004FE30BBDDE90423002047
:107178002C4907F0ABFC41EC100B0390029109F08D
:1071880013FB0398029953EC102B8DED060B07F0B7
:10719800BFF909F1FF39CDE904015FFA89F9DDE9A1
:1071A800060107F02BFEB9F1000FCCD104E0012550
:1071B800002601E025464646099BD9B2BAF1000FE0
:1071C8000BD132462B465046FEF72EF90123009389
:1071D800504651463A46534609E032462B4601206E
:1071E800FEF722F90120009001463A460023FEF7F7
:1071F8000EFAFEF7D1FA01200BB0BDE8F04FFEF70A
:10720800C0BA00BFAFF300800000000084D7774108
:10721800956479E17FFDA53DBBBDD7D9DF7CDB3D1A
:1072280000E9A4350000F03FFFFF0F001F4B1B785B
:10723800022B10B539D01E4B1E4A19681E4B1F4C25
:107248001B68CB189342236018DC0020FFF734FF3B
:1072580001202168FFF730FF194B1C780020012C12
:1072680005D10146FEF7B9F92046002104E00721BF
:10727800FEF7B3F901200721FEF7AFF9114B1B7890
:10728800022B12D10A4C104B22681B689A420CDA66
:107298000E4B1B78012B08D10D4B186800F070F8C5
:1072A8000C4B22681B68D318236010BD604D00206A
:1072B8008C40002080D1F008284100202C4100207B
:1072C800000D00208C3A0020684000206440002017
:1072D80044400020883A002008B5FEF7D3FD094B4A
:1072E8005A78187002435A701AB19A7801329A7013
:1072F80030B99B78034A012B02D90023537093704D
:1073080008BD00BF580C002007B50420012105F076
:10731800ADFE4FF46043009301238DF8043002233F
:107328008DF805300448002369468DF806308DF83D
:10733800073005F0F3FA0EBD00080240084B1A6842
:107348004FF47A73B2FBF3F2064B013A5A60064ADD
:10735800F02182F8231000229A6007221A607047F1
:10736800A401002010E000E000ED00E0034B5A68A3
:1073780012B15A68013A5A60704700BF580C002091
:10738800024B58605A68002AFCD17047580C0020FC
:1073980030B585B004460D4601A85C490A220BF0B9
:1073A8001FFE5B4B1B78032B10D8DFE803F00205A8
:1073B800080B01A8574907E001A8574904E001A8AC
:1073C800564901E0564901A80BF0F4FE04AA131926
:1073D80013F80C3C5D19EDB22F2D01D80A3502E0E7
:1073E800392D01D90A3DEDB204AB1C194FF6FF70D7
:1073F80004F80C5CFCF71AFF0020FDF70DF80DF1FE
:1074080003050F24204623345A21002315F8012FA1
:10741800A4B2FDF71BF8B4F5A57FF3D164205A2177
:107428002C220023FDF712F80023CD205A212C220C
:10743800FDF70CF80020FCF7F9FE354B1B78032B01
:1074480062D8DFE803F002284B5601A931480BF057
:10745800B1FE0A2200212F480CF050F8314A324B75
:1074680012781860012A06D1304A904201DC0132B4
:107478001A602F4A06E0B0F5FA5FBCBF4FF4FA5223
:107488001A602C4A1B689342C4BF274B1A602A4BC8
:107498001A682A4B20E001A91F480BF08BFE0A222C
:1074A80000211D480CF02AF81E4A254B1278186056
:1074B800012A06D11D4A904201DC01321A601C4A99
:1074C80006E0B0F5FA5FBCBF4FF4FA521A60194AE9
:1074D8001B68934218DD1A4B1A6015E001A90F4882
:1074E8000BF068FE0D4800210A220CF007F8154B36
:1074F80009E001A90A480BF05DFE094800210A22AB
:107508000BF0FCFF104B186005B030BDC19F05089B
:1075180076400020524000206C400020144100209A
:1075280048400020000D0020804000203F420F000E
:1075380080D1F00840420F00784000208C400020A5
:1075480030410020844000204440002010B50D4BFD
:107558000D4C1A680D4821460BF004FE0C4B0D48E3
:107568001A6821460BF0FEFD0B4B0C481A682146A1
:107578000BF0F8FD0A4B0B481A682146BDE810408D
:107588000BF0F0BD80400020CB9F05085240002042
:10759800304100206C40002084400020144100202D
:1075A800444000204840002008B500210A220D4828
:1075B8000BF0A4FF0C4B002118600A220B480BF0BB
:1075C8009DFF0B4B002118600A220A480BF096FF1A
:1075D800094B002118600A2208480BF08FFF084B5E
:1075E800186008BD52400020804000206C400020F8
:1075F80030410020144100208440002048400020F1
:1076080044400020014B93ED020A7047580C0020BB
:10761800014B93ED030A7047580C0020034B83ED90
:10762800000AC3ED010A83ED021A7047D45E0020F8
:10763800014B1860704700BF8C400020014B186850
:10764800704700BF80400020014B1868704700BF9A
:107658003041002008B54FF49570FEF749FB40F221
:107668006523C31A584240EB030008BD08B5C6207D
:10767800FEF73EFB40F28D13C21A504240EB020067
:1076880008BD4FF4957040F26521FEF723BBC62074
:1076980040F28D11FEF71EBB08B5F9F74DF9BCEEA7
:1076A800C00A4FF4967010EE101AFEF730FBF9F787
:1076B80049F901464FF49870FEF729FBF9F748F9A4
:1076C800BCEEC00A4FF49A7010EE101ABDE80840DC
:1076D800FEF71DBB38B5FFF7BDFFC0B14FF496707C
:1076E800FEF72EFB124D134C28604FF49870FEF7EE
:1076F80027FB20604FF49A70FEF722FB0E4B2A6896
:1077080018600E4B1A61226898615A6106E00B4BAB
:107718000B4A1A610B4A5A610B4A9A61074A0B4B8A
:1077280050699169126958601A60996038BD00BF44
:107738000C0D0020080D0020040D0020580C00201E
:10774800E17A843F14AE3740CCBC8C2CD45E002048
:1077580060EEA00AB7EE007AF0EE606A70EE077A83
:1077680040EE006A47EEA70A36EEC77A08B5C7EEBC
:10777800200A10EE900A07F02BF80022084B07F0B9
:107788007BF80022074B06F0C5FE07F057FB07EE13
:10779800900AFDEEE77A17EE900A9F3008BD00BF09
:1077A800000059400000E03F38B52DED028BF7EEA0
:1077B800008AB0EE608A70EE288A10EE900A28EEF1
:1077C800088A07F005F808EEA88A00220F4B07F090
:1077D80053F8044618EE100A0D4606F0F9FF024663
:1077E8000B462046294607F071F90022084B06F09F
:1077F80091FE07F023FB07EE900AFDEEE77A17EEFD
:10780800900A7730BDEC028B38BD00BF000069409C
:107818000000E03FF0B56A4D2DED068B95E80F00AE
:107828008DB008AE103586E80F000FCD01AC0FC43F
:1078380095E807004FF6FF7384E807009F2077213B
:107848006422FAF782FBA020772164224FF6FF73A7
:10785800FAF77BFB9E20772164224FF6FF73FAF735
:1078680074FB9F20762164224FF6FF73FAF76DFBB5
:107878004FF6FF73782164229F20FAF766FB0020F9
:10788800FCF730FB9F2077216522FCF705FD9F2040
:1078980077216422FCF700FD07AD0C36F7EE009A5D
:1078A8000435F7EE008A95ED009A4FF49674B0EE21
:1078B80068AA18EE900A06F08BFF3FA3D3E90023CD
:1078C80006F0DAFF07F0BAFA08EE900A38EEE98A0D
:1078D800B0EE490AF0EE480AFFF73AFFB0EE490A5F
:1078E800F0EE480A0746FFF75FFFBFB281B20F22EA
:1078F8003846FCF704FA013CDBD14FF49674F7EEF6
:10790800008A18EE900A06F063FF2BA3D3E9002340
:1079180006F0B2FF07F092FA08EE900A39EEE88A0C
:10792800B0EE490AF0EE480AFFF712FFB0EE490A36
:10793800F0EE480A0746FFF737FFBFB281B20F22C1
:107948003846FCF7DCF9013CDBD1B542A8D16C46DE
:1079580007AE043494ED009A4FF4C875F7EE008A28
:1079680018EE900A06F034FF13A3D3E9002306F0BB
:1079780083FF07F063FA08EE900A38EECA8AF0EE41
:10798800490AB0EE480AFFF7E3FEB0EE480AF0EE07
:10799800490A0746FFF708FFBFB281B200223846FE
:1079A800FCF7ADF9013DDBD1B442D2D10DB0BDEC4D
:1079B800068BF0BDAFF30080295C8FC2F528F03F3D
:1079C800A8950408121A06EE902A081AB8EEE67A64
:1079D80006EE900AF8EEE67AC7EE277A9FED047A6B
:1079E80067EE877AFDEEE77A17EE900A704700BFD8
:1079F8000000A0438A1A06EE902A081AB8EEE67A22
:107A080006EE900AF8EEE67AC7EE277A9FED047A3A
:107A180067EE877AFDEEE77A17EE900A704700BFA7
:107A28000000484370B506460D460024610704D59A
:107A3800A0B231462A46FCF762F90134B4F5A07FBA
:107A4800F4D170BD70B506460D460024600704D514
:107A5800A1B230462A46FCF752F90134C82CF5D1B8
:107A680070BD114B11481B781149124A0068012B4F
:107A7800114B09D1126808601A60104B1A68104B34
:107A88001A60104B1A680CE01268D2011A600B4B8E
:107A98001A680B4BD2011A600A4B1A68C0010860B9
:107AA800D201094B1A607047000D00208040002069
:107AB80078400020304100206840002084400020A9
:107AC800883A00205C40002028410020024B1A68B8
:107AD800024B1A60704700BF784000208C4000209D
:107AE80008B5FFF7BEFFBDE80840EFE70022F0B594
:107AF8001346202603254FF02C0C00E02646303E86
:107B0800F6B217460132092E10F8014B0AD897FB36
:107B1800F5F605FB16772FB9CE1801F803C0747077
:107B2800023301E0CC540133092AE7D12022CA5498
:107B3800CB1848225A707A229A700022DA70F0BD67
:107B480070B58CB005460C4608A80E491E460BF0C9
:107B580009FB08A86946FFF7C9FF6A460A4904A84D
:107B68000BF000FBBDF84000FCF760FB3046FCF76B
:107B780073FB2846214604AA0023FCF785FC0CB0B9
:107B880070BD00BFD19F0508929D05082DE9F047FB
:107B9800084B2DED0A8B1B78022BC4B000F0EC8447
:107BA800054B1A78054B5AB91A68802392FBF3FAE9
:107BB80008E000BF604D0020000D00208C40002030
:107BC800D3F800A0FFF7D8F9D34C84ED070AFFF7E4
:107BD800D9F994ED097AD4ED077A37EE077AF0EE01
:107BE800086A37EE277ACD4BCD4A9D6887EE267A0C
:107BF800D3ED018A84ED027A84ED097A93ED007A57
:107C080067EE277A82ED007AC4ED077A17EE900ABC
:107C1800C2ED018A84ED080A10EE108A06F0D8FD3C
:107C2800064640460F4606F0D3FD41EC100B41ECEA
:107C3800190B08F061FD59EC108BB0EE490AF0EE13
:107C4800690A08F059FE304653EC102B394606F005
:107C580013FE07F0F3F842464B4608EE100A394681
:107C6800304606F009FE07F0E9F8DFEDAE7A9FED41
:107C7800AE7A78EEA78A09EE900AC8EE878A68EE8F
:107C8800087A79EEE89AB1EE488A49EEA97A9FED2A
:107C9800A7BA67EE877ADFEDA6BA88EE278AC9EE1B
:107CA800A79A84ED038A18EE100A06F091FDCDE933
:107CB8000601504606F07AFD91A3D3E9002306F0A9
:107CC800DBFD064628460F4606F082FD02460B46B7
:107CD8003046394606F0D0FD02460B46DDE906017E
:107CE80006F016FC07F0AAF80AEE100A29EEA98A8F
:107CF8006AEE0ACAB1EE4A9A78EE2C7A8D4B89EE72
:107D0800279AC9EEA7AAB4EE4B9AF1EE10FAC8BFAB
:107D1800B0EE4B9AB4EE6B9AF1EE10FA48BFB0EEA3
:107D28006B9AC3ED00AA83ED019A1AEE900A06F049
:107D38004FFD0022804BCDE9020106F0E9FB69EE18
:107D4800097A044617EE900A0D4606F041FD2246D0
:107D580006460F462B462046294606F08DFD32463C
:107D68003B4606F0D7FB41EC100B08F0A9FE0022B9
:107D7800DDE90201704B59EC108B06F0CBFB024693
:107D88000B4606F079FD32463B4606F0C3FB41EC54
:107D9800100B08F095FE4046494655EC104B07F08D
:107DA8004DF8294608EE900A204607F047F807EEF6
:107DB800900AC8EEA78A614D614CB7EE00CA18EE6A
:107DC800900A06F005FD50A3D3E9002306F0C6FF8C
:107DD800DFED5C7A002818BFF0EE678AF4EE4C8A73
:107DE800DFED597AF1EE10FAC8BFF0EE678ADFEDE1
:107DF800577A6AEE277AC5ED008A17EE900A06F0E0
:107E0800E7FCDFED537A37EEC88A064678EE6CCA8F
:107E18000F46C4E902671CEE900A06F0D9FC47EC4D
:107E2800106B41EC110BC4E9000108F0C1FD38EEFC
:107E38008C8A3CEE68CA51EC100B88EE0C8A06F06E
:107E4800FDFF444B1B7880F00048B4EE4B8AF1EEFE
:107E580010FAC8BFB0EE4B8AB4EE6B8AF1EE10FA96
:107E680048BFB0EE6B8A022BC5F8048032D13A4F76
:107E78003E68002E2EDB394B394DC3F800A0B40004
:107E8800621C5B6825F814A018EE900A25F81230D9
:107E980006F09EFC0022334B06F0EEFC06F0AEFF27
:107EA80004F10209013625F81900404606F090FC55
:107EB80017A3D3E9002306F0DFFC06F077FF0334AD
:107EC800B6F5FA7FC8BF4FF0FF3325F814003E60BF
:107ED800C8BF3B60FFF75CF80F4C84ED0A0AFFF758
:107EE8005DF884ED0B0AFDF7C1FE524620631E497A
:107EF80034A80BF037F9A06A06F06AFC36E000BF38
:107F08001F85EB51B81E19402D431CEBE2361A3F72
:107F1800CDCCCCCC0C5FC440580C0020D45E0020E3
:107F28009C01002000008C420000F042003C1C46EE
:107F3800003C1CC6584D002000004940444C00201D
:107F4800104F002017B7D13872F97F3F0AD7233D69
:107F580017B7D1398C3A00207C4000204C4D0020C6
:107F6800244F00200000F040D69F050802460B462B
:107F780024A873490BF0F6F8E06A06F029FC0246DB
:107F88000B4628A86F490BF0EDF819EE900A06F099
:107F98001FFCCDE90401DDE904236B492CA80BF093
:107FA800E1F86A49DDE9062330A80BF0DBF8DDE9E2
:107FB8000223674910A80BF0D5F819EE100A06F04D
:107FC80007FCCDE90A01DDE90A23624914A80BF090
:107FD800C9F818EE900A06F0FBFBCDE90801DDE9C7
:107FE80008235D4918A80BF0BDF8404606F0F0FBE1
:107FF80006460F4632463B4658491CA80BF0B2F8D5
:1080080018EE100A06F0E4FB804689464B465449B0
:10801800424620A80BF0A6F80CA85249226B0BF098
:10802800A1F8514B1B78013BDBB2012B00F2968281
:108038004E4B1B78072B00F29182DFE813F0080003
:108048008F02A3002A016D01C7015F0225020220E9
:10805800FCF7E2F94FF6FF70FCF7FEF81F20FCF77B
:10806800E5F819210023424A2D20FCF70DFA4FF6B6
:10807800FF70FCF7F1F800200024FCF7D7F80F2078
:10808800B42152464FF6FF730094FFF759FD0F20B5
:10809800772124AA2346FCF7F7F9A0200DEB00026C
:1080A80077212346FCF7F0F90F20412118AA23462F
:1080B800FCF7EAF9A02041211CAA2346FCF7E4F9C1
:1080C8000F2065212CAA2346FCF7DEF930AA2346A7
:1080D800A0206521FCF7D8F90F20532110AA2346C8
:1080E800FCF7D2F9A020532114AA2346FCF7CCF9B7
:1080F8000F209B2120AA2346FCF7C6F91D4B1B6BBA
:10810800B3F57A7FCCBF4FF4FC604FF47840FCF7AE
:10811800A3F80CAAA0209B210023FCF7B5F9164B65
:108128001B780221012B0CBF144A154A4FF48C709E
:108138000023FCF7A9F91F20FCF78EF80EE200BF18
:10814800E09F0508EB9F0508F69F050800A00508B5
:108158000AA0050815A0050820A005082BA00508F9
:1081680036A0050842A005088C3A002024410020CA
:108178004FA00508580C0020000D00206EA005082F
:1081880072A00508DDE904233EA8B1490AF0EAFF18
:10819800DDE9062341A8AF490AF0E4FFDDE902233F
:1081A80038A8AD490AF0DEFFDDE90A233BA8AB4950
:1081B8000AF0D8FFE62002213EAA0023FCF764F962
:1081C800E620162141AA0023FCF75EF90220C82107
:1081D80038AA0023FCF758F93BAA00230220DC2127
:1081E800FCF752F9DFED9E7A68EEA78A4FF6E07544
:1081F80018EE900A06F0ECFA47EC106BCDE9020194
:1082080008F07AFA59EC108B47EC106B08F074FB05
:10821800002057EC106BFCF71FF80A215246002388
:1082280005200095FFF78CFC4FF47840FBF7FEFF24
:10823800DDE9020142464B4606F01EFB76A3D3E970
:10824800002306F067F906F0B1FD324684B23B46DA
:10825800DDE9020106F010FB02460B4670A1D1E9E8
:10826800000106F055F906F0A1FD81B22046F9F7A4
:108278009CFE9D20772105220023FCF707F89F200C
:10828800752105220123FCF701F82846FBF7CEFFEC
:1082980064E1744B1868744B52461968FFF792FBF7
:1082A800B0F59F7F044602DD704B02221A709FEDE5
:1082B800708AF4EEC8AAF1EE10FA14D5F5EEC0AA49
:1082C800F1EE10FA0FDDFDEEEAAA4FF4FA711AEE9C
:1082D800902A0020FFF78EFBA3B281B24FF6FF72FF
:1082E8001846FBF70CFDB4EEC89AF1EE10FA40F10F
:1082F8003581DFED607AB4EEE79AF1EE10FA40F3DB
:108308002D81BDEEC99A5C4819EE102A4FF4FA7116
:10831800FFF770FBA4B2ECE0524B1868524B524680
:108328001968FFF74FFBB0F59F7F064602DD4F4BFC
:1083380002221A70F5EEC09AF1EE10FA1DDDDDE9A1
:10834800040139A3D3E9002306F008FDA8B138A336
:10835800D3E90023DDE9040106F08EFA02460B4654
:108368000020464906F0D4F806F020FDB4B281B2E8
:108378004FF6FF722046FBF7C2FC1AEE100A06F011
:1083880027FA2DA3D3E9002304460D4606F004FD81
:10839800002800F0E3802046294623A3D3E90023E0
:1083A80006F0DCFC002800F0D98025A3D3E90023DF
:1083B8002046294606F060FA0022314B06F0AAF85A
:1083C80006F0F4FCB6B281B2304694E0DDE908016B
:1083D8001DA3D3E9002306F0DFFC002800F0BE80CF
:1083E800204B1868204B52461968FFF7EBFAB0F596
:1083F8009F7F044602DD1D4B02221A709DED080B7B
:1084080008F0D8FA53EC102B1046194600221D4BE1
:10841800A4B206F031FA99E00000000000E06340E1
:108428000000000000C05D409A9999999999B93F58
:108438000000000000409F409A9999999999B9BF06
:108448000000000000408F4076711B0DE02DA03F1A
:1084580076A0050880A005088AA0050894A005084C
:108468000000C8428040002030410020604D0020BC
:108478000000FA430000FAC30CFEFFFF0000694049
:1084880000005940000054C047A3D3E900233046F8
:10849800394606F0F1F946A3D3E9002306F016FBA6
:1084A80006F0CCFC384B08EE100A1868374B5246D9
:1084B8001968FFF787FAB0F59F7F02DD344B022277
:1084C8001A70DFED347A48EEE77A84B2FDEEE77A87
:1084D800204617EE901A4FF6FF7289B2FBF70FFC91
:1084E800BDEEC88A6FF0B30018EE102AB421FFF76A
:1084F80081FA81B220464FF4FC622DE0DFED267A46
:10850800B4EEE78AF1EE10FA28D51F4B18681F4B16
:1085180052461968FFF756FAB0F59F7F044602DD08
:108528001B4B02221A7049EC108B08F043FA53ECEB
:10853800102B104619460022184B06F09DF90246EA
:108548000B4600201649A4B205F0E2FF06F02EFC07
:108558004FF6FF7281B22046FBF7D1FB114B1B7817
:10856800022B09D043B14FF6FF7300930520DC219D
:1085780052460023FFF7E4FA44B0BDEC0A8BBDE88D
:10858800F08700BFAFF3008080400020304100201A
:10859800604D0020000048430000C84200005940D8
:1085A800000069402441002000000000008076405F
:1085B8001F85EB51B81E1940F7B5044600283ED078
:1085C8001F4B204F188801210419FBF7F7FA0120E7
:1085D800FBF748F9A4B2A6B20025E85B0235FBF721
:1085E8008FF9B5F5C67FF8D14FF6FF752046C7223B
:1085F80001212B46FBF7F8FC114B1E80124B1C681F
:10860800124B36B21B6806EE906A1B1BB8EEE67A70
:1086180006EE903AF8EEE67A67EE277A17EE900AB9
:1086280006F0D6F800220A4B06F050FA06F0BEFB18
:10863800DC212218002305200095FFF781FAFEBDF2
:10864800384C0020624D002080400020304100203E
:108658000000744013B50F4CA38EADF80630BDF87A
:1086680006309BB253B1BDF806004FF6FF7380B2D7
:108678000121C722FBF7B8FC0023A386064B1B7811
:10868800022B06D1054C94F90000FFF795FF002353
:1086980023701CBD580C0020604D0020282A0020A3
:1086A80038B54FF47A7441F288352046FEF794F8CD
:1086B8000134C0B2A4B200F06FF9AC42F5D138BDB4
:1086C800054B06491A6801EB8201013202F01F02CC
:1086D80081ED000A1A607047404C0020CC4C002005
:1086E800054B06491A6801EB8201013202F01F02AC
:1086F80081ED000A1A607047E05E0020504C0020AF
:10870800094A0A4913680968994209D0084901EBDE
:108718008301013303F01F0391ED000A13607047D2
:108728009FED040A704700BF4C4C0020404C0020CD
:10873800CC4C002000000000094A0A491368096867
:10874800994209D0084901EB8301013303F01F0363
:1087580091ED000A136070479FED040A704700BF4F
:10876800084F0020E05E0020504C00200000000070
:10877800024A00231360024A136070474C4C0020E1
:10878800404C0020024A00231360024A13607047DD
:10879800084F0020E05E002070477047FEE7FEE7C4
:1087A800FEE7704770477047FEF7E0BD08B5022046
:1087B80003F002FE48B1054BD3F880305B69984757
:1087C8000220BDE8084003F005BE08BD9040002027
:1087D80000F062BA014802F0DBBA00BF903A00200C
:1087E800704700BF414BD3F8882042F47002C3F8A9
:1087F80088203F4B1A6842F001021A6000229A60F2
:10880800196821F0847121F480311960394959605F
:10881800196882B021F480211960DA60009201920F
:108828001A6842F480321A601A6802F4003201921F
:10883800009A01320092019A1AB9009AB2F5A06F13
:10884800F2D12B4B1B6813F4003318BF012301939B
:10885800019B012B2ED1264B1A6C42F080521A64D0
:10886800254A116841F4804111609A689A609A68B3
:1088780042F400429A609A6842F4A0529A601F4AF1
:108888005A601A6842F080721A601968184A890199
:10889800FBD51B4B40F205611960936823F0030375
:1088A8009360936843F002039360936803F00C03AA
:1088B800082BFAD10E4B9A6822F400029A60114AEA
:1088C800C3F884201A6842F080621A601A6812019C
:1088D800FCD5064B4FF000629A60D3F8882042F42A
:1088E8007002C3F8882002B0704700BF00ED00E0B6
:1088F800003802401030002400700040085440073F
:10890800003C024080400030184B194A996801F039
:108918000C01042903D0082903D0164B19E0164B83
:1089280017E059685A6811F4800F596814BF124B40
:10893800104B02F03F02B3FBF2F30C4A5268C2F349
:108948000142C1F38811013252004B43B3FBF2F3E9
:10895800074A1360054B9A68054BC2F303129A182D
:108968001968127921FA02F21A6070470038024039
:10897800A40100200024F40000127A0008B5402069
:1089880003F01AFD30B1FBF7DDFE4020BDE80840DA
:1089980003F020BD08BD0000014608B5044805F0F5
:1089A800D5FC0348402105F07EFD0028F9D008BD1C
:1089B80000440040F0B589B04FF4E1330120019341
:1089C80000232B4CADF808301E460146ADF80A309E
:1089D800ADF80C30ADF810300C23ADF80E3004F0C3
:1089E80045FB4FF40030012104F064FB20680221AC
:1089F800072204F013F807226068032104F00EF838
:108A08000125022704232068059305A98DF81A601B
:108A18008DF81B508DF818708DF8197003F07EFFD3
:108A280008236068059305A98DF8187003F076FF90
:108A3800A06801A905F0E0FB2A4640F225510D483F
:108A480005F018FD262307A88DF81C308DF81D6049
:108A58008DF81E608DF81F5000F06EFBA068294647
:108A680005F047FC044A054B1A6009B0F0BD00BF89
:108A7800B801002000440040A18900082C5F0020B4
:108A8800024B9868002105F034BC00BFB8010020F3
:108A980010B5094C40F22551204605F00EFD50B1A5
:108AA800A288D2B2112A02D1044B01211970044BB9
:108AB80019884A401A8010BD00440040160C002056
:108AC800900C00201FB5214B0C46186000214FF078
:108AD800804004F02CFF012100224FF0804005F077
:108AE80056FA022C01D10B2303E0012C02D142F6E5
:108AF800DF6302930523ADF804304FF08040002374
:108B080001A9ADF80C30ADF8063004F07BFE4FF04B
:108B18008040012105F05BFA4FF08040012104F00C
:108B2800E4FE01210A464FF0804005F030FA4FF08C
:108B38008040012104F0FBFE044B19680029FCD198
:108B48004FF0804004F0F3FE1FBD00BF940C0020DE
:108B58007047F0B5012085B02D4D014604F086FA26
:108B68004FF4D0530026019303270223284601A976
:108B78008DF808308DF809708DF80A608DF80B6053
:108B880003F0CCFE284609210A2203F047FF2846B5
:108B98000B210A2203F042FF0A2228460C2103F087
:108BA8003DFF01244FF48063284601A901938DF805
:108BB8000A408DF80B408DF8097003F0AFFE0A21CA
:108BC8000A46284603F02AFF21464FF4804004F065
:108BD8007DFA8020214604F055FA31464FF00060B6
:108BE80000F0DEFA4FF4A06000F09CFA1C2303A802
:108BF8008DF80C308DF80D608DF80E408DF80F4013
:108C080000F09AFA2046214604F054FA05B0F0BD67
:108C18000000024007B54FF4C06000F083FA432318
:108C28008DF8043001A801238DF805308DF8063041
:108C38008DF8073000F080FA0EBD044811B9012103
:108C480003F0DDBE012103F0DCBE00BF00080240D6
:108C5800022137E7012135E737B5042001210D4D01
:108C680004F004FA022301248DF805302846002375
:108C780069468DF806308DF8073000948DF8044069
:108C880003F04CFE2846214603F0B9FEC820FFF742
:108C9800E1FF3EBD0008024008B54FF080400121C9
:108CA80005F08AF988B101214FF0804005F08FF96D
:108CB800064B196819B11A68013A1A6008BD4FF0D5
:108CC8008040BDE8084004F032BE08BD940C002086
:108CD8007047012070470349034A02204FF4B773D5
:108CE80000F09CB89EA00508EC9504080349044AC6
:108CF800022040F2371300F091B800BF9EA005088B
:108D0800FC9504080349044A022040F2011300F0CC
:108D180085B800BF9EA00508199604080249034AB1
:108D28000220F52300F07AB89EA0050832960408C0
:108D38000249034A0220EA2300F070B89EA0050801
:108D48004C9604080249034A0220DF2300F066B863
:108D58009EA00508649604080249034A0220C82315
:108D680000F05CB89EA00508819604080249034AF1
:108D78000220BC2300F052B89EA00508A69604085D
:108D88000249034A0220A62300F048B89EA005081D
:108D9800C59604080249034A02208B2300F03EB816
:108DA8009EA00508E39604080249034A022080238E
:108DB80000F034B89EA00508009704080249034A49
:108DC8000220682300F02AB89EA005081597040819
:108DD8000249034A0220522300F020B89EA0050849
:108DE8002F970408FDF730BFFDF736BF04490A681E
:108DF80001320A6003490346022000F00FB800BFA1
:108E0800980C0020BFA00508FDF72CBF80F080005B
:108E1800092801D8FDF7ECBE704700BF0EB403B0B7
:108E280070470A2810B5044602D10D20FFF7F9FF54
:108E3800064A13681BB103F8014B136010BD044BBD
:108E48001B680BB12046984710BD00BF9C0C002042
:108E58002C5F002010B5044601E0FFF7E2FF14F88C
:108E6800010B0028F9D110BD2DE9F04F044685B05B
:108E78000D464FF00A0A00E035462078002800F039
:108E8800C480252801D0013467E06078302803D1F8
:108E9800A0780123033407E02D2802D002340023F0
:108EA80002E0A078022303344FF0000805E00AFB33
:108EB800080814F8010BA8F13008A0F13002D2B26A
:108EC800092AF4D96C2801D04C2803D114F8010BD5
:108ED80043F00403002800F09880602886BFA0F1C2
:108EE8002002D2B202464F2A3DD006D8432A2DD0BE
:108EF800442A09D0422A30D133E0552A04D0582ACE
:108F080029D0532A29D101E00A272DE02E1D2F68E8
:108F1800002500E001357A5D002AFBD104E020201D
:108F2800FFF77FFF4D4601E0980704D4454505F15A
:108F38000109F4D34D463846FFF78CFF03E02020A3
:108F4800FFF76FFF01354545F9D395E728782E1DC2
:108F5800FFF767FF90E7102706E0FFF762FF2E464E
:108F68008AE7022700E008272E1D442A296804D131
:108F7800002902DA494243F00803002200E02A46A9
:108F8800B1FBF7FE07FB1E11CDB2092D714607D9BB
:108F9800782814BF4FF0070C4FF0270C6544EDB24A
:108FA80030350DF80250551CBEF1000F02D0102DBF
:108FB800E5D10F22190705D504A94D192D2105F86A
:108FC800101C951C13F0010F0CBF4FF0200B4FF035
:108FD800300B9B072F4604D508E05846FFF721FFC2
:108FE8004F46474507F10109F7D34F46013D1DF8A4
:108FF8000500FFF716FF002DF8D103E02020FFF74A
:1090080010FF01374745F9D336E705B0BDE8F08FC3
:1090180070B5064D0C462E68286001E0FFF701FF89
:1090280014F8010B0028F9D12E6070BD2C5F0020C8
:109038000FB407B504A951F8040B0191FFF714FF09
:10904800BDE80E4004B070470EB417B505A9084C2A
:1090580051F8043B206018460191FFF705FF22688C
:10906800002313702360BDE81E4003B0704700BFA3
:109078009C0C00200EB433B505A9074C51F8043BED
:109088002568206018460191FFF7EEFE2560BDE8CF
:109098003C4003B0704700BF2C5F002070B51E46EF
:1090A80004461C481546FFF7C3FF022E1FD0042EA6
:1090B80025D0012E2AD105E0A15D1748FFF7B8FF9A
:1090C800013600E00026AE42F6DB2020FFF7A9FEBD
:1090D800002609E0A05DA0F12003DBB25E2B88BF6B
:1090E8002E20FFF79EFE0136AE42F3DB0EE034F889
:1090F800021B0A48FFF79CFF013DF8D106E054F82F
:10910800041B0748FFF794FF013DF8D10A20BDE88A
:10911800704086E6E2A00508E9A00508EFA005086A
:10912800F5A0050840F0BE60024B40F42020D8604E
:10913800704700BF00ED00E0C37810B503B3164BCD
:109148004278DB688478DB43C3F30223C3F104016C
:10915800C9B202FA01F10F2242FA03F2C9B222405F
:109168000A430E4B01781201CB18D2B283F80023C0
:1091780003780122590903F01F0302FA03F307E0F9
:1091880003780122590903F01F0302FA03F320317F
:10919800024A42F8213010BD00ED00E000E100E095
:1091A80021F0604121F07F01014B0843986070472E
:1091B80000ED00E0044B1A6909B1104301E022EA0E
:1091C80000001861704700BF00ED00E0044B1A680A
:1091D80004280CBF42F0040222F004021A6070470F
:1091E80010E000E037B50023104C0193054603203A
:1091F800FFF72EFDEB681A69013C019213D0019A22
:10920800002AF4DA019A42F001020192019A1A61E5
:10921800064A1969013A019102D00199C907F8D49F
:109228000320FFF715FD00203EBD00BF410D0300E0
:1092380010B5C47874B900EB820003339B10D0F8E2
:10924800D000224603E051F8044C01320460043196
:109258009A42F8D1002010BD033230B59210D0F8F0
:10926800D0400B46002003E02568013043F8045C39
:1092780004339042F8D101EB800030BD0122F0B5F3
:109288000023827040220129C37082800CD10823F8
:109298000370042343704FF4A073C3800223037246
:1092A800C1724FF0A04309E041B90C2303700623B3
:1092B80043704FF4A063C3801F4BC17203F5006273
:1092C8000261C3604678044601461A46002508E054
:1092D80002F5106C02F530620A65C1F814C0013558
:1092E8003A460431B54202F12007F1D303F5806212
:1092F800426103F58862C0F8CC20067803F5A065C2
:109308000146002203E0C1F88C50013220350431B7
:10931800B242F8D31946002202E0C4F8CC10013258
:109328000434B24201F58051F7D303F56063C0F805
:109338000C310020F0BD00BF0000044038B5037AAE
:10934800C2680025012B04461FD1936B417A65F34F
:10935800104309B143F480139363D3686FF3861302
:109368006FF396536FF351436FF3D343D3602046A3
:10937800FFF738FFE378012B19D1052363F3440580
:10938800E36845F020059D6011E0D36843F0400391
:10939800D360FFF727FF637AE268002B0CBF4FF416
:1093A80004134FF4441393631420FFF753FCE3783A
:1093B800012B07D1E3689D68052262F3440545F057
:1093C80020059D60002038BDC3689A6842F00102FC
:1093D8009A6000207047C3689A6822F001029A6078
:1093E8000020704707B500230193019B43F0200339
:1093F8000193019B61F38A130193019BC268136176
:10940800064B1169013B019102D001998806F8D4F5
:109418000320FFF71DFC00200EBD00BF410D030017
:1094280007B500230193019B43F010030193019BAF
:10943800C2681361064B1169013B019102D0019981
:10944800C906F8D40320FFF703FC00200EBD00BFB7
:10945800410D030008B5C268D36801296FF35D7335
:109468006FF39E7302D143F0005302E009B943F051
:1094780080433220D360FFF7EDFB002008BDC368AE
:10948800586900F001007047C3685B6913F0010F69
:1094980014BF002001207047C368586900F001001C
:1094A8007047C3685A69986910407047C36858681C
:1094B800704743699B6813F0010F14BF0020012017
:1094C8007047C36800229A614FF0FF325A615A60B0
:1094D8006FF080425A610B4A9A61C2789969002AF2
:1094E8000CBF1022002242F0487221EA02010A430E
:1094F8009A619A6922F0005222F008029A610020CB
:10950800704700BF0008008043691A6861F30102D0
:109518001A607047D0F8CC3018686FF382006FF388
:1095280041006FF3C3006FF34510704738B5044628
:109538000D46FFF782FB2046FFF7ECFFC0F3072339
:1095480003F01003DBB233B9012D04D1D4F8CC30C9
:1095580040F480501860C0F3072303F01003DBB217
:109568002BB125B9D4F8CC3065F30C301860C8207D
:10957800BDE83840FFF76EBB43695869704738B596
:109588000546FFF7C7FFD5F8CC3040F480741C605F
:109598006420FFF75FFBD5F8CC306FF30824142064
:1095A8001C60FFF757FB012038BD70B50446FFF774
:1095B80053FBD4F80C3100251D60237A012B08BF1A
:1095C8002946204618BF0121FFF79EFF2046FFF7D6
:1095D800D6FF63691A686FF382021A60E37A012B77
:1095E8002E460ED1E36880225A6262F30F05E0220C
:1095F80062F30F06C0F26005C0F260069D62C3F810
:10960800006110212046FFF7EDFE2046FFF708FF16
:10961800002322464FF0FF35184604E0D2F88C109C
:1096280001338D60C860217804328B42F6D320461E
:109638000121FFF77BFF2046FFF743FF002070BDA5
:1096480070B500EB810301F11504D3F8902000EB0D
:1096580044154FF0FF339360C37895F81551012BEB
:109668000CBF04230023032D2BD8DFE805F0021FCD
:10967800021300EB411404F56C7443F08903A578D8
:1096880043F482637DB9247943F04003CCB143F0BD
:10969800200316E000EB411443F0990394F8B24319
:1096A80043F4C0636CB143F480730AE000EB4414E4
:1096B80043F0010394F8124143F408730CB143F4E6
:1096C800C073D360436901249D6904FA01F42C43F3
:1096D8009C61C3689C69153100EB411044F000742B
:1096E8009C6190F81011002361F39C5390F81111BC
:1096F80061F3CE2390F8121161F3CF3390F8131170
:10970800A1F1020CDCF1000141EB0C0161F35143C2
:1097180090F8151100F58874B0F8160161F39343B9
:1097280060F30A03032908BF43F0005313600020C5
:1097380070BD70B501F11E04640186B003590A4674
:10974800002583B100EB4111013BB1F8B6135B185A
:10975800B3FBF1F39BB2B3F5807F05D90902015140
:109768004FF4807300E0012300EB421191F8B243FB
:1097780001F56C712CB1C98800EB42145943C4F847
:10978800C01300EB4211D1F8C01361F3120563F363
:10979800DC4500EB421393F8B84364F35E7500EBC5
:1097A8008204D4F890402561C578012D08BFD3F80C
:1097B800BC33456908BF63612368AE6816F0010FC2
:1097C80014BF0026012666F35D7343F000436FF370
:1097D8009E732360C378002B31D102F1150300EB8F
:1097E800431393F8124154BB49B393F81531032B33
:1097F8001DD8DFE803F0020F020FC368DC6A0331EB
:109808000194C1F38F01A4B28C4210D2996941F03E
:1098180020010BE02B6903310493C1F38F019BB244
:109828008B4204D2C368996941F08061996100EB69
:109838004211B1F8C033D1F8BC13FFF7F9FC00208E
:1098480006B070BD00EB810186B0D1F89020136896
:1098580043F04043C3F3074111F00C0101D008293C
:1098680002D1C168C96A01E041690969C1F30741C8
:1098780009B961F3DF731360002006B0704703462F
:1098880010B503EB81030124D3F890304FF0004268
:1098980064F3DC421A611A68002042F0004260F367
:1098A8009E721A6010BD43694FF0FF31002210B557
:1098B8009A610446596101460AE0D1F88C000368B0
:1098C8006FF3DF7343F080436FF3CF3303600132EC
:1098D800237804319A42F0D32046FFF7A1FD2046B1
:1098E8001021BDE810407DE5002310B51A46044656
:1098F800C0F8103303F1C60044F8202003F1D40067
:1099080004EB80004260E01801330F2B80F89023AD
:10991800F0D10823A4F8B6332046FFF7AFFC204661
:10992800FFF759FD2046FFF709FD01212046FFF703
:1099380091FD2046FFF739FE2046FFF745FD002040
:1099480010BDD0F8CC301868C0F34140704708B556
:10995800FFF715FE002008BDD0F810037047D0F8B7
:10996800140370474369986880B27047401890F8AC
:109978009F037047D43100EB81004068704740185E
:1099880090F89003704708B5FFF75AFE08BD4218D3
:1099980008B5002382F89F3301F11E0200EB421242
:1099A8005360FFF7C6FE08BD80B584B000AF78608D
:1099B8004FF00003FB6040F20C23C2F200031B6867
:1099C8001B6878689847FB6843F00803FB607B686E
:1099D800DB68FA685A614FF00103184607F110076F
:1099E800BD4680BD80B584B000AF78604FF00003FD
:1099F800FB6040F20C23C2F200031B689B68786886
:109A08009847FB6843F00053FB607B68DB68FA68A3
:109A18005A614FF00103184607F11007BD4680BD93
:109A280080B485B000AF78607B68D3F890301B684D
:109A3800BB60BB6843F00043BB60BB6843F0804336
:109A4800BB607B68D3F89030BA681A604FF00003A7
:109A5800FB60FB6843F40013FB607B68DB68FA6813
:109A68005A614FF00103184607F11407BD4680BC40
:109A7800704700BF80B588B000AF78604FF0000332
:109A8800FB724FF000037B617B6943F010037B613D
:109A98007B68DB687A68D268926911467A696FEAEE
:109AA80002020A409A617B68DB681B6ABB61BB697A
:109AB800C3F30303DBB2FB72FB7ADBB27A6803F110
:109AC80022034FEA8303D3189B681B68FB60BB69BA
:109AD800C3F34343DBB2022B40F09A80BB69C3F364
:109AE8000A139BB2002B40F39480FB7ADBB27A68AE
:109AF8004FEA4313D31803F56F731B68002B00F06C
:109B08008880FB7ADBB27A684FEA4313D31803F5EF
:109B18006F731A68BB69C3F30A139BB2786811465E
:109B28001A46FFF799FBBB69C3F30303DBB2BA69B3
:109B3800C2F30302D2B279684FEA42128A1802F5D8
:109B48006F721168BA69C2F30A1292B28A187968F8
:109B58004FEA4313CB1803F56F731A60BB69C3F35D
:109B68000303DBB2BA69C2F30302D2B2796802F125
:109B78001E024FEA42128A1802F104021168BA69F9
:109B8800C2F30A1292B28A18796803F11E034FEAE7
:109B98004313CB1803F104031A60FB7ADBB27A682B
:109BA80003F11E034FEA4313D31803F104031B68A0
:109BB800FB61FB7ADBB27A6803F1D4034FEA8303D3
:109BC800D318FA695A60FB7ADBB27A6803F1220388
:109BD8004FEA8303D3189B681B693B613B69C3F356
:109BE800C9439BB2002B14DDFB6843F00043FB60C4
:109BF800FB686FF39E73FB60FB7ADBB27A6803F154
:109C080022034FEA8303D3189B68FA681A6000E0BE
:109C180000E000BF7B6943F010037B617B68DB6871
:109C28007A68D268926911467A690A439A614FF054
:109C38000103184607F12007BD4680BD80B59CB0DA
:109C480000AF786039607A683B6803F122034FEA15
:109C58008303D3189B68FB66FB6E9B68BB66FB6E31
:109C6800DB687B66BA6E7B6E1340BB667A683B68BE
:109C780003F122034FEA8303D3189B681B683B66F2
:109C88004FF000037B6697F8683003F00403DBB2FB
:109C9800002B22D04FF00003BB65BB6D43F00403DB
:109CA800BB65BA6DFB6E9A607A683B6803F1220364
:109CB8004FEA8303D3189B68DB687B657B6D43F0B1
:109CC80002037B657A683B6803F122034FEA83034A
:109CD800D3189B687A6DDA6098E097F8683003F0DB
:109CE8002003DBB2002B0AD04FF000033B653B6D2D
:109CF80043F020033B653A6DFB6E9A6086E097F867
:109D0800683003F00803DBB2002B3ED07A683B686A
:109D180003F122034FEA8303D3189B68DB68FB64D3
:109D2800FB6C43F00203FB647A683B6803F122038F
:109D38004FEA8303D3189B68FA6CDA607A683B6849
:109D4800D31803F564734FF005021A704FF000033F
:109D5800BB64BB6C43F01003BB64BA6CFB6E9A60C7
:109D68004FF000037B647B6C43F008037B647A6CE0
:109D7800FB6E9A60BB6E6FF30413BB663B68DBB285
:109D880078681946FFF75EFD40E097F8693003F000
:109D98000403DBB2002B39D07A683B6803F1220355
:109DA8004FEA8303D3189B68DB683B643B6C43F042
:109DB80002033B647A683B6803F122034FEA83039A
:109DC800D3189B683A6CDA603B68DBB2786819464E
:109DD800FFF738FD4FF00003FB63FB6B43F0100304
:109DE800FB63FA6BFB6E9A607A683B68D31803F5DD
:109DF80064734FF008021A704FF00003BB63BB6B2B
:109E080043F48063BB63BA6BFB6E9A6097F8693062
:109E180003F00203DBB2002B28D07A683B6803F119
:109E280022034FEA8303D3189B68DB687B637B6B51
:109E380043F002037B637A683B6803F122034FEA2D
:109E48008303D3189B687A6BDA603B68DBB2786867
:109E58001946FFF7F7FC4FF000033B633B6B43F4F5
:109E680000733B633A6BFB6E9A60DEE197F86830EB
:109E780003F00103DBB2002B00F0A5807B68DB78E0
:109E8800012B1DD17A683B6803F122034FEA830353
:109E9800D3189B681B69FB657A683B6803F11E034E
:109EA8004FEA4313D3181A68FB6DC3F31203D21A8F
:109EB80079683B6803F1D4034FEA8303CB185A60EF
:109EC8007A683B68D31803F564734FF001021A707F
:109ED8007B683A6802F1C6024FF0000143F822108D
:109EE8004FF00003FB62FB6A43F00103FB62FA6A6E
:109EF800FB6E9A6097F8623003F00C03DBB2002B1C
:109F080006D097F8623003F00C03DBB2082B3BD184
:109F18007A683B6803F122034FEA8303D3189B68EE
:109F2800DB68BB62BB6A43F00203BB627A683B68CA
:109F380003F122034FEA8303D3189B68BA6ADA60F5
:109F48003B68DBB278681946FFF77CFC4FF00003EA
:109F58007B627B6A43F010037B627A6AFB6E9A60CD
:109F68007A683B684FEA4313D31803F572731B787A
:109F780083F00103DAB279683B684FEA4313CB18E0
:109F880003F572731A7050E197F8623003F00C030E
:109F9800DBB20C2B40F048813B6E43F000533B662C
:109FA8007A683B6803F122034FEA8303D3189B685E
:109FB8003A6E1A607A683B68D31803F566734FF0F7
:109FC8000102DA7130E197F8683003F00203DBB27E
:109FD800002B00F084807A683B6803F122034FEA83
:109FE8008303D3189B68DB683B623B6A6FF34103CA
:109FF8003B627A683B6803F122034FEA8303D31874
:10A008009B683A6ADA607A683B68D31803F5647328
:10A018001B78DBB2012B08D17A683B68D31803F5AB
:10A0280066734FF00102DA714EE07A683B68D31824
:10A0380003F564731B78DBB2052B08D17A683B689B
:10A04800D31803F566734FF00402DA713CE07A68BE
:10A058003B68D31803F564731B78DBB2062B08D072
:10A068007A683B68D31803F564731B78DBB2082B56
:10A0780010D17B683A6802F1C6024FF0000143F83C
:10A0880022107A683B68D31803F566734FF0030211
:10A09800DA7119E097F8623003F00C03DBB20C2B8D
:10A0A80012D17A683B684FEA4313D31803F57273E9
:10A0B8001B7883F00103DAB279683B684FEA4313EF
:10A0C800CB1803F572731A704FF00003FB61FB693C
:10A0D80043F00203FB61FA69FB6E9A60A5E097F80A
:10A0E800683023F07F03DBB2002B3ED07A683B68F0
:10A0F80003F122034FEA8303D3189B68DB68BB6133
:10A10800BB6943F00203BB617A683B6803F1220331
:10A118004FEA8303D3189B68BA69DA607B683A68A8
:10A1280002F1C60253F8223003F101017B683A6854
:10A1380002F1C60243F822107A683B68D31803F587
:10A1480064734FF006021A703B68DBB278681946F0
:10A15800FFF778FB4FF000037B617B6943F08003D6
:10A168007B617A69FB6E9A605FE097F8683003F06C
:10A178001003DBB2002B58D097F8623003F00C03C1
:10A18800DBB20C2B1DD17A683B6803F122034FEA3E
:10A198008303D3189B68DB683B613B6943F0020388
:10A1A8003B617A683B6803F122034FEA8303D318C3
:10A1B8009B683A69DA603B68DBB278681946FFF752
:10A1C80041FB7A683B68D31803F564734FF00302C8
:10A1D8001A704FF00003FB60FB6843F01003FB604C
:10A1E800FA68FB6E9A6097F8623003F00C03DBB2F2
:10A1F800002B06D097F8623003F00C03DBB2082B73
:10A2080013D13B6E43F000433B663B6E6FF39E7386
:10A218003B667A683B6803F122034FEA8303D3184D
:10A228009B683A6E1A6000E000BF4FF001031846C1
:10A2380007F17007BD4680BD80B59AB000AF786061
:10A2480039607A683B6803F122034FEA8303D31825
:10A258009B687B667B6E9B683B667B6EDB68FB65F9
:10A268003A6EFB6D13403B667A683B6803F1220344
:10A278004FEA8303D3189B681B68BB6597F8603067
:10A2880003F00403DBB2002B22D04FF000037B6500
:10A298007B6D43F004037B657A6D7B6E9A607A6808
:10A2A8003B6803F122034FEA8303D3189B68DB68FA
:10A2B8003B653B6D43F002033B657A683B6803F1FD
:10A2C80022034FEA8303D3189B683A6DDA6080E271
:10A2D80097F8603003F02003DBB2002B0AD04FF070
:10A2E8000003FB64FB6C43F02003FB64FA6C7B6E99
:10A2F8009A606EE297F8613003F00203DBB2002B3C
:10A3080028D07A683B6803F122034FEA8303D31805
:10A318009B68DB68BB64BB6C43F00203BB647A6870
:10A328003B6803F122034FEA8303D3189B68BA6C96
:10A33800DA603B68DBB278681946FFF783FA4FF0BA
:10A3480000037B647B6C43F400737B647A6C7B6EE4
:10A358009A603EE297F8603003F00103DBB2002B0D
:10A3680038D07B683A6802F1C6024FF0000143F822
:10A3780022107A683B6803F122034FEA8303D3185B
:10A388009B68DB683B643B6C43F002033B647A6880
:10A398003B6803F122034FEA8303D3189B683A6CA6
:10A3A800DA603B68DBB278681946FFF74BFA4FF082
:10A3B8000003FB63FB6B43F00103FB63FA6B7B6EEB
:10A3C8009A607A683B68D31803F564734FF001020A
:10A3D8001A70FEE197F8603003F00803DBB2002B37
:10A3E80030D04FF00003BB63BB6B43F00803BB6383
:10A3F800BA6B7B6E9A607A683B6803F122034FEA76
:10A408008303D3189B68DB687B637B6B43F0020391
:10A418007B637A683B6803F122034FEA8303D3180E
:10A428009B687A6BDA603B68DBB278681946FFF79D
:10A4380009FA7A683B68D31803F564734FF005028C
:10A448001A70C6E197F8603003F01003DBB2002BF6
:10A4580038D07B683A6802F1C6024FF0000143F831
:10A4680022107A683B6803F122034FEA8303D3186A
:10A478009B68DB683B633B6B43F002033B637A6892
:10A488003B6803F122034FEA8303D3189B683A6BB6
:10A49800DA603B68DBB278681946FFF7D3F94FF00A
:10A4A8000003FB62FB6A43F01003FB62FA6A7B6EEF
:10A4B8009A607A683B68D31803F564734FF0030217
:10A4C8001A7086E197F8603023F07F03DBB2002B27
:10A4D8003ED07A683B6803F122034FEA8303D3181E
:10A4E8009B68DB68BB62BB6A43F00203BB627A68A5
:10A4F8003B6803F122034FEA8303D3189B68BA6AC7
:10A50800DA603B68DBB278681946FFF79BF97B682D
:10A518003A6802F1C60253F8223003F101017B6860
:10A528003A6802F1C60243F822107A683B68D318E9
:10A5380003F564734FF006021A704FF000037B6254
:10A548007B6A43F080037B627A6A7B6E9A6040E1A3
:10A5580097F8603003F04003DBB2002B38D07B68FB
:10A568003A6802F1C6024FF0000143F822107A68F7
:10A578003B6803F122034FEA8303D3189B68DB6827
:10A588003B623B6A43F002033B627A683B6803F133
:10A5980022034FEA8303D3189B683A6ADA603B6860
:10A5A800DBB278681946FFF74DF94FF00003FB61FD
:10A5B800FB6943F04003FB61FA697B6E9A607A6835
:10A5C8003B68D31803F564734FF004021A7000E176
:10A5D80097F8613003F00403DBB2002B3AD07A68B5
:10A5E8003B6803F122034FEA8303D3189B68DB68B7
:10A5F800BB61BB6943F00203BB617A683B6803F146
:10A6080022034FEA8303D3189B68BA69DA603B6870
:10A61800DBB278681946FFF715F94FF000037B6144
:10A628007B6943F010037B617A697B6E9A607A6874
:10A638003B68D31803F564734FF008021A704FF0A3
:10A6480000033B613B6943F480633B613A697B6E7D
:10A658009A60BEE097F8603003F00203DBB2002B8B
:10A6680000F0B7807A683B6803F122034FEA83035E
:10A67800D3189B68DB68FB60FB686FF34103FB60E2
:10A688007A683B6803F122034FEA8303D3189B6877
:10A69800FA68DA607A683B68D31803F564731B7844
:10A6A800DBB2012B22D17A683B68D31803F56673B5
:10A6B8004FF00102DA7197F85A3003F00C03DBB25D
:10A6C800082B7CD17A683B684FEA4313D31803F50B
:10A6D80072735B7883F00103DAB279683B684FEAFA
:10A6E8004313CB1803F572735A7068E07A683B68B5
:10A6F800D31803F564731B78DBB2032B08D17A688F
:10A708003B68D31803F566734FF00202DA7156E01E
:10A718007A683B68D31803F564731B78DBB2042BA3
:10A728001AD17A683B6803F115034FEA4313D3182B
:10A7380003F588731B79012B05D13B68DBB2786878
:10A748001946FFF79CF87A683B68D31803F56673D7
:10A758004FF00202DA7132E07A683B68D31803F5E9
:10A7680064731B78DBB2052B08D17A683B68D31871
:10A7780003F566734FF00402DA7120E07A683B68EB
:10A78800D31803F564731B78DBB2062B17D17B68EB
:10A798003A6802F1C60253F82230032B0FD17A68C7
:10A7A8003B68D31803F566734FF00302DA717B68D0
:10A7B8003A6802F1C6024FF0000143F822104FF048
:10A7C8000003BB60BB6843F00203BB60BA687B6EE2
:10A7D8009A604FF00103184607F16807BD4680BD2F
:10A7E80080B588B000AF78604FF00003FB614FF090
:10A7F8000003FB604FF000033B614FF00003BB61B7
:10A808004FF000037B617B68D3F8CC301B68BB61D9
:10A818007B68D3F8CC301B687B617B696FF382035C
:10A828007B617B696FF341037B617B696FF3C303D2
:10A838007B617B696FF345137B613B7E03F0020309
:10A84800DBB2002B0FD07B6943F002037B6140F23F
:10A858000C23C2F200031B685B6878689847FB69A1
:10A8680043F00103FB613B7E03F00803DBB2002BDE
:10A8780075D07B6943F008037B613B7E03F00403DA
:10A88800DBB2002B63D0BB7E03F00603DBB2042BE4
:10A8980005D0BB7E03F00603DBB2022B35D17B6803
:10A8A8005B691B683B61BB7E03F00603DBB2042BCC
:10A8B80017D17B685B6941F270725A603B7C03F088
:10A8C8000303DBB2022B24D07B681B7A022B04D152
:10A8D80078684FF00201FEF717FE7868FEF74FFE22
:10A8E80017E07B685B694BF680325A603B7C03F06B
:10A8F8000303DBB2012B0CD078684FF00101FEF79F
:10A9080003FE7868FEF73BFE03E07868FEF737FE43
:10A9180000E000BF40F20C23C2F200031B68DB68B2
:10A92800786898474FF00003FB60FB6843F00053DA
:10A93800FB607B68DB687A68D26892691146FA68BE
:10A948006FEA02021140FA680A439A6107E040F28E
:10A958000C23C2F200031B681B69786898473B7E8A
:10A9680003F02003DBB2002B07D07B6943F0200300
:10A978007B61FB6943F00103FB617B68D3F8CC3052
:10A988007A691A60FB69184607F12007BD4680BD41
:10A9980080B586B000AF78607B685B691B69BB6077
:10A9A8003B7BC3F3C303DBB27A6803F11E034FEAB0
:10A9B8004313D3181B6803F103034FEA9303FB8285
:10A9C800A3E03B894FEA8303BB82BA8A3B7BC3F38C
:10A9D800C303DBB2796803F11E034FEA4313CB18B4
:10A9E8001B689A421DD93B7BC3F3C303DBB27A6869
:10A9F80003F11E034FEA4313D3181B68BB824FF0C1
:10AA080000033B613B6943F080633B617B68DB6823
:10AA18007A68D268926911463A696FEA02020A4076
:10AA28009A613B7BC3F3C303DBB27A6803F11E036D
:10AA38004FEA4313D3181B6803F103034FEA930348
:10AA4800FB823B7BC3F3C303DBB27A684FEA431351
:10AA5800D31803F56F7319683B7BC3F3C303DBB2E9
:10AA68001A46BB8A7868FEF7E3FB3B7BC3F3C30354
:10AA7800DBB23A7BC2F3C302D2B279684FEA421220
:10AA88008A1802F56F721168BA8A8A1879684FEACB
:10AA98004313CB1803F56F731A603B7BC3F3C303EF
:10AAA800DBB23A7BC2F3C302D2B2796802F11E026A
:10AAB8004FEA42128A181168BA8A8A1A796803F129
:10AAC8001E034FEA4313CB181A603B7BC3F3C3033F
:10AAD800DBB23A7BC2F3C302D2B2796802F11E023A
:10AAE8004FEA42128A1802F104021168BA8A8A18D7
:10AAF800796803F11E034FEA4313CB1803F10403EB
:10AB08001A607B685B691B69BB603B89FA8A9A4259
:10AB18000DD23B7BC3F3C303DBB27A6803F11E0398
:10AB28004FEA4313D3181B68002B7FF44AAF4FF04A
:10AB38000103184607F11807BD4680BD80B588B0E7
:10AB480000AF78607B68DB68DB6AFB603B7CC3F343
:10AB5800C303DBB27A6803F11E034FEA4313D31829
:10AB68001B6803F103034FEA9303FB83A3E0BB894C
:10AB78004FEA8303BB83BA8B3B7CC3F3C303DBB2CB
:10AB8800796803F11E034FEA4313CB181B689A42F6
:10AB98001DD93B7CC3F3C303DBB27A6803F11E0300
:10ABA8004FEA4313D3181B68BB834FF00003BB6104
:10ABB800BB6943F02003BB617B68DB687A68D268B5
:10ABC80092691146BA696FEA02020A409A613B7CAF
:10ABD800C3F3C303DBB27A6803F11E034FEA4313DE
:10ABE800D3181B6803F103034FEA9303FB833B7CF1
:10ABF800C3F3C303DBB27A684FEA4313D31803F5F0
:10AC08006F7319683B7CC3F3C303DBB21A46BB8B73
:10AC18007868FEF70DFB3B7CC3F3C303DBB23A7CD9
:10AC2800C2F3C302D2B279684FEA42128A1802F517
:10AC38006F721168BA8B8A1879684FEA4313CB1878
:10AC480003F56F731A603B7CC3F3C303DBB23A7C32
:10AC5800C2F3C302D2B2796802F11E024FEA42126D
:10AC68008A181168BA8B8A1A796803F11E034FEAA9
:10AC78004313CB181A603B7CC3F3C303DBB23A7CA3
:10AC8800C2F3C302D2B2796802F11E024FEA42123D
:10AC98008A1802F104021168BA8B8A18796803F1DC
:10ACA8001E034FEA4313CB1803F104031A607B68B1
:10ACB800DB68DB6AFB60BB89FA8B9A420DD23B7C6E
:10ACC800C3F3C303DBB27A6803F11E034FEA4313ED
:10ACD800D3181B68002B7FF44AAF4FF001031846C6
:10ACE80007F12007BD4680BD80B586B000AF78600B
:10ACF8004FF000037B614FF000033B617868FEF77B
:10AD08003BFC0346FB604FF000037B6134E0BB89EA
:10AD18001A467B6942FA03F303F00103DBB2002B06
:10AD280026D07A687B6903F122034FEA8303D3189C
:10AD38009B681B68BB607B7A23F07F03DBB2002B28
:10AD48000BD049F64543C0F60003786879699847FF
:10AD580003463A6913433B610AE04AF24123C0F6CD
:10AD6800000378687969984703463A6913433B6159
:10AD78007B6903F101037B617B681B781A467B6959
:10AD88009A42C4D83B69184607F11807BD4680BDEA
:10AD980080B584B000AF78604FF00003FB604FF0DF
:10ADA8000003BB607868FEF777FB0346002B00F0D2
:10ADB8008B807868FEF775FB0346BB60BB68002B89
:10ADC80002D14FF0000380E03B7A03F00803DBB2C6
:10ADD800002B09D049F6B113C0F6000378689847EC
:10ADE8000346FA681343FB603B7A03F01003DBB2B7
:10ADF800002B09D049F67D23C0F6000378689847F0
:10AE08000346FA681343FB603B7A03F02003DBB286
:10AE1800002B09D04AF64533C0F6000378689847F6
:10AE28000346FA681343FB60FB7A03F00403DBB2C2
:10AE3800002B09D04AF69913C0F6000378689847A2
:10AE48000346FA681343FB60FB7A03F00203DBB2A4
:10AE5800002B09D04AF6F143C0F6000378689847FA
:10AE68000346FA681343FB60FB7A03F00103DBB285
:10AE7800002B09D04AF2E973C0F6000378689847B6
:10AE88000346FA681343FB60FB7A03F02003DBB246
:10AE9800002B09D049F6ED13C0F6000378689847EF
:10AEA8000346FA681343FB60BB7A03F02003DBB266
:10AEB800002B09D049F62923C0F600037868984783
:10AEC8000346FA681343FB60FB68184607F110074E
:10AED800BD4680BD0123C0F8103300207047012310
:10AEE800C0F81433002070470023C0F81433184604
:10AEF80070470020704738B504460021FDF79DFED5
:10AF0800E36800254FF0FF329D6120465A61FEF745
:10AF180062FAC4F81053284638BD70B501230025DD
:10AF280040220C46CB700B778A7181F82130064697
:10AF38000D704D708D7081F82050097900F02BFB51
:10AF48006179304600F027FB284670BD2DE9F041B5
:10AF5800069F1646984604460D46FDF7FAFD002062
:10AF6800FDF77AFE31462046FFF7D7FF2946C6F897
:10AF78007C80C6F880702046FEF7B6FCD6F8803094
:10AF88001B6898472046BDE8F041FDF743BE0B1FFC
:10AF9800DBB2012B10B5044606D8D0F880305B6CC4
:10AFA80098470B23237010BD062905D10B23037086
:10AFB800D0F880301B68984710BD002370B58B749B
:10AFC8000B7F013B05460C460A2B00F2C980DFE8DF
:10AFD80013F00B001200390040005800650079009A
:10AFE80080009900A900B90001F11401627900F00C
:10AFF8003BFD022343E04979FEF7B8FC012819D14B
:10B00800237D618B584A03F0800339B141F28831BE
:10B0180011800BB1032307E0052305E032211180DD
:10B028000BB1092300E0072323772846FEF79AFC93
:10B03800208295E0032840F093800B232377052393
:10B04800A3748DE00B798A89896800F044FD042394
:10B0580015E00979FEF78AFC012802D10923237734
:10B0680003E0042823D0032808D02846FEF77AFCFA
:10B07800238AC01A3C4B1B88984271D90B2323772B
:10B088006EE04B7900EB4313012283F8C9234B7917
:10B098008A89896800F0FDFC0623F0E74979FEF704
:10B0A80065FC012801D10723E9E7042803D1637867
:10B0B80023700C23E3E7022801D10523DFE70328E7
:10B0C8004ED1DBE70B7900210A4600F004FD082386
:10B0D800D5E70979FEF74AFC0128064627D0032858
:10B0E800CCD02846FEF73EFC238AC01A1E4B1B888C
:10B0F8009842C3D8042E33D1637823700C23237766
:10B10800032070BD4B7900EB431393F8C92382F0F9
:10B11800010283F8C9234B7900210A4600F0B9FCE3
:10B128000A23ACE74979FEF721FC012803D16378AB
:10B1380023700D23A3E7022801D109239FE70328E1
:10B1480010D19BE78B7B0133DBB2022B8B7301D8C9
:10B15800012394E708238B744B7802200B7070BD91
:10B16800002070BD002070BDA00C002070B594B008
:10B17800022305460C468DF84F30FEF7EDFB18B15B
:10B188002846FEF7ECFB28B923781BB1032B01D026
:10B198000323237023780B2B00F29181DFE813F04F
:10B1A8000C001F0026006D018F01580040014C0162
:10B1B800590131018F015E012846FEF7CDFB0028B9
:10B1C80000F07D8101232370C820FDF743FD284648
:10B1D800FEF7BDFBD4F88030DB6898476FE1D5F8FF
:10B1E8001433012B40F06B81022367E1D4F88030DF
:10B1F8009B6898470021284600F0B4F980216071C7
:10B20800284600F0AFF920712846FEF79AFB05237F
:10B21800C0B22370D4F8803084F821009B69984725
:10B22800A079217994F8202094F821300190002603
:10B238002846009600F048F9A0796179019094F8C1
:10B24800202094F821300096284600F03DF936E198
:10B25800A378092B00F23381DFE813F00A002800F5
:10B26800380060006B007F009800B100C9002B0116
:10B2780028462146082200F01DFD0646002840F019
:10B288001E8194F829306179A3710122A27000907F
:10B29800019332463346284600F043F9A3792179D1
:10B2A8000193009628463246334634E02846214624
:10B2B800122200F0FFFC002840F00181D4F8803011
:10B2C80004F12200DB699847022330E02846214632
:10B2D800012200F045FD0646002840F0F0800220DB
:10B2E800FDF7B8FC012384F82030D4F880301B6ABD
:10B2F80098470323A370217994F8202000963346B9
:10B308002846019600F00DF9617994F820200096FE
:10B3180001962846334600F004F9D0E02846214635
:10B32800092200F019FE002840F0C9800423A37008
:10B33800C5E0E28E2846214600F00EFE002840F0C7
:10B34800BE80D4F8803004F134005B6A04F13E0119
:10B3580004F1500298470523E9E794F8302072B1C8
:10B36800FF2300932846214603AB00F07BFC00280E
:10B3780040F0A580D4F8803003A89B6A03E0D4F895
:10B38800803050489B6A98470623D0E794F83120CC
:10B3980072B1FF2300932846214603AB00F062FCFC
:10B3A800002840F08C80D4F8803003A8DB6A03E0E2
:10B3B800D4F880304348DB6A98470723B7E794F806
:10B3C80032206AB1FF2300932846214603AB00F0E0
:10B3D80049FC002873D1D4F8803003A81B6B03E024
:10B3E800D4F8803037481B6B984708239FE794F8B8
:10B3F80039202846214600F0C0FC00285FD10923E7
:10B4080095E7D4F880309B6B9847012857D1E36FB4
:10B4180028461B6821469847002850D106234DE04E
:10B42800E36F28469B68214698478DF84F009DF8A2
:10B438004F3043B9072341E0E36F2846DB682146D4
:10B4480098478DF84F009DF84F102046FFF79FFD55
:10B4580035E028462146FFF7B0FD30E02146284672
:10B46800FFF75BFDD4F880305B689847E36F04F121
:10B4780020015B682846984721E0D4F880301B6992
:10B48800984721462846FFF748FDD4F880305B6886
:10B498009847E36F04F120015B68284698472846DF
:10B4A80000F085F80023237028460121FEF71CFAD6
:10B4B80005E0D4F880305B6B98470923237014B0FB
:10B4C80070BD00BFFCA00508F8B501F5327430F86E
:10B4D800146001F1150400EB441406F07F0784F8AA
:10B4E80010219DF8182084F8117184F81521BDF8F1
:10B4F8001C2084F81331A4F81621C6F3C01600EBFB
:10B50800411204F5887584F81261002482F8C84352
:10B5180082F8C9430BB901232B71FEF791F800207B
:10B52800F8BD70B5BDF814401AB100EB411585F8A7
:10B53800B02301F1150200EB4215B5F81661A642D9
:10B5480005F5887501D004B1EC8000EB421292F841
:10B5580013419C4202D00BB182F81331FEF770F808
:10B56800002070BD10B502460023B2F99045002CAA
:10B5780008DB03F532726FEA41416FEA514120F866
:10B58800121006E00133DBB20232082BEDD14FF680
:10B59800FF73D8B210BD072907D801F5327130F80A
:10B5A800113023F4004320F81130002070470023A5
:10B5B800A0F89435A0F89635A0F89835A0F89A35F3
:10B5C800A0F89C35A0F89E3518467047F8B5314D5F
:10B5D80095F8423006460F46052B58D8DFE803F0A9
:10B5E8000357571309272B6D1B689847042385F8C1
:10B5F80042303046FDF75DFF012848D1254B032234
:10B6080083F8422043E095F8462095F840302149D8
:10B6180000F0A3FA204B01221A703046052385F862
:10B628004230FEF79FF980B2A5F84C002FE0FEF7F4
:10B6380099F9B5F84C30174C9BB2C01AB5F84A3096
:10B64800984221D294F840103046FEF78FF901282D
:10B658000AD1114B1A78012A19D100221A70236DC8
:10B6680020465B68984712E094F840103046FEF791
:10B678007DF904280BD194F8482094F840303046DE
:10B68800394600F095FB10B9032384F842300020B6
:10B69800F8BD00BF785F0020A20C0020384B93F85B
:10B6A800453073B50446042B66D8DFE803F003324F
:10B6B8000340530000F58873009309230193012286
:10B6C8004FF4045300F0B4FA002855D12D4B94F8E8
:10B6D800102194F813111A7094F811215A7094F8E3
:10B6E800122102EB01225A8094F8142194F81811BF
:10B6F8001A7194F815215A7194F816219A7194F8D0
:10B70800172102EB01221A811D4B012083F8450005
:10B7180035E000F5887300931A4B1B8901220193C9
:10B728004FF4085300F084FA30BB03220EE02123C3
:10B7380000220B750A234B75CA820A834A83134673
:10B7480000F06CF908B1032816D104220C4B83F8D9
:10B75800452011E0212300220B7501250B234B7591
:10B76800CD820A834A831346164600F057F928B952
:10B77800034B83F8456002E0012000E028467CBDC9
:10B78800785F0020CC5F002038B5114D95F8401047
:10B79800044649B1FEF756F895F840102046FFF7E1
:10B7A800FAFE002385F84030094D95F8411051B153
:10B7B8002046FEF747F895F841102046FFF7EBFEC4
:10B7C800002385F84130034B00221A7038BD00BFB2
:10B7D800785F0020A20C00202DE9F347344B0622A5
:10B7E80083F8422091F84420012A07460C4658D194
:10B7F80091F84520012A04BF2E4A1A65002283F8D1
:10B80800422083F8452091F8522083F84820B1F867
:10B818005420A3F8462091F85620092AA3F84A2074
:10B8280003D8234B0A22A3F84A2094F842A0204DBB
:10B83800BAF1020F28BF4FF0020A26464FF000085F
:10B848004FF0030927E096F852100B0608D5384642
:10B8580085F84410FFF786FE014685F8400009E0A8
:10B8680085F8431096F852103846FFF77BFE0146DC
:10B8780085F84100B5F8460094F82020019094F826
:10B888002130CDF800903846FFF71EFE08F1010878
:10B898005FFA88F80836D045D5D1074B00201870D4
:10B8A80004E0D1F880301B6C98470120BDE8FC8784
:10B8B800785F002034020020A20C002030B543EA53
:10B8C80002229DF80C40CA8221250023049A0D7596
:10B8D8000B83092523464D754C83BDE8304000F0A5
:10B8E8009DB800BF70474A4A00232DE9F0471370FE
:10B8F80053709370D37005461A46E9180133897856
:10B908000139C9B2022998BF0122062BF5D1012AB3
:10B918007CD03F4991F802C00A784B782846022625
:10B9280001F10A098778BFB18C1801322771D2B2A8
:10B93800002406E0013409EB040A1AF801ACBA4500
:10B9480003D05FFA84F8E045F4D3E04504D1CC187D
:10B95800877801332774DBB20136F6B20130082E3E
:10B96800E0D12B4C012B2270637041D1207CE07018
:10B97800FDF757FA2B78102B1BD022460AD8022B3A
:10B988001BD003D89BB1012B1DD112E0042B16D07C
:10B99800052B0AE0402B12D004D8142B11D0202BF1
:10B9A80011D10AE0412B0CD0502B0CD109E0A37522
:10B9B80009E0174B02229A7505E0012302E00323F0
:10B9C80000E004239375124A937DD178114A012B24
:10B9D80005D803EB4103D05CFDF718FA0AE0032011
:10B9E80000FB013102EB8102D2F8C030984701E038
:10B9F8000023E370064A137802F10A0193700023CA
:10BA08000432985C58540133062BFAD1BDE8F0870C
:10BA1800A30C002040970408FDF7F6B9C878012860
:10BA280010B504D002284FF0010319D108E00C78B2
:10BA38008B814C7008240C708A600877022308E018
:10BA48000A7F0D2A03D10020CB70087710BD0B2A7E
:10BA580001D1CB7010BD0C2A04D1CB70032010BDCE
:10BA6800184610BD184610BD00EB421310B500244F
:10BA780083F8B24300EB42130324C3F8BC13082134
:10BA8800C3F8C01383F8B8431146FDF780FFC0B26E
:10BA980010BD38B500EB4314002584F8B2535C019F
:10BAA8000519C5F8BC1300EB4311C1F8C02312B93E
:10BAB800012285F8C923041900EB431294F8C9132D
:10BAC800002914BF0221002182F8B8131946FDF796
:10BAD8005EFF002038BD38B500EB4314012584F81B
:10BAE800B2530225C4F8BC1384F8B853C4F8C02371
:10BAF8001946FDF74CFF002038BD38B500EB43155B
:10BB0800002485F8B24300EB4315C5F8C02395F827
:10BB1800C923C5F8BC13A24214BF0222224685F8E5
:10BB2800B8231946FDF733FF204638BD38B500EB7A
:10BB380043140125C4F8C02394F8C823C4F8BC13DF
:10BB4800002A14BF0222002284F8B25384F8B823D2
:10BB58001946FDF71CFF002038BDF8B504461F46FE
:10BB68000E46154602201A460E49FDF757F904EB12
:10BB78004713012283F8B22393F8C823C3F8BC63A0
:10BB8800002A14BF0221002182F0010283F8B813B1
:10BB9800C3F8C05383F8C82320463946FDF7F7FE9B
:10BBA8000020F8BD00A1050838B500EB43150024B6
:10BBB80085F8B24300EB4315C5F8C02395F8C823B0
:10BBC800C5F8BC13A24214BF0221214682F001022B
:10BBD80085F8B81385F8C8231946FDF7D8FE20461E
:10BBE80038BD38B500EB4314012584F8B253254617
:10BBF800C4F8BC13C4F8C023002485F8B843194618
:10BC0800FDF7C5FE204638BD38B500EB43150024C6
:10BC180085F8B24300EB4315C5F8BC13C5F8C0233B
:10BC280085F8B8431946FDF7B2FE204638BD00BF77
:10BC380010B562F07F020A750622BDF80C404A75FD
:10BC4800CB8240F2094203F47F43B3F5407F0CBF37
:10BC580013460023029A0B8323464C83BDE8104009
:10BC6800FFF7DCBE73B5BDF818601D4642F440739B
:10BC780000F588728DE8440000220446FFF7D8FFDB
:10BC8800B8B994F81131032B13D194F81031023B51
:10BC98009E42A8BF1E46B6B2034606E0E21802332B
:10BCA80092F8122105F8012B9BB2B342F6D3002378
:10BCB8002B707CBD73B500F5887316468DE8480077
:10BCC80000224FF4807304460D46FFF7B1FF0028A9
:10BCD80045D194F8103185F8223094F8113185F85F
:10BCE800233094F8132194F8123103EB0223AB8428
:10BCF80094F8143185F8263094F8153185F82730F2
:10BD080094F8163185F8283094F81731082E85F8FC
:10BD1800293024D994F8192194F8183103EB022317
:10BD28006B8594F81B2194F81A3103EB0223AB8539
:10BD380094F81D2194F81C3103EB0223EB8594F849
:10BD48001E3185F8303094F81F3185F8313094F879
:10BD5800203185F8323094F8213185F833307CBDB4
:10BD680010B500230524CA821A460B754C750B833F
:10BD78004B83BDE81040FFF751BE10B500230924DE
:10BD8800CA821A460B754C750B834B83BDE810406D
:10BD9800FFF744BE10B50A83012400220C75CB823C
:10BDA8000B2413464C754A83BDE81040FFF736BE96
:10BDB80030B54FEA431302240C75C31801244C759F
:10BDC800002412F0800F0A83CC824C8314BF83F8BE
:10BDD800C84383F8C943002225461346BDE83040CE
:10BDE800FFF71CBE2DE9F04F93461A7802705A7877
:10BDF80089B042709A780691D97802EB0122428084
:10BE08001A7902715979417199798171D979C17118
:10BE1800197A0172BDF84810092940F29480022A63
:10BE280000F293804B4A092192F800C0548881E0BF
:10BE38001A789B1889185A78042A89B27AD19E7878
:10BE480093F803A0069F09254FFA86F8BAF1020F66
:10BE580005FB08726ED81D781F7900955D790195EC
:10BE68009D790295DD7903951D7A022F049504D9F1
:10BE7800384B83F800C05C8067E04FEA48050595B9
:10BE8800CDF81C800025814650E018781B18091849
:10BE98005878052889B249D10798844511D0009867
:10BEA8009670107004205070019882F803A05071A9
:10BEB8000298177190710398D0710498B446107263
:10BEC80016E0187993F8058000EB0820844230DCEE
:10BED80000989670107004205070019882F803A0A2
:10BEE80050710298177190710398D071049810726C
:10BEF800059893F8008040FA85F40BEBC4000BF822
:10BF080034805C7844709C788470DC78C47093F8D2
:10BF180005801C7904EB082484809C7984715C7901
:10BF28001879013500EB0424A4B2EDB268B2B84226
:10BF3800ABDB484642888A423FF67AAF054B002081
:10BF48005880187002E0002000E0032009B0BDE826
:10BF5800F08F00BFBA0C0020F7B54FF4007300F55E
:10BF6800887701921546002206460C460097FFF78F
:10BF78005FFE034633B113E0F11891F8101199549C
:10BF8800013300E0074A99B2A942F5D304F134001D
:10BF980004F13E0104F150023B460095FFF722FFF1
:10BFA800FEBD00BFDE5F002003780A88D3180B802F
:10BFB8000378C018704700BF036823F001030360CB
:10BFC8000023036043608360C360036121234361EE
:10BFD8002C4B98421CD02C4B984220D02B4B98428B
:10BFE80025D02B4B98422AD02A4B98422FD02A4B47
:10BFF800984233D0294B984237D0294B984204D1E4
:10C008004FF03D5243F8AC2C7047264B984203D171
:10C018003D2243F8082C7047234B984204D14FF433
:10C02800746243F8202C7047204B984204D14FF497
:10C03800741243F8382C70471D4B984204D14FF0C6
:10C04800746243F8502C70471A4B984203D11A4A2D
:10C0580043F8642C7047194B984203D1184A43F8A7
:10C068007C2C7047174B984203D1174A43F8942CFD
:10C078007047164B984204BF4FF03D5243F8AC2C22
:10C08800704700BF106002402860024040600240D4
:10C09800586002407060024088600240A060024020
:10C0A800B8600240106402402864024040640240C4
:10C0B80058640240706402403D00002088640240D9
:10C0C800400F0020A064024000003D20B8640240F8
:10C0D8000268134B10B51340CC680A6822434C69B8
:10C0E80022438C692243CC6922430C6A22434C6A5E
:10C0F80022438C6A22434C6B22438C6B22431343AA
:10C10800036042690C6BCB6A22F007022343134396
:10C1180043610B6943604B6883608B68C36010BDE3
:10C128003F801CF00023036043608360C3600361A9
:10C1380043618361C361036243628362C3620363D1
:10C14800436383637047036811B143F0010301E05F
:10C1580023F0010303607047036811B143F40043FF
:10C1680001E023F4004303607047036811B143F012
:10C17800200301E023F0200303607047416070470B
:10C18800406880B27047036812B143F4002301E0AD
:10C1980023F40023036001617047036811B143F47D
:10C1A800802301E023F48023036070470AB1016112
:10C1B8007047C16070470068C0F3C04070470068AE
:10C1C80000F001007047406900F0380070470A4AE3
:10C1D8000A4B10B50A4CA04288BF13468A004CBFD0
:10C1E8005B681B6821F0F02121F0821119420CBF15
:10C1F8000020012010BD00BF006402400060024022
:10C208000F64024010B5084B084A094CA04288BF89
:10C21800134611F0005F21F0F02121F0821114BFC4
:10C22800D960996010BD00BF006002400064024000
:10C238000F6402400B0607D5436912B143F080032F
:10C2480001E023F080034361802909D001F01E0139
:10C25800036812B119430160704723EA01010160C4
:10C268007047124B124A10B5124CA0428CBF1446AC
:10C278001C4621F0F02323F0C3132BB1026802F00F
:10C288001E0202EAD12202E0426902F0800288001E
:10C298004CBF6368236821F0F02121F08210184018
:10C2A80002D0101C18BF012010BD00BF0060024062
:10C2B800006402400F64024010B5084B084A094C5C
:10C2C800A04288BF134611F0005F21F0F02121F051
:10C2D800821114BFD960996010BD00BF0060024090
:10C2E800006402400F640240044B00221A605A6046
:10C2F8009A60DA60024A5A61704700BF003C014008
:10C30800FFFF7F00837910B5002B29D01A4B0168F5
:10C318001C68CA4314401C605C6822405A60027959
:10C3280002F1804202F59E321468214311600268CE
:10C338009C68D1430C409C60DC682140D9604179FD
:10C34800102906D1996811439960D9680A43DA60BF
:10C3580010BD01F1804303F59E3319680A4308E0D4
:10C368000379016803F1804303F59E331A6822EAD2
:10C3780001021A6010BD00BF003C014000230C22DE
:10C3880003600371427183717047024B1A6902435B
:10C398001A617047003C0140034B5B6918420CBFAF
:10C3A80000200120704700BF003C0140014B58614C
:10C3B800704700BF003C0140054B1A685B690340A9
:10C3C80004D010420CBF0020012070471846704767
:10C3D800003C0140014B5861704700BF003C0140E0
:10C3E8004FF0204318B943F2DB021A6003E043F22E
:10C3F800D20243F820204FF02042411C6FF07043D6
:10C4080042F8213002F5827242F82030704770B548
:10C4180084684568C368C16A026825431D43036987
:10C428001D4343691D4383691D43C3691D43036A53
:10C438001D43436A1D43836A1D43036B0D431D431C
:10C448004FF02043082C43F8225005D153F82240DE
:10C4580044F0400443F82240436B9E691D6835430D
:10C468005E6845EA06159E6845EA0625DE6845EADF
:10C4780006451E695B6945EA0655541C45EA03658D
:10C488004FF02043B1F5804F43F8245010D1836B0F
:10C49800986919680143586841EA0011986841EAA7
:10C4A800002118695B6941EA005141EA036101E032
:10C4B8006FF07041014B43F8221070BD040100A0D9
:10C4C800022242604FF480524262416B4FF40052A4
:10C4D80010B5826200230F22FF2403608360C360CB
:10C4E800036143618361C3610362C36203630A60DA
:10C4F8004A608C60CA600A614A618B61816B0A601C
:10C508004A608C60CA600A614A618B6110BD4FF055
:10C51800204321B153F8202042F0010203E053F8F0
:10C528002010024A0A4043F820207047FEFF0F00FF
:10C5380010280CBF064B074B4FF040024FF0180174
:10C5480019605A604FF0FC329A60DA60704700BF99
:10C55800600000A0800000A030B5836844681C43D8
:10C56800C36844F008041C4303691C43436944EA54
:10C578004324836944EA4334C36999685A680904BF
:10C5880041EA02211A68DB68114341EA0361036A40
:10C598009A685D68120442EA05221D68DB682A432E
:10C5A80042EA03620368102B0CBF034B034B1C6069
:10C5B8009960DA6030BD00BF600000A0800000A074
:10C5C80010230360C269002343608360C360036172
:10C5D80043618361FC23136053609360D360026AF4
:10C5E800136053609360D360704741B110280CBF4B
:10C5F800074B084B1A6842F004021A60704710286B
:10C608000CBF034A034A044B11680B401360704780
:10C61800600000A0800000A0FBFF0F0041B11028BF
:10C628000CBF084B084B1A6842F040021A6070476A
:10C6380010280CBF034A044A044B11680B401360CE
:10C64800704700BF600000A0800000A0BFFF0F007F
:10C65800102802D1024B58697047024B586970473D
:10C66800600000A0800000A0054B18221A6000227C
:10C678005A604FF0FC329A60DA601A61704700BF66
:10C68800A00000A00268436842F0100242EA432278
:10C69800836842EA4332144B10B51A60C268916845
:10C6A8005468090441EA04211468D268214341EA24
:10C6B80002629A60026991685468090441EA042197
:10C6C8001468D268214341EA0262DA6042699168DB
:10C6D8005068090441EA00211068D268014341EA20
:10C6E80002621A6110BD00BFA00000A0C26800234A
:10C6F800036043608360FC23136053609360D360DE
:10C708000269136053609360D36042691360536099
:10C718009360D3607047054B18B11A6842F0040261
:10C7280002E01968024A0A401A607047A00000A097
:10C73800FBFF0F0062B1102801D10E4B03E0B0F5EA
:10C74800807F03D10C4B5A68114311E00B4BFAE779
:10C75800102804D1074B5A6822EA010108E0B0F515
:10C76800807F0CBF044B054B5A686FEA01011140EA
:10C7780059607047600000A0800000A0A00000A0E1
:10C78800102801D1064B04E0B0F5807F0CBF054BA3
:10C79800054B5B680B420CBF00200120704700BFAF
:10C7A800600000A0800000A0A00000A0102804D114
:10C7B800074B5A6822EA010108E0B0F5807F0CBFF8
:10C7C800044B054B5A686FEA0101114059607047E4
:10C7D800600000A0800000A0A00000A0102801D1E7
:10C7E800084B04E0B0F5807F0CBF074B074B5B6834
:10C7F80013EA010004D013EAD1010CBF0020012084
:10C80800704700BF600000A0800000A0A00000A04A
:10C81800102804D1084B5A6822EAD10109E0B0F582
:10C82800807F0CBF054B064B5A684FEAD10122EABC
:10C8380001015960704700BF600000A0800000A09F
:10C84800A00000A008B52C4B984205D10120014654
:10C8580000F048FC012048E0284B984205D102200E
:10C86800012100F03FFC02203FE0254B984205D112
:10C878000420012100F036FC042036E0214B9842C8
:10C8880005D10820012100F02DFC08202DE01E4BC9
:10C89800984205D11020012100F024FC102024E04A
:10C8A8001A4B984205D12020012100F01BFC2020C2
:10C8B8001BE0174B984205D14020012100F012FCE3
:10C8C800402012E0134B984205D18020012100F04E
:10C8D80009FC802009E0104B98420BD14FF480707E
:10C8E800012100F0FFFB4FF480700021BDE80840F3
:10C8F80000F0F8BB08BD00BF000002400004024081
:10C9080000080240000C02400010024000140240DF
:10C9180000180240001C0240002002402DE9F047A8
:10C928000023D1F800801A464FF0010C03270CFAB7
:10C9380002F404EA0805A5422ED1066817FA03F4A2
:10C94800E443264006600E79D0F8009006FA03FA10
:10C95800013E4AEA0909012EC0F8009014D88668F9
:10C9680091F8059026408660866809FA03F949EA35
:10C9780006068660466826EA050545608D7946689C
:10C988009540ADB235434560C5682C40C460CC794C
:10C99800C5689C402C43C46001320233102AC6D1BA
:10C9A800BDE8F0874FF6FF730360002303714371FE
:10C9B8008371C371704782B04FF480330193019B38
:10C9C8000B430193019BC361C161019BC361C369AF
:10C9D8000193C369019302B07047036919420CBF00
:10C9E800002001207047006980B2704743691942EE
:10C9F8000CBF002001207047406980B27047018356
:10CA08007047418370470AB101837047418370477B
:10CA18004161704743694B404361704701F0070328
:10CA2800C908083130B59B0050F821500F249C40AC
:10CA380025EA040440F8214050F8214012FA03F393
:10CA48001C4340F8214030BD08B5134B984207D12C
:10CA58004FF40010012100F069FB4FF4001014E0BE
:10CA68000E4B984207D14FF48000012100F05EFB85
:10CA78004FF4800009E00A4B98420BD14FF40000B4
:10CA8800012100F053FB4FF400000021BDE80840ED
:10CA980000F04CBB08BD00BF0054004000580040E7
:10CAA800005C00407FB50446868868460D4600F065
:10CAB8006DFA02992C482B6826F03F063604B1FB24
:10CAC800F0F0360C80B20643A680228822F00102DC
:10CAD8001204120C2280254A93420AD85B00B1FB4B
:10CAE800F3F301309BB280B22084032B98BF042358
:10CAF80021E0EE884BF6FF72964205D1032253439C
:10CB0800B1FBF3F39BB206E019225343B1FBF3F3F5
:10CB18009BB243F480431A054FF4967208BF43F062
:10CB2800010350434FF47A7290FBF2F0013080B267
:10CB380043F400432084A38323886989AA889BB28D
:10CB480043F001032380238823F4816323F0020345
:10CB58001B040A431B0C13439BB223802A89AB890D
:10CB680013439BB223817FBD40420F00A086010082
:10CB780041F288330360002383804BF6FF72038100
:10CB880043814FF48043C28083817047038819B181
:10CB98009BB243F0010303E023F001031B041B0CC9
:10CBA80003807047038819B19BB243F4807303E094
:10CBB80023F480731B041B0C03807047038819B18E
:10CBC8009BB243F4007303E023F400731B041B0CB3
:10CBD8000380704712B141F0010101E001F0FE014C
:10CBE80001827047038819B19BB243F4806303E064
:10CBF80023F480631B041B0C0380704783899BB25A
:10CC080001F0FE0123F0FE030B4383817047838903
:10CC180019B19BB243F0010303E023F001031B04A5
:10CC28001B0C83817047038819B19BB243F0400302
:10CC380003E023F040031B041B0C038070470388A8
:10CC480029B16FEA43436FEA53439BB201E05B04A7
:10CC58005B0C03807047038819B99BB243F08003CB
:10CC680003E023F080031B041B0C03807047B1F51D
:10CC7800804F838B04D023F480431B041B0C02E0F9
:10CC88009BB243F4804383837047B1F5006F0388F8
:10CC980003D19BB243F4006303E023F400631B0455
:10CCA8001B0C03807047B1F5005F038803D19BB26A
:10CCB80043F4005303E023F400531B041B0C0380CC
:10CCC8007047038819B19BB243F0100303E023F0C7
:10CCD80010031B041B0C0380704701827047008AF5
:10CCE800C0B27047038819B19BB243F4805303E084
:10CCF80023F480531B041B0C03807047B1F5006FAD
:10CD0800038803D19BB243F4006303E023F4006378
:10CD18001B041B0C03807047038819B19BB243F0B6
:10CD2800200303E023F020031B041B0C038070473F
:10CD3800008BC0F307207047838819B19BB243F476
:10CD4800006303E023F400631B041B0C838070471B
:10CD5800838819B19BB243F4805303E023F48053D2
:10CD68001B041B0C8380704782B000230193019041
:10CD7800019BCB180193019B188880B202B07047C1
:10CD880083889BB20AB1194301E023EA010181803B
:10CD98007047838A008B9BB243EA0040084020F02A
:10CDA8007F40431A584240EB03007047838A008B48
:10CDB8009BB243EA004020F07F40704782B00023D6
:10CDC800009301930B0F01900093009B21F07F418A
:10CDD80013B1019B143302E0019B090C1833019332
:10CDE800019B1B6819420CBF0020012002B070474C
:10CDF800C94389B2818270478388808A80B208409B
:10CE08009BB206D001F0E06113EA11410CBF00208B
:10CE180001207047C94389B2818270470A4B1A685A
:10CE280042F001021A6000229A60196821F08471A8
:10CE380021F48031196005495960196821F480216D
:10CE48001960DA60704700BF0038024010300024D3
:10CE5800024B00221A701870704700BF0238024057
:10CE6800034B1A6822F0F80242EAC0021A607047BF
:10CE780000380240014B1860704700BF000047426D
:10CE8800064B002201281A701A7002D0042804D117
:10CE980001E01870704705221A7070477038024018
:10CEA800014B1860704700BF800E4742014341EABA
:10CEB800821200995B08013B42EA016141EA0341A1
:10CEC800014B5960704700BF00380240014B1860A1
:10CED800704700BF600047428001034B40EA017180
:10CEE800C3F88410704700BF00380240014B186037
:10CEF800704700BF68004742014B1860704700BF89
:10CF08004C004742034B9A6822F0EC6202430A4302
:10CF18009A60704700380240034B9A6822F07842C2
:10CF280002430A439A60704700380240034B9A68EC
:10CF380022F0030202439A60704700BF00380240A3
:10CF4800024B986800F00C00704700BF00380240A0
:10CF5800034B9A6822F0F00202439A60704700BFC0
:10CF680000380240034B9A6822F4E05202439A6068
:10CF7800704700BF00380240034B9A6822F46042B1
:10CF880042EAC0029A607047003802401E4B9A6815
:10CF980002F00C02042A10B503D0082A03D01B4B58
:10CFA80018E01B4B16E059685A6811F4800F59684D
:10CFB80014BF174B154B02F03F02B3FBF2F3124AB2
:10CFC8005268C2F30142C1F3881101324B43520047
:10CFD800B3FBF2F30C4903608B680E4A0468C3F391
:10CFE8000313D35C34FA03F343608C68C4F38224DC
:10CFF800145D33FA04F484608968C1F34231525CE9
:10D00800D340C36010BD00BF003802400024F400C4
:10D0180000127A003C02002000F44073B3F5407F10
:10D02800084B08D1996820F0704221F4F81122F4D5
:10D0380040720A439A601A6F000542EA1050186756
:10D04800704700BF00380240014B1860704700BFAE
:10D058003C0E4742014B1860704700BF400E4742E4
:10D06800014B1860704700BF5C014742044B1A6BC4
:10D0780009B1104301E022EA00001863704700BFBD
:10D0880000380240044B5A6B09B1104301E022EA10
:10D0980000005863704700BF00380240044B9A6B89
:10D0A80009B1104301E022EA00009863704700BF0D
:10D0B80000380240044B1A6C09B1104301E022EA1F
:10D0C80000001864704700BF00380240044B5A6CD7
:10D0D80009B1104301E022EA00005864704700BF1C
:10D0E80000380240044B1A6909B1104301E022EAF2
:10D0F80000001861704700BF00380240044B5A69AD
:10D1080009B1104301E022EA00005861704700BFEE
:10D1180000380240044B9A6909B1104301E022EA41
:10D1280000009861704700BF00380240044B1A6A3B
:10D1380009B1104301E022EA00001862704700BFFD
:10D1480000380240044B5A6A09B1104301E022EA50
:10D1580000005862704700BF00380240044B1A6D47
:10D1680009B1104301E022EA00001865704700BFCA
:10D1780000380240044B5A6D09B1104301E022EA1D
:10D1880000005865704700BF00380240044B9A6D94
:10D1980009B1104301E022EA00009865704700BF1A
:10D1A80000380240044B1A6E09B1104301E022EA2C
:10D1B80000001866704700BF00380240044B5A6EE2
:10D1C80009B1104301E022EA00005866704700BF29
:10D1D80000380240044B1A7809B1104301E022EAF2
:10D1E80000001870704700BF0D3802404309012B3A
:10D1F800074A01D1136803E0022B0CBF136F536F6A
:10D2080000F01F0033FA00F000F00100704700BF83
:10D218000038024007B5002301933120FFF7E6FFED
:10D22800019B01330193019BB3F5A06F01D0002846
:10D23800F3D03120FFF7DAFF003018BF01200EBD10
:10D24800024B5A6F42F080725A67704700380240AA
:10D25800034BDB6818420CBF00200120704700BF59
:10D2680000380240014B1870704700BF0E3802406A
:10D2780008B5154B98420BD101214FF48050FFF7A8
:10D2880061FF4FF480500021BDE80840FFF75ABF06
:10D298000E4B984207D14FF480400121FFF746FF1B
:10D2A8004FF4804009E00A4B98420BD14FF40040FC
:10D2B8000121FFF73BFF4FF400400021BDE8084083
:10D2C800FFF734BF08BD00BF003001400038004000
:10D2D800003C00400B88028810B54C8823438C889A
:10D2E8002343CC8823430C8923434C8923438C89CB
:10D2F8002343CC8902F44152234313439BB2038056
:10D30800838B23F400631B041B0C83830B8A038227
:10D3180010BD838B23F47B6323F00F031B041B0CCA
:10D328008383022303848B68F0B5858B022BADB20F
:10D3380038D0294A8E889468002E14BF0226012608
:10D34800240203D5946824F400049460D2F884403D
:10D35800D2F884705268DFF884C002F03F02BCFB48
:10D36800F2F2C4F388145443C7F30272B4FBF2F424
:10D37800CA88B2F5007F4FF00A0201D1240A02E000
:10D388007601B4FBF6F46243B2FBF3F305330A22E9
:10D398009BB2B3FBF2F303F001021202C3F34F0393
:10D3A80092B200E000229C1EA4B2FE2C28BF0022EC
:10D3B800CC8828BF0223134323439BB203840B88E2
:10D3C8004A882B4343F4006313438A8813438A89AA
:10D3D80013439BB28383F0BD0038024000127A00E9
:10D3E8000023038043808380C3800381438183813A
:10D3F800C3810723038270470023022203804380EE
:10D408008380C380826083817047038819B19BB28F
:10D4180043F0400303E023F040031B041B0C03808C
:10D428007047838B19B19BB243F4806303E023F404
:10D4380080631B041B0C83837047038823F40063F9
:10D448001B041B0C038003889BB20B4303807047AB
:10D45800B1F5804F038803D19BB243F4804303E0C6
:10D4680023F480431B041B0C038070474FF6FF63B3
:10D478009942038803D09BB243F4807303E023F4FA
:10D4880080731B041B0C03807047838819B19BB2FF
:10D4980043F0040303E023F004031B041B0C838004
:10D4A8007047838819B19BB243F0100303E023F05F
:10D4B80010031B041B0C83807047838B23F47B634E
:10D4C80023F00F031B041B0C8383022303840B88A4
:10D4D800828BB3F5007F10B592B205D0002B0CBF3C
:10D4E8004FF48073002301E04FF480734C8822438B
:10D4F8008C88898942F4006222430A4392B213431A
:10D50800838310BD808980B270478181704703880A
:10D5180019B19BB243F4005303E023F400531B04F6
:10D528001B0C0380704703889BB243F4805303802D
:10D538007047012902D0008B80B27047808A80B280
:10D548007047008A80B2704783889BB20AB119433A
:10D5580001E023EA010181807047090901238B401A
:10D568009BB21AB1828892B2134303E0828892B2C6
:10D5780022EA030383807047038919420CBF002005
:10D5880001207047C94389B20181704710B584886A
:10D598000089012301F00F0280B213FA02F2104051
:10D5A800A4B205D009098B401C420CBF0020012001
:10D5B80010BD01F00F0101238B40DB439BB20381B7
:10D5C800704700BF08B501214FF48040FFF7BAFD4E
:10D5D8004FF480400021BDE80840FFF7B3BD014B80
:10D5E800186070470038014001F0030289080A4BAF
:10D5F800023130B5920053F821500F24944025EAA7
:10D60800040443F8214053F8214010FA02F214436D
:10D6180043F8214030BD00BF00380140014B18607D
:10D62800704700BFDC002742014B1860704700BFFD
:10D6380000042742024B186AC0F30020704700BF5D
:10D648000038014030B5048C24F001042404240C73
:10D658000484058B048CADB2A4B225F0F305154300
:10D6680024F00A0445EA031544F00104ADB20C4362
:10D678000583048430BD30B5048C24F010042404E0
:10D68800240C0484048B058C24F44074ADB2240566
:10D69800240D25F0A00544EA022445F0100544EACB
:10D6A800033445EA0115A4B2ADB20483058430BD44
:10D6B80008B5474B984205D101200146FFF742FDC6
:10D6C80001203DE0B0F1804F05D101200146FFF770
:10D6D8002DFD012076E03F4B984205D10220012123
:10D6E800FFF724FD02206DE03B4B984205D1042052
:10D6F8000121FFF71BFD042064E0384B984205D157
:10D7080008200121FFF712FD08205BE0344B984206
:10D7180005D110200121FFF709FD102052E0314BFF
:10D72800984205D120200121FFF700FD202049E083
:10D738002D4B984209D102200121FFF703FD022059
:10D748000021BDE80840FFF7FDBC284B984207D1EF
:10D758004FF480300121FFF7F5FC4FF48030EFE7FC
:10D76800234B984207D14FF400300121FFF7EAFC20
:10D778004FF40030E4E71F4B984207D14FF4802064
:10D788000121FFF7DFFC4FF48020D9E71A4B9842BC
:10D7980005D140200121FFF7C9FC402012E0174BBA
:10D7A800984205D180200121FFF7C0FC802009E0C4
:10D7B800134B98420BD14FF480700121FFF7B6FC50
:10D7C8004FF480700021BDE80840FFF7AFBC08BDEA
:10D7D800000001400004004000080040000C004028
:10D7E80000100040001400400004014000400140C7
:10D7F800004401400048014000180040001C00405F
:10D80800002000401C4A038890429BB212D002F5C7
:10D81800806290420ED0B0F1804F0BD0A2F58032DA
:10D82800904207D002F58062904203D002F58062F0
:10D83800904203D14A8823F0700313430F4A904261
:10D8480008D002F58062904204D023F440730A891C
:10D858009BB2134303804B68C3620B880385064B56
:10D86800984203D003F58063984201D18B7A0386EE
:10D8780001238382704700BF000001400010004070
:10D888004FF0FF334360002303800381438083729A
:10D898007047018582827047038823F070031B0458
:10D8A8001B0C0B430380704741627047C16270478D
:10D8B800406A7047008D80B27047038819B19BB2E7
:10D8C80043F0020303E023F002031B041B0C038054
:10D8D8007047038819B19BB243F0040303E023F0B7
:10D8E80004031B041B0C03807047038819B19BB207
:10D8F80043F0800303E023F080031B041B0C038028
:10D908007047038823F008031B041B0C038003885B
:10D918009BB20B4303807047038823F440731B04B6
:10D928001B0C038003889BB20B430380704703885A
:10D9380019B19BB243F0010303E023F001031B0478
:10D948001B0C03807047038C23F001031B041B0C82
:10D95800038470B5038C8488028B0D884E8822F06E
:10D9680073021204120C2A438D8923F002031B044C
:10D9780035431B0CADB22B430E4DA842A4B203D0C5
:10D9880005F58065A8420ED1CD894E8A23F008039B
:10D998002B438D8823F004032B430D8A354324F44D
:10D9A8004074ADB22C43848002838A684263038446
:10D9B80070BD00BF00000140038C23F010031B045E
:10D9C8001B0C0384038C828830B5048B0D8824F4E7
:10D9D800E6442404240C23F0200344EA05241B0411
:10D9E8008D891B0C43EA05134D8843EA0513134D33
:10D9F800A84292B2A4B29BB203D005F58065A842B2
:10DA080015D1CD8923F080039BB243EA05134FF665
:10DA1800BF751D408B8845EA03130D8A22F44062C6
:10DA280042EA85024D8A42EA85029BB292B282801E
:10DA38008A6804838263038430BD00BF000001400C
:10DA4800038C23F480731B041B0C0384038C8288CF
:10DA580030B5848B0D8824F073042404240C23F43B
:10DA680000731B042C438D891B0C43EA05234D8846
:10DA780043EA0523124DA84292B29BB203D005F5A2
:10DA88008065A84215D1CD8923F400639BB243EA8F
:10DA980005234FF6FF351D408B8845EA03230D8A81
:10DAA80022F4405242EA05124D8A42EA05129BB21C
:10DAB80092B282808A688483C263038430BD00BFC7
:10DAC80000000140038C23F480531B041B0C0384C7
:10DAD800038C30B58488828B0D8822F4E6421204C8
:10DAE800120C23F4005342EA05221B048D891B0CF7
:10DAF80043EA05334D8843EA05330B4DA842A4B2E7
:10DB080092B29BB203D005F58065A84205D10D8A73
:10DB180024F4804444EA8514A4B2848082838A6809
:10DB28000264038430BD00BF00000140002303806D
:10DB38004380838083608381C381038243827047EB
:10DB480030B5058C0124ADB28C4025EA040400F1FF
:10DB58001803048409B1082907D149084FF68F70C2
:10DB6800CC582040C850C8580AE00439C1F34E01C7
:10DB780048F6FF70CC582040C8501202C85892B2DC
:10DB88000243CA5030BD4163704781637047C16327
:10DB9800704701647047038B23F070031B041B0C50
:10DBA8000B4303837047038B23F4E0431B041B0CD4
:10DBB80043EA01239BB203837047838B23F07003EE
:10DBC8001B041B0C0B4383837047838B23F4E043B4
:10DBD8001B041B0C43EA01239BB283837047038B0E
:10DBE80023F008031B041B0C0B4303837047038BB0
:10DBF80023F400631B041B0C43EA01239BB2038339
:10DC08007047838B23F008031B041B0C0B4383838F
:10DC18007047838B23F400631B041B0C43EA012326
:10DC28009BB283837047038B23F004031B041B0CF4
:10DC38000B4303837047038B23F480631B041B0C83
:10DC480043EA01239BB203837047838B23F00403C9
:10DC58001B041B0C0B4383837047838B23F4806363
:10DC68001B041B0C43EA01239BB283837047038B7D
:10DC780023F080031B041B0C0B4303837047038BA7
:10DC880009025B0441EA53439BB203837047838BC9
:10DC980023F080031B041B0C0B4383837047838B87
:10DCA80009025B0441EA53439BB283837047038CA8
:10DCB80023F002031B041B0C0B4303847047038CE3
:10DCC80023F008031B041B0C0B4303847047038CCD
:10DCD80023F020031B041B0C43EA01139BB20384AB
:10DCE8007047038C23F080031B041B0C43EA0113C9
:10DCF8009BB203847047038C23F400731B041B0C32
:10DD080043EA01239BB203847047038C23F4006326
:10DD18001B041B0C43EA01239BB203847047038C4A
:10DD280023F400531B041B0C43EA01339BB2038406
:10DD3800704710B5048C01238B40A4B224EA030376
:10DD48000384038C12FA01F10B439BB2038410BDC8
:10DD580010B5048C04238B40A4B224EA0303038483
:10DD6800038C12FA01F10B439BB2038410BD00230C
:10DD78000122038043808280C38003817047406B07
:10DD88007047806B7047C06B7047006C7047038B9F
:10DD980023F00C031B041B0C0383038B9BB20B4364
:10DDA80003837047038B23F440631B041B0C03831A
:10DDB800038B9BB243EA01239BB203837047F8B5F8
:10DDC8000C464988A288B4F800E023890546002952
:10DDD8000CBF02270027012A14BF01260226BEF124
:10DDE800000F10D1FFF72EFC2846E188FFF7CFFF80
:10DDF8002846394632462389FFF73DFCE188284604
:10DE0800BDE8F840CEE7FFF736FC2846E188FFF783
:10DE1800C9FF2846394632462389FFF713FCE188B3
:10DE28002846BDE8F840B2E7838B23F00C031B04B7
:10DE38001B0C8383838B9BB20B4383837047838B39
:10DE480023F440631B041B0C8383838B9BB243EA3C
:10DE580001239BB283837047F8B50D460B88AA88C7
:10DE6800498804463BB92B89FFF7ECFBE988204633
:10DE7800BDE8F8408BE7042B07D12B89FFF7FBFBA4
:10DE8800E9882046BDE8F8408CE7082BB5F808C0BB
:10DE9800078C1DD127F480773F043F0C0784868BBD
:10DEA800038CB6B29BB226F0F30623F4206346EA4D
:10DEB8000C1C43EA01211FFA8CFC89B24CEA0202CD
:10DEC80041F4807182830184E988BDE8F840ABE7BA
:10DED80027F480573F043F0C0784868B038C26F475
:10DEE800407623F4005336055B04360D5B0C46EA96
:10DEF800022243EA013342EA0C329BB2E98892B229
:10DF080043F4805382830384BDE8F84097E74A8846
:10DF18000B8813438A881343CA8813430A89134317
:10DF28004A8913438A8913439BB2A0F84430704747
:10DF38000023038043808380C380038143818381DE
:10DF48007047B0F8443029B16FEA43436FEA53434E
:10DF58009BB201E05B045B0CA0F8443070478388F7
:10DF680019B19BB243F0040303E023F004031B043C
:10DF78001B0C83807047838819B19BB243F001035F
:10DF880003E023F001031B041B0C83807047838983
:10DF98009BB20AB1194301E023EA0101818170476C
:10DFA80081827047038A19420CBF00200120704704
:10DFB800C94389B201827047038A828911EA030042
:10DFC80092B203D011420CBF002001207047C94310
:10DFD80089B2018270470A43A0F8482070478389B4
:10DFE8009BB20AB1194301E023EA0101818170471C
:10DFF800838819B19BB243F0080303E023F00803B8
:10E008001B041B0C83807047038923F007031B0440
:10E018001B0C03817047038923F070031B041B0C3E
:10E028000B43038103899BB243F0070303817047C5
:10E0380038B50D4611460122602D044602D1FFF77E
:10E048001AFB01E0FFF7FEFA238923F070031B0493
:10E058001B0C1D43258123899BB243F007032381B1
:10E0680038BD038923F070031B041B0C0B43038189
:10E078007047838823F070031B041B0C83808388FC
:10E088009BB20B4383807047038923F007031B046B
:10E098001B0C038103899BB20B43038170470389DF
:10E0A80023F080031B041B0C038103899BB20B43E1
:10E0B8000381704710B50489E4B20C43144344EA61
:10E0C8000324A4B2048110BD10B50446FFF7F2FF83
:10E0D80023899BB243F48043238110BD10B50446C5
:10E0E800FFF7E8FF238923F077031B041B0C43F099
:10E0F8007703238110BD70B50489068B058C26F43F
:10E108004076ADB226F0030624F00704360425F065
:10E1180022052404360C1543240C46F4807645EA7F
:10E128000315214346F00106ADB20181068305843B
:10E1380070BD838819B19BB243F0800303E023F0DC
:10E1480080031B041B0C83807047A0F85010704795
:10E1580008B5234B984205D110200121FEF7F2FFA4
:10E16800102037E01F4B984207D14FF400300121AF
:10E17800FEF7DCFF4FF4003009E01B4B98420BD14F
:10E188004FF480200121FEF7D1FF4FF480200021B9
:10E19800BDE80840FEF7CABF144B984207D14FF4B8
:10E1A80000200121FEF7C2FF4FF40020EFE7104BDB
:10E1B800984207D14FF480100121FEF7B7FF4FF4C2
:10E1C8008010E4E70B4B984209D120200121FEF78B
:10E1D800B9FF20200021BDE80840FEF7B3BF08BD05
:10E1E800001001400044004000480040004C00403E
:10E1F8000050004000140140038ACA889BB223F4EF
:10E20800405330B513430D46038283890989AA8890
:10E2180023F4B0530A43698923F00C031B040A430F
:10E228001B0C92B213438381838AAA899BB223F47D
:10E238004073134385B0838204466846FEF7A6FE02
:10E248001A4B9C4203D003F580639C4201D1039B87
:10E2580000E0029BA28912B2002A4FF019012A6835
:10E2680001FB03F101DA520000E092006423B1FBE4
:10E27800F2F1B1FBF3F21201100903FB1011A089AE
:10E2880000B2002806DAC9003231B1FBF3F303F01B
:10E29800070305E009013231B1FBF3F303F00F0383
:10E2A8001A4392B2228105B030BD00BF0010014070
:10E2B8004FF4165303600C2200238380C38003812C
:10E2C8004281838170470B88028A10B54C882343AA
:10E2D8008C88C988234392B20B4322F470629BB2A4
:10E2E8001343038210BD0023038043808380C380CF
:10E2F8007047838919B19BB243F4005303E023F4B8
:10E3080000531B041B0C83817047038B03F47F436A
:10E318000383038B9BB20B4303837047838929B123
:10E328006FEA43436FEA53439BB201E05B045B0C23
:10E3380083817047838A19B19BB243F4006303E079
:10E3480023F400631B041B0C83827047C905C90DA5
:10E35800818070478088C005C00D7047038A23F00C
:10E368000F031B041B0C0382038A9BB20B4303821B
:10E378007047838919B19BB243F0020303E023F08D
:10E3880002031B041B0C83817047838923F40063F9
:10E398001B041B0C838183899BB20B4383817047C9
:10E3A800038A23F020031B041B0C0382038A9BB2FD
:10E3B8000B4303827047038A19B19BB243F480432D
:10E3C80003E023F480431B041B0C038270478389FA
:10E3D8009BB243F0010383817047838A19B19BB2D2
:10E3E80043F0080303E023F008031B041B0C83829B
:10E3F8007047038BDBB20383038B9BB243EA012391
:10E4080003837047838A19B19BB243F0200303E06A
:10E4180023F020031B041B0C83827047838A19B1E5
:10E428009BB243F0100303E023F010031B041B0C02
:10E4380083827047838A23F004031B041B0C8382A6
:10E44800838A9BB20B4383827047838A19B19BB23C
:10E4580043F0020303E023F002031B041B0C838236
:10E468007047838A9BB20AB1194301E023EA01018C
:10E4780081827047C1F3421310B501F01F010124D6
:10E4880014FA01F1A34201D10C3004E0022B01D1AE
:10E49800103000E0143003680AB1194301E023EAA0
:10E4A8000101016010BD038819420CBF0020012042
:10E4B8007047C94389B201807047012210B501F045
:10E4C8001F03C1F342149A40012C01D1838903E050
:10E4D800022C0CBF038A838A9BB21340028892B233
:10E4E80043B1090A012313FA01F111420CBF0020BC
:10E4F800012010BD184610BD090A01238B40DB43DB
:10E508009BB20380704700BF81F0004102E000BF6A
:10E5180083F0004330B54FEA41044FEA430594EADB
:10E52800050F08BF90EA020F1FBF54EA000C55EA16
:10E53800020C7FEA645C7FEA655C00F0E2804FEAE7
:10E548005454D4EB5555B8BF6D420CDD2C4480EAC9
:10E55800020281EA030382EA000083EA010180EAF9
:10E56800020281EA0303362D88BF30BD11F0004F47
:10E578004FEA01314FF4801C4CEA113102D040427D
:10E5880061EB410113F0004F4FEA03334CEA1333B8
:10E5980002D0524263EB430394EA050F00F0A780D0
:10E5A800A4F10104D5F1200E0DDB02FA0EFC22FACB
:10E5B80005F2801841F1000103FA0EF2801843FABF
:10E5C80005F359410EE0A5F120050EF1200E012AB0
:10E5D80003FA0EFC28BF4CF0020C43FA05F3C018EE
:10E5E80051EBE37101F0004507D54FF0000EDCF167
:10E5F800000C7EEB00006EEB0101B1F5801F1BD310
:10E60800B1F5001F0CD349085FEA30004FEA3C0C13
:10E6180004F101044FEA445212F5800F80F09A8009
:10E62800BCF1004F08BF5FEA500C50F1000041EB0D
:10E63800045141EA050130BD5FEA4C0C404141EB11
:10E64800010111F4801FA4F10104E9D191F0000F38
:10E6580004BF01460020B1FA81F308BF2033A3F1BB
:10E668000B03B3F120020CDA0C3208DD02F1140CB2
:10E67800C2F10C0201FA0CF021FA02F10CE002F1ED
:10E688001402D8BFC2F1200C01FA02F120FA0CFCE6
:10E69800DCBF41EA0C019040E41AA2BF01EB04512F
:10E6A800294330BD6FEA04041F3C1CDA0C340EDC2D
:10E6B80004F11404C4F1200220FA04F001FA02F370
:10E6C80040EA030021FA04F345EA030130BDC4F12E
:10E6D8000C04C4F1200220FA02F001FA04F340EA23
:10E6E8000300294630BD21FA04F0294630BD94F0D4
:10E6F800000F83F4801306BF81F480110134013DBB
:10E708004EE77FEA645C18BF7FEA655C29D094EA2B
:10E71800050F08BF90EA020F05D054EA000C04BFA9
:10E728001946104630BD91EA030F1EBF0021002094
:10E7380030BD5FEA545C05D14000494128BF41F033
:10E74800004130BD14F580043CBF01F5801130BD97
:10E7580001F0004545F0FE4141F470014FF0000022
:10E7680030BD7FEA645C1ABF194610467FEA655CD3
:10E778001CBF0B46024650EA013406BF52EA033575
:10E7880091EA030F41F4002130BD00BF90F0000F63
:10E7980004BF0021704730B54FF4806404F132049F
:10E7A8004FF000054FF0000150E700BF90F0000F58
:10E7B80004BF0021704730B54FF4806404F132047F
:10E7C80010F0004548BF40424FF000013EE700BF4F
:10E7D80042004FEAE2014FEA31014FEA02701FBFDF
:10E7E80012F07F4393F07F4F81F06051704792F0B1
:10E7F800000F14BF93F07F4F704730B54FF460742B
:10E8080001F0004521F0004120E700BF50EA010275
:10E8180008BF704730B54FF000050AE050EA010222
:10E8280008BF704730B511F0004502D5404261EB92
:10E8380041014FF4806404F132045FEA915C3FF4D3
:10E84800DCAE4FF003025FEADC0C18BF03325FEA6C
:10E85800DC0C18BF033202EBDC02C2F1200300FA21
:10E8680003FC20FA02F001FA03FE40EA0E0021FA46
:10E8780002F11444C1E600BF70B54FF0FF0C4CF430
:10E88800E06C1CEA11541DBF1CEA135594EA0C0FE6
:10E8980095EA0C0F00F0DEF82C4481EA030621EA21
:10E8A8004C5123EA4C5350EA013518BF52EA03355C
:10E8B80041F4801143F4801338D0A0FB02CE4FF00E
:10E8C8000005E1FB02E506F00042E0FB03E54FF03E
:10E8D8000006E1FB03569CF0000F18BF4EF0010E36
:10E8E800A4F1FF04B6F5007F64F5407404D25FEA32
:10E8F8004E0E6D4146EB060642EAC62141EA5551E5
:10E908004FEAC52040EA5E504FEACE2EB4F1FD0C26
:10E9180088BFBCF5E06F1ED8BEF1004F08BF5FEAA4
:10E92800500E50F1000041EB045170BD06F0004656
:10E9380046EA010140EA020081EA0301B4EB5C0403
:10E94800C2BFD4EB0C0541EA045170BD41F48011FB
:10E958004FF0000E013C00F3AB8014F1360FDEBF20
:10E96800002001F0004170BDC4F10004203C35DAFC
:10E978000C341BDC04F11404C4F1200500FA05F37F
:10E9880020FA04F001FA05F240EA020001F0004220
:10E9980021F0004110EBD37021FA04F642EB060196
:10E9A8005EEA430E08BF20EAD37070BDC4F10C04C0
:10E9B800C4F1200500FA04F320FA05F001FA04F284
:10E9C80040EA020001F0004110EBD37041F1000170
:10E9D8005EEA430E08BF20EAD37070BDC4F120057B
:10E9E80000FA05F24EEA020E20FA04F301FA05F2E3
:10E9F80043EA020321FA04F001F0004121FA04F28B
:10EA080020EA020000EBD3705EEA430E08BF20EA5A
:10EA1800D37070BD94F0000F0FD101F00046400094
:10EA280041EB010111F4801F08BF013CF7D041EA16
:10EA3800060195F0000F18BF704703F0004652001A
:10EA480043EB030313F4801F08BF013DF7D043EAEB
:10EA58000603704794EA0C0F0CEA135518BF95EAA1
:10EA68000C0F0CD050EA410618BF52EA4306D1D128
:10EA780081EA030101F000414FF0000070BD50EA47
:10EA8800410606BF1046194652EA430619D094EAD1
:10EA98000C0F02D150EA013613D195EA0C0F05D1BB
:10EAA80052EA03361CBF104619460AD181EA03010F
:10EAB80001F0004141F0FE4141F470014FF00000C7
:10EAC80070BD41F0FE4141F4780170BD70B54FF062
:10EAD800FF0C4CF4E06C1CEA11541DBF1CEA1355E2
:10EAE80094EA0C0F95EA0C0F00F0A7F8A4EB0504C4
:10EAF80081EA030E52EA03354FEA013100F08880BB
:10EB08004FEA03334FF0805545EA131343EA126383
:10EB18004FEA022245EA111545EA10654FEA002638
:10EB28000EF000419D4208BF964244F1FD0404F5F1
:10EB3800407402D25B084FEA3202B61A65EB03054D
:10EB48005B084FEA32024FF480104FF4002CB6EB0A
:10EB5800020E75EB030E22BFB61A754640EA0C008A
:10EB68005B084FEA3202B6EB020E75EB030E22BFCA
:10EB7800B61A754640EA5C005B084FEA3202B6EB0B
:10EB8800020E75EB030E22BFB61A754640EA9C00CA
:10EB98005B084FEA3202B6EB020E75EB030E22BF9A
:10EBA800B61A754640EADC0055EA060E18D04FEA58
:10EBB800051545EA16754FEA06164FEAC30343EAF8
:10EBC80052734FEAC2025FEA1C1CC0D111F4801FC5
:10EBD8000BD141EA00014FF000004FF0004CB6E7BE
:10EBE80011F4801F04BF01430020B4F1FD0C88BF5D
:10EBF800BCF5E06F3FF6AFAEB5EB030C04BFB6EB68
:10EC0800020C5FEA500C50F1000041EB045170BD5A
:10EC18000EF0004E4EEA113114EB5C04C2BFD4EB87
:10EC28000C0541EA045170BD41F480114FF0000E0B
:10EC3800013C90E645EA060E8DE60CEA135594EA87
:10EC48000C0F08BF95EA0C0F3FF43BAF94EA0C0F8A
:10EC58000AD150EA01347FF434AF95EA0C0F7FF4FF
:10EC680025AF104619462CE795EA0C0F06D152EA53
:10EC780003353FF4FDAE1046194622E750EA410637
:10EC880018BF52EA43067FF4C5AE50EA41047FF448
:10EC98000DAF52EA43057FF4EBAE12E74FF0FF3CAD
:10ECA80006E000BF4FF0010C02E000BF4FF0010C7E
:10ECB8004DF804CD4FEA410C7FEA6C5C4FEA430CF7
:10ECC80018BF7FEA6C5C1BD001B050EA410C0CBF46
:10ECD80052EA430C91EA030F02BF90EA020F0020A8
:10ECE800704710F1000F91EA030F58BF994208BF0F
:10ECF80090422CBFD8176FEAE37040F001007047CC
:10ED08004FEA410C7FEA6C5C02D150EA013C07D122
:10ED18004FEA430C7FEA6C5CD6D152EA033CD3D06D
:10ED28005DF8040B704700BF8446104662468C4667
:10ED38001946634600E000BF01B5FFF7B7FF00289A
:10ED480048BF10F1000F01BD4DF808EDFFF7F4FFC3
:10ED58000CBF012000205DF808FB00BF4DF808ED4E
:10ED6800FFF7EAFF34BF012000205DF808FB00BF71
:10ED78004DF808EDFFF7E0FF94BF012000205DF893
:10ED880008FB00BF4DF808EDFFF7CEFF94BF012048
:10ED980000205DF808FB00BF4DF808EDFFF7C4FF41
:10EDA80034BF012000205DF808FB00BF4FEA410294
:10EDB80012F5001215D211D56FF47873B3EB6252C5
:10EDC80012D94FEAC12343F0004343EA505311F0EC
:10EDD800004F23FA02F018BF404270474FF000007E
:10EDE800704750EA013005D111F0004008BF6FF0BC
:10EDF800004070474FF00000704700BF4A0011D232
:10EE080012F5001211D20DD56FF47873B3EB62527C
:10EE18000ED44FEAC12343F0004343EA505323FA88
:10EE280002F070474FF00000704750EA013002D1FD
:10EE38004FF0FF3070474FF0000070474FEA410233
:10EE4800B2F1E04324BFB3F5001CDCF1FE5C0DD940
:10EE580001F0004C4FEAC0024CEA5070B2F1004F8A
:10EE680040EB830008BF20F00100704711F0804F8D
:10EE780021D113F13872BCBF01F00040704741F452
:10EE880080114FEA5252C2F11802C2F1200C10FA56
:10EE98000CF320FA02F018BF40F001004FEAC1233A
:10EEA8004FEAD32303FA0CFC40EA0C0023FA02F3DE
:10EEB8004FEA4303CCE77FEA625307D150EA0133B4
:10EEC8001EBF4FF0FE4040F44000704701F0004084
:10EED80040F0FE4040F40000704700BF4BB942B913
:10EEE800002908BF002802D04FF0FF31084600F083
:10EEF80037B882B0EC462DE9005000F01BF8DDF879
:10EF080004E002B00CBC7047F8B5144606460F463C
:10EF18001D4600F027F804FB01F300FB0535A4FBB0
:10EF28000023EB18069CB21A67EB0303C4E900231D
:10EF3800F8BD00BFF8B5144606460F461D4600F05A
:10EF480075F900FB05F5A0FB042304FB0155EB183C
:10EF5800069CB21A67EB0303C4E90023F8BD00BF9F
:10EF6800704700BF00292DE9F0071D46C0F29E80BA
:10EF78000024002DC0F2958007460D4616469C4693
:10EF8800002B3ED18A4254D9B2FA82F343B1C3F17D
:10EF9800200620FA06F501FA03F19A402943984021
:10EFA800160CB1FBF6F597B206FB15114FEA104C9B
:10EFB80007FB05F34CEA01418B4209D9891805F191
:10EFC800FF3C80F015818B4240F21281023D891886
:10EFD800C3EB010CBCFBF6F306FB13C180B207FBC5
:10EFE80003F740EA0140874207D9591E821880F08A
:10EFF8000581974240F20281023B43EA0542002321
:10F0080003E08B420AD900231A461046194614B168
:10F01800404261EB4101BDE8F0077047B3FA83F362
:10F02800002B40F087808C4501D38242ECD8012226
:10F03800EBE712B90123B3FBF2F2B2FA82F6002E23
:10F048003AD1891A150C1FFA82FC0123B1FBF5F796
:10F0580005FB17114FEA10480CFB07F648EA014177
:10F068008E4207D9891807F1FF3802D28E4200F282
:10F07800DA804746891BB1FBF5F605FB161180B20D
:10F088000CFB06FC40EA0140844507D9711E821832
:10F0980080F0B080944540F2AD80023E46EA0742D7
:10F0A800B3E7E443524263EB430365E7404261EB55
:10F0B80041014FF0FF345CE7B240C6F1200521FA68
:10F0C80005F320FA05F701FA06F9150CB3FBF5F874
:10F0D80047EA09091FFA82FC05FB18374FEA19416C
:10F0E8000CFB08F341EA0747B040BB420AD9BF18F6
:10F0F80008F1FF3180F09580BB4240F29280A8F180
:10F108000208BF18FE1AB6FBF5F305FB13611FFAD8
:10F1180089F90CFB03F649EA01418E4206D95F1EC4
:10F12800891878D28E4276D9023B8918891B43EA1E
:10F1380008438BE7C3F1200726FA07F80CFA03F215
:10F1480048EA020C21FA07F105FA03FA4FEA1C49CA
:10F1580020FA07F5B1FBF9F845EA0A0509FB181783
:10F168002A0C1FFA8CFA0AFB08F142EA0747B9424F
:10F1780006FA03F609D917EB0C0708F1FF324ED24D
:10F18800B9424CD9A8F1020867447F1AB7FBF9F2D3
:10F1980009FB1271ADB20AFB02FA45EA01418A4540
:10F1A80007D9551E11EB0C0137D28A4535D9023AD9
:10F1B800614442EA08424FEA124C1FFA86F808FBFB
:10F1C8000CF7360C95B208FB05F806FB057505EB40
:10F1D800184506FB0CFCAF4288BF0CF5803CCAEB17
:10F1E80001010CEB1546B14212D309D000230CE7FC
:10F1F8006546EDE60E4646EA074206E70B46FCE69C
:10F208001FFA88F800FA03F308EB0545AB42EDD284
:10F21800013A0023F9E63B4688E72A46C9E79046C3
:10F22800B3E788466EE7023F891823E72DE9F00F18
:10F23800144605460E46002B3FD18A424AD9B2FAF7
:10F2480082F343B1C3F1200025FA00F201FA03F674
:10F258009C4016439D40210CB6FBF1F22F0CA0B246
:10F2680001FB126C00FB02F347EA0C46B34208D9D3
:10F27800571E361980F0FF80B34240F2FC80023AF4
:10F288003619F61AB6FBF1F301FB1361ADB200FBB8
:10F2980003F045EA0141884207D95E1E091980F04A
:10F2A800EC80884240F2E980023B43EA02420023B4
:10F2B80010461946BDE8F00F70478B4243D8B3FAA1
:10F2C80083F4002C42D18B42234601D382423BD89F
:10F2D8000122EDE712B90123B3FBF2F4B4FA84F288
:10F2E800002A40F08A80091B260CA7B20123B1FB33
:10F2F800F6F006FB10114FEA154C07FB00F24CEA3A
:10F3080001418A4207D9091900F1FF3C02D28A4219
:10F3180000F2D3806046C2EB010CBCFBF6F206FBA0
:10F3280012C1ADB207FB02F745EA0145AF4207D962
:10F33800511E2C1980F0A380A74240F2A080023A07
:10F3480042EA0042B4E700231A46B1E7C4F12007B5
:10F3580022FA07F603FA04F3334321FA07FA4FEACD
:10F36800134C01FA04FB20FA07F141EA0B0BBAFB34
:10F37800FCF70CFB17A61FFA83F84FEA1B4508FB9E
:10F3880007F945EA0645A94502FA04FA04D97A1E9E
:10F39800ED18C0F088801746C9EB0505B5FBFCF6EB
:10F3A8000CFB16521FFA8BFB08FB06F84BEA0241CE
:10F3B800884503D9721EC91870D3164646EA074213
:10F3C800170C1FFA8AFC0CFB07F695B24FEA1A4392
:10F3D8000CFB05FC03FB056505EB1C4503FB07F36C
:10F3E800AE4288BF03F58033C8EB010103EB154338
:10F3F800994250D347D000235AE79440C2F12008DD
:10F40800260C20FA08F721FA08F501FA02F9B5FBEB
:10F41800F6F847EA090906FB1855A7B24FEA194C4E
:10F428004CEA054C07FB08F3634500FA02F509D9D5
:10F438001CEB040C08F1FF323DD263453BD9A8F11F
:10F448000208A444C3EB0C02B2FBF6F306FB13203C
:10F458001FFA89F907FB03F249EA00418A4206D9F3
:10F46800581E091925D28A4223D9023B0919891A3B
:10F4780043EA08433BE73A4603E7334615E70A46BB
:10F4880042EA004214E71FFA8CF100FA04F001EB9B
:10F498000545A842AFD2013A002309E788458CD92F
:10F4A800023EC9188AE7A9457FF675AF023FED18F5
:10F4B80072E70346DBE79046C4E7023809192AE7F2
:10F4C800002103E00A4B5B584350043109480A4BBA
:10F4D80042189A42F6D3094A02E0002342F8043B54
:10F4E800074B9A42F9D3F9F77DF900F00DF8704708
:10F4F80024A60508000000200C0B0020100B00209B
:10F50800E4610020FEE70000814B824A2DE9F341C7
:10F518004FF4FA661E60804BDFF868821A607F4AF3
:10F528007F4B1A607F4B42F210721A607E4B642444
:10F538001C607E4B4FF0FF321A607D4B00251D701A
:10F54800012788F80070F7F7F9FEF6F72BFF204639
:10F55800F7F78EFBF6F74CFF2046F7F789FBF7F72E
:10F56800D3FEF7F721FDF7F799FB2046F7F780FB65
:10F57800F9F720FA2046F7F77BFB4FF4FA50F7F734
:10F58800E3FA2046F7F774FBF6F764FE2046F7F730
:10F598006FFB2846F7F7ACFB6648F7F769FBF4F70B
:10F5A800BFF92046F7F764FB634B03F110022946C5
:10F5B8008DE8240028465A681B68F4F7B7FB3046E4
:10F5C800F7F756FB2846F4F731FE4FF6FF70F4F7CD
:10F5D80043FE32200321594A2B46F4F755FF962063
:10F5E8008C21574A2B46F4F74FFF9620554AA02105
:10F5F8002B46F4F749FFB421534A2B469620F4F7DB
:10F6080043FF3046F7F734FBDC21504A2B462846A7
:10F61800F4F73AFF4E48F7F72BFB2046F7F728FB9D
:10F62800F6F7E0FB2046F7F723FB9FED4A0AF7F7CA
:10F6380077FB2046F7F71CFB474B484A00933946AF
:10F64800474B4848FBF782FC2046F7F711FBF5F7D4
:10F65800E5F92046F7F70CFB1420F6F731F92846B0
:10F66800F6F781F92046F7F703FBF6F705FB204686
:10F67800F7F7FEFAF6F78EFE2046F7F7F9FAF6F7EF
:10F6880001FC08B188F80050374B1D70F1F7E8FD10
:10F69800F5F77AF908B9354803E0354B35480022C3
:10F6A8001A70F1F7F4FD344E344DF5F7E1FDF8F733
:10F6B800D8F9F8F70BFAF8F70DF8F7F747FF3746D8
:10F6C800F6F702FC337833B1012B02D1F7F79AFC35
:10F6D80001E0F7F7BFFC00243C70F7F7FDFDF3F7F6
:10F6E800A1FBF8F7B7FF2A8812B2012AE8D124480B
:10F6F8004FF40051FDF787F9F8F748FAF7F796FD48
:10F708001F484FF400512246FDF77DF92C80D7E7BA
:10F718005C400020E06735008040002080C3C901BC
:10F728003041002084400020444000207C400020DC
:10F73800604D002000127A00207801081F9F0508FC
:10F74800399F0508459F0508519F05085A9F0508D8
:10F75800002D31010000FA44C4010020904000202F
:10F7680024020020903A002064400020B40D0020BC
:10F778008C3A0020A00F002088400020FC0B0020BD
:10F7880000080240000D002010B4314C0180B1F592
:10F79800807F44608270C37052D00DD9B1F5806FFC
:10F7A80039D017D9B1F5006F2ED0B1F5805F24D0CC
:10F7B800FF2040B210BC704720293AD014D9402904
:10F7C80030D08029F4D123494FF02012C2608160E3
:10F7D8000020EEE7B1F5007FEAD11F4B4FF008118A
:10F7E800C16083600020E4E71029E1D11B494FF094
:10F7F8000122C26081600020DBE7194B4FF0011144
:10F80800C16083600020D4E7164A4FF00213C3603A
:10F8180082600020CDE714494FF00412C260816075
:10F828000020C6E7114B4FF04011C16083600020F3
:10F83800BFE70F4A4FF08013C36082600020B8E72B
:10F848000C4A4FF01013C36082600020B1E700BF7C
:10F85800389E0408768E0508468E050836900508F9
:10F86800388E05083A8E05083E8E0508B68E0508BE
:10F87800368F0508568E05082DE9F00FB2B02E9088
:10F8880030932E9B00882E9C5B68309FA4682D9037
:10F89800451E03EB4506BF08209328942C952F910D
:10F8A8001F921E96319700F03A814FEA900A4FEA6C
:10F8B800CA0B00F003002F99299003F1080504EB07
:10F8C8000B00CDF884A0CDF8A8B019951A921B9713
:10F8D800189617912B90179A189E13883380B2F8B0
:10F8E80002C0A6F802C09488B480D788F78008368A
:10F8F8001896219F199E0832179256F8041C56F83C
:10F90800082C4FF0000A4FF0000B002F00F069821E
:10F91800CDE904ABCDE906ABCDE902ABCDE900AB4F
:10F92800289CBC46029BDDF80C902568C2FBC539B3
:10F938004FF0000848EA030ACB46CDE902AB049B26
:10F94800DDF814B0C1FBC53BCDF824B0CDF820805C
:10F95800DDE908ABC1EA02004AEA030ACDE904ABD3
:10F96800069BDDF81CB03268C0FBD53BCDF82CB047
:10F97800CDF82880DDE90AABC2EA01074AEA030AA2
:10F98800CDE906AB9DE80108C7FBD50BCDF834B02F
:10F99800CDF83080DDE90CAB4AEA000A63680298CA
:10F9A800CDE900AB0834DDF80CB0C1FBC30BCDF8D2
:10F9B8003CB0CDF83880DDE90EAB4AEA000ACDE963
:10F9C80002AB71680498DDF814B0C2FBC30BCDF824
:10F9D80044B0CDF84080DDE910AB4AEA000ACDE931
:10F9E80004AB0698DDF81CB0C7FBD30BCDF84CB0C0
:10F9F800CDF84880DDE912ABC1EA02054AEA000AFF
:10FA0800CDE906AB9DE80108C5FBD30BCDF854B092
:10FA1800CDF85080DDE914AB08364AEA000ABCF19B
:10FA2800010CCDE900AB7FF47DAF2A9D19982B9B83
:10FA38002E18299F002F35D01868039F029BC2FB00
:10FA4800C03700241D971C94DDE91C4544EA0304D3
:10FA5800CDE90245049B059DC1FBC03500272395D0
:10FA68002297DDE9224544EA0304CDE90445C1EAC9
:10FA78000203079D069AC3FBD02525952497DDE947
:10FA8800244544EA02043368C3EA0101CDE9064586
:10FA980053465D46C1FBD03527952697DDE926AB51
:10FAA8004AEA030A069A029C0499039D079FD30B0E
:10FAB800059AE60BC90B46EA454043EA474441EA42
:10FAC800424604F30F0500F30F0C199BCCEA0547D7
:10FAD80006F30F001A9D1B9E2F604FEADA3A08338F
:10FAE8004AEA4B4B0BF30F04C0EA04426A6008353C
:10FAF800711E19931A951B917FF4EDAE319A2F9EC2
:10FB08001E991F9BDDF880B0D00037180D182F976D
:10FB18000BEB000A1F181E951F97CDF880A0DDF883
:10FB2800C0C01CF0030BCDF820B000F086802D9BE0
:10FB3800DDF8BC80CDF808B05808DDF880A0DDF805
:10FB4800A0B00690CDF81080049A1E9E32F8025B91
:10FB5800069826F8025B0492BAF80270BBF80230E5
:10FB6800BAF80020BBF800401E9617FB03F112FB01
:10FB780004F6451E4FEAE17711EB06082B4605F01F
:10FB8800010047EBE6790AF104020BF10401002DAC
:10FB98003BD0A8B1B2F800C0BBF8047054884888BC
:10FBA8001CFB07F518EB050749EBE57614FB00F994
:10FBB80017EB090846EBE97904320431013B24D0FC
:10FBC8000F88B2F800C0568848888C8895881CFB36
:10FBD80007FC18EB0C0816FB00F7D088CE8849EB19
:10FBE800EC7C15FB04F518EB07084CEBE77918EBF0
:10FBF800050710FB06FC49EBE57417EB0C0844EB12
:10FC0800EC7908320831023BDAD11F9A02994FEA9F
:10FC1800D83545EA494404F30F0322F8023B4F1E46
:10FC28000AF1020A1F9202978ED1DDF880A0DDF852
:10FC380020B00AEB4B0ACDF880A02C9E2E98B50870
:10FC480040683FD0209F47EA000212F0030F00F1FE
:10FC5800080307F1080214BF002101219F4298BF41
:10FC6800904294BF00260126314277D097E842009F
:10FC7800016001216C1EA942466004EA010419D002
:10FC880044B192E81200196002215C60083208331E
:10FC9800A9420FD092E850001C605E60966802F19D
:10FCA800080BD2689E600231DA601033A9420BF16A
:10FCB8000802EFD1DDF880C0ED000CEB050B401910
:10FCC800CDF880B02C9C14F0030343D05A0854009C
:10FCD800002A00F08E80209D40EA050717F0030FE8
:10FCE800209F14BF00250125011D3E1D012B94BF37
:10FCF800002505F001058F4298BFB04294BF00214E
:10FD080001210D4275D039689200BF18A3420160E5
:10FD180020971044C4EB03011CD0209B013933F811
:10FD2800024B0A4620F8024B01F0010192B129B1B9
:10FD380033F8021B013A20F8021B0BD01C4601467F
:10FD480034F802CB21F802CB5D88A31C4580881CBF
:10FD5800023AF3D132B0BDE8F00F7047B7F800C0EF
:10FD6800A0F800C07C884480BE888680691EFE8812
:10FD78000C46BA4601F00101C680002C9AD089B120
:10FD8800B2F800B0A3F800B051885980B2F804C0A6
:10FD9800A3F804C0B2F806B00832A3F806B00833D6
:10FDA800013C87D016881E8051885980B2F804B06B
:10FDB800A3F804B0B2F806C0A3F806C016891E81DD
:10FDC80003F1080B5189ABF802109389ABF80430A2
:10FDD800D6891032023C0BF10803ABF80660E1D17A
:10FDE80068E7289BCDE904ABCDE906ABCDE902ABCA
:10FDF8001FE6194691E700BF2DE9F00F9CB0067881
:10FE08000F900F9C40880F9DA4686D681990B3FBF4
:10FE1800F6FA471E4FEA5A0804EB4709AAEB4803CB
:10FE280040460A940D951A97CDF86C800C9114925F
:10FE3800CDF82C901193002800F0B5811746199A37
:10FE4800199CCDF848809108CA00159104F0030365
:10FE5800A9181792169310971891760075084FEA0B
:10FE6800450C002D00F03B840B9FDDF8308047EAFD
:10FE7800080010F0030F14BF0021012108F1040449
:10FE8800381D012E94BF002101F00101804598BF63
:10FE9800A74294BF4FF000094FF0010911EA090F7A
:10FEA80000F01D84BB46D8F8002001236F1EAB422A
:10FEB800CBF8002007EA03072146024614D237B1DF
:10FEC800246802230431021DAB4204600CD20C46A4
:10FED800104654F8047B40F8047B496802335160AB
:10FEE800211D021DAB42F2D3DDF83080DDF82CB0C5
:10FEF8004FEA4C05664508EB05020BEB0503CCEB16
:10FF080006001DD0013832F802CB014623F802CB97
:10FF180000F00100A1B128B132F8029B013923F8A1
:10FF2800029B0DD014461F4634F8029B27F8029B0B
:10FF3800B2F802A0A21CA3F802A0BB1C0239F1D19E
:10FF48000C9ADDF83CC00B989CF80080710053189F
:10FF58000A9E0C93159BCDF84C80451806EB480279
:10FF68000B950E92002B00F0B18300240025CDE9FB
:10FF78000445CDE9024507930D9913460A9AB3F84B
:10FF880004A0B2F806B0CDF804A0B3F806A00E8815
:10FF98001588CDF820B0CDF824A0DDE902AB15FB1B
:10FFA80006F51AEB050A4BEBE57BCDE902AB1F889A
:10FFB8004888B2F802C0B3F80290B2F804808C887E
:10FFC800CDF81880DDE904AB16FB07F61AEB060A34
:10FFD8004BEBE67BDDE902671CFB00F5761910FBAD
:10FFE80009F047EBE5771AEB000A4BEBE07BCDE92C
:08FFF80002ABDDF818B0DDF8E2
:020000040801F1
:1000000004C0B1F80680099D1BFB04F016EB000A42
:1000100047EBE07BDDE9026714FB0CF4361947EB94
:10002000E477089C14FB08F00831083208331AEB17
:10003000000418FB05F84BEBE075079816EB080A6F
:1000400047EBE87B0138CDE90245CDE904AB0790E9
:1000500099D1179E0E9C0A9B1899A7199A190E9769
:10006000169F002F73D00E9B31F8020B32F8024B13
:1000700033F8026BDDE90289DDE904AB14FB00F41F
:100080007D1E10FB06F618EB040849EBE4791AEB29
:10009000060A4BEBE67B2F4605F00100CDE902890D
:1000A000CDE904AB002D52D0002873D031F8024BBB
:1000B00032F8020B33F8025B10FB04F614FB05F078
:1000C000DDE90245DDE90489A41945EBE67518EB85
:1000D000000849EBE079013FCDE90245CDE904890B
:1000E00035D0C246CB46DDE902890D461446049759
:1000F000214628461A4630F8026B31F8027B32F866
:1001000002CB6D8864885B8817FB06F718EB07083D
:1001100016FB0CF649EBE7791AEB060714FB05FA18
:100120004BEBE67B15FB03FC8C1C931C0499851C94
:1001300018EB0A0849EBEA7917EB0C0A4BEBEC7B5E
:100140008A1ECDE902890492D2D1CDE904AB029D89
:1001500003990498DDF828A0059BEA0B109D42EA5C
:100160004148129908F30F09A5F80090DDF84C906A
:10017000C70B0AEB8908281D4A1E47EA4346CDF8FB
:10018000288006F30F0410906C8012920AD00F9C06
:10019000267866E6DDE904AB0D4614460497DDE9F2
:1001A0000289A5E7149F1B9B07EB83061496119FFA
:1001B000002F00F0A681DDF864B0DDF86480DDF882
:1001C00034C04FEA9B09CDF81C904FEAC90908F0EA
:1001D000030A0CEB090BCDF82090CDF810A0CDF858
:1001E00024B0DDF83CC09CF8006075084FEA450C6F
:1001F000002D00F07E820C990B980B9F40EA0104C1
:1002000014F0030F14BF002201220C1D0430012E34
:1002100094BF002202F00102814298BFA74294BF1E
:10022000002301231A4200F06482BA4601230F68BA
:10023000691EAB42CAF80070024601EA0307214674
:1002400014D237B127680223211D021DAB4207607B
:100250000CD20C46104654F8047B40F8047B4968E5
:1002600002335160211D021DAB42F2D3DDF8309004
:10027000DDF82C804FEA4C05664509EB050208EBDA
:100280000503CCEB06001DD0013832F802BB014655
:1002900023F802BB00F00100A1B128B132F8025BE3
:1002A000013923F8025B0DD014461F4634F802AB27
:1002B00027F802ABB2F802C0A21CA3F802C0BB1C14
:1002C0000239F1D1DDF82CA0DDF830B007987600C6
:1002D0000AEB060C0BEB0608CDF82CC0CDF83080ED
:1002E000002800F0F0810A9ADDF834805788B2F8CF
:1002F00000A0DDF828909488B9F80690B8F8062098
:1003000084460D9841880588B8F8040017FB01F66B
:100310001AFB05F3B3461BEB03014FEAE67714FB28
:1003200000F047EBE3750F180A9B19FB02F145EB50
:10033000E0750CF1FF3617EB010AB14606F001003B
:1003400008F1080203F1080345EBE17B002E00F001
:10035000858048B3DDF834C01E88BCF80840588852
:10036000518897889D88B2F80680B3F806C016FBBE
:1003700004F41AEB040A10FB01F14BEBE4761AEBE0
:10038000010415FB07FB46EBE17014EB0B011CFBB2
:1003900008F640EBEB740832083311EB060A44EB25
:1003A000E67BB9F1010959D0CDE902ABCB46B3F8F0
:1003B0000080B3F808901688CDF8389018FB06F640
:1003C000DDE902895D88548898889188B2F806C072
:1003D000DF88B2F808A015FB04F418EB060810FB40
:1003E00001F149EBE67918EB040817FB0CF749EB30
:1003F000E47918EB010849EBE17918EB070849EBC0
:10040000E779CDE90289DDF838905D8954899889CA
:100410009189B2F80EC0DE8919FB0AF7DDE902897D
:1004200015FB04F418EB070810FB01F149EBE77921
:1004300018EB040849EBE47916FB0CF618EB010401
:1004400049EBE17510321033A01945EBE671BBF1B1
:10045000020BCDE90201AAD182468B460DF120089C
:1004600098E816006318049D9DB332F802CB33F868
:10047000026B16FB0CF4013D1AEB040A294605F049
:1004800001004BEBE47B25B358B132F8028B33F813
:10049000020B10FB08F71AEB070A4BEBE77B691E10
:1004A00017D01446184634F8025B30F8027B5288A5
:1004B0005B8817FB05F81AEB08064BEBE87713FB94
:1004C00002FBA21C831C16EB0B0A47EBEB7B0239E9
:1004D000E7D10F9DDDF8508095F800C00A9A119E73
:1004E0004FEADA3343EA4B4404F30F0028F8020BD7
:1004F00002EB4C07711E0A97CDF8508011917FF4E2
:1005000070AE1A9E0F9CB508A06842D00A9F47EAB9
:10051000000616F0030F07F1080200F1080314BFEC
:10052000002101219F4298BF904294BF4FF0000AE2
:100530004FF0010A11EA0A0F7FD097E842000160EC
:1005400001216C1EA942466004EA010419D044B19D
:1005500092E81200196002215C6008320833A94257
:100560000FD092E850001C605E60966802F10804AB
:10057000D2689E600231DA601033A94204F10802A9
:10058000EFD1DDF828A0ED000AEB05094019CDF800
:100590002890DDF868A01AF003034AD05A085400E6
:1005A000002A00F0A480DDF828B040EA0B0515F021
:1005B000030F14BF002501250BF10406011D012BBB
:1005C00094BF002505F001058B4598BFB04294BF4C
:1005D0004FF0000C4FF0010C15EA0C0F00F0878073
:1005E000DBF8001092009344A3420160CDF828B0DC
:1005F0001044C4EB03011CD00A9B013933F8024BB1
:100600000A4620F8024B01F0010192B129B133F8FA
:10061000021B013A20F8021B0BD01C46014634F89D
:1006200002CB21F802CB5D88A31C4580881C023ACE
:10063000F3D11CB0BDE8F00F7047B7F80090A0F8F8
:1006400000907C884480BE888680691EFE880C46A7
:10065000B84601F00101C680002C92D091B11188FA
:100660001980B2F802C0A3F802C0B2F804A0A3F83F
:1006700004A0B2F806900832A3F806900833013CB3
:100680003FF47FAF11881980B2F802C0A3F802C00E
:10069000B2F80490A3F80490B2F806A0A3F806A05C
:1006A00016891E8103F1080C5189ACF80210938958
:1006B000ACF80430D6891032023C0CF10803ACF8D7
:1006C0000660DFD15DE70D9A0A9B4FF0000A4FF0FC
:1006D000000BC8E600260027CDE904670A9A0D99A9
:1006E000CDE90267BCE430460B9B0C9A0EE4194638
:1006F00082E730460B9B0C9AC6E500BF0000000065
:1007000000B553EC102B42F2FB1223F00043C3F66A
:10071000E972934285B026DD4FF6FF72C7F6EF729D
:1007200093420BDD51EC100B02460B46FDF7F4FE35
:1007300002460B4643EC102B05B000BD684600F0A6
:10074000BFFB00F0030001289DED000B9DED021B97
:100750001AD0022810D0F8B900F0D2FE53EC102BBA
:1007600010461946E4E79FED101B00F0C9FE53EC5C
:10077000102B10461946DBE700F0C2FE53EC102B9D
:10078000104603F10041D3E701F0F6FB53EC102BC8
:10079000104603F10041CBE7012001F0EDFB53ECE3
:1007A000102B10461946C3E70000000000000000AF
:1007B0002DE9F04759EC108BC9F30A56A6F57E7463
:1007C000073C132C4D46CA46474626DC002C4FDB1F
:1007D0004FF6FF76C0F20F0646FA04F606EA090560
:1007E00055EA080517D044A3D3E9002351EC100BB8
:1007F000FDF794FE00220023FEF7D2FA00284AD02B
:10080000B9F1000F6EDB2AEA060A4FF000085346E2
:10081000424643EC102BBDE8F087332C0CDDB4F5D9
:10082000806FF8D151EC100B3A460B46FDF776FE7F
:1008300041EC100BBDE8F087A6F58265033D4FF053
:10084000FF3323FA05F515EA080FE4D02AA3D3E90C
:10085000002351EC100BFDF761FE00220023FEF790
:100860009FFAC0B1B9F1000F1CDB28EA050813E0BC
:1008700021A3D3E9002351EC100BFDF74FFE00221A
:100880000023FEF78DFA38B1B9F1000F1BDB4FF0F2
:100890000008C24600E0CA465346424643EC102BCD
:1008A000BDE8F087142C09D0C6F5866303334FF0FA
:1008B000010808FA03F818EB0708D6D30AF1010A71
:1008C00028EA0508E8E729F0004848EA07084FF059
:1008D000000AD045CBF6F07A08BFCA4618BF4FF0E1
:1008E0000008D9E74FF4801343FA04F409EB040A33
:1008F00089E700BFAFF300809C7500883CE4377E39
:1009000000B553EC102B42F2FB1223F00043C3F668
:10091000E972934285B027DD4FF6FF72C7F6EF729A
:1009200093420BDD51EC100B02460B46FDF7F4FD34
:1009300002460B4643EC102B05B000BD684600F0A4
:10094000BFFA00F0030001289DED000B9DED021B96
:100950001DD0022812D008BB012001F00DFB53EC82
:10096000102B10461946E3E700209FED111B01F004
:1009700003FB53EC102B10461946D9E7012001F078
:10098000FBFA53EC102B104603F10041D0E700F0C6
:10099000B7FD53EC102B10461946C9E700F0B0FD27
:1009A00053EC102B104603F10041C1E7AFF3008078
:1009B000000000000000000000F0E6B8D0B52DED0A
:1009C000048BB0EE408AF0EE608A3C4C8AB000F0B6
:1009D000DBF994F90030B0EE409AF0EE609A013302
:1009E00035D0B0EE480AF0EE680A01F04FFD00285D
:1009F0002DD051EC180B00220023FEF7BDF930B3C7
:100A00002F4B24780193002308938DED028B8DEDFD
:100A1000048B002C23D000270026CFF6F07751EC72
:100A2000180B00220023CDE90667FEF791F9002894
:100A300025D002239C42009336D0684601F05EFD2B
:100A4000002831D0089B002B27D19DED069BB0EEEE
:100A5000490AF0EE690A0AB0BDEC048BD0BD4FF62E
:100A6000FF774FF06046CCF2EF7751EC180B002285
:100A70000023CDE90667FEF76BF90028D9D10123E1
:100A8000022C009315D0684601F038FD88B10D485E
:100A900001F036FD8DED060BD4E701F0EFFF089B6A
:100AA0009DED069B0360D2E701F0E8FF222303607F
:100AB000C8E701F0E3FF21230360E8E74C020020D0
:100AC00024A1050888A3050810B52DED048BB0EE10
:100AD000408AF0EE608A294C8AB000F02DFC94F92F
:100AE0000030B0EE409AF0EE609A01332BD0B0EEB9
:100AF000480AF0EE680A01F0C9FC20B351EC180B6B
:100B000000220023FEF72EF9E8B11D4B2478019353
:100B100001230093002308938DED048B8DED028B50
:100B2000CCB10020002102460B46FDF7D3FF022C7A
:100B3000CDE9060115D101F0A1FF21230360089B37
:100B4000ABB99DED069BB0EE490AF0EE690A0AB01A
:100B5000BDEC048B10BD0022002343EC172B8DED60
:100B6000067B684601F0CAFC0028E8D1E3E701F003
:100B700085FF089B9DED069B0360E4E74C02002087
:100B80002CA1050800000000F8B5B0EE407AF0EEA8
:100B9000607A53EC112B544210461D46002125F07B
:100BA0000047044353EC102B47EAD474C7F6F071A6
:100BB0008C4216463DD85442344323F0004242EA68
:100BC000D4748C4235D805F1404101F580110143C0
:100BD0004FD0AC1704F00204164344EAD37435D066
:100BE000384341D00021C7F6F0718F424FD0002129
:100BF000C7F6F0718A4237D0D21B12153C2A42DC6C
:100C0000002D7DDB53EC112B51EC170BFDF762FF30
:100C100041EC100B01F030FC01F06AFA51EC100BC2
:100C2000012C68D0022C57D0002C48D141EC170B76
:100C300007E051EC170B53EC112BFDF76FFC41EC67
:100C4000170BB0EE470AF0EE670AF8BD032CC7D8C1
:100C500001A151F824F000BF430C0108430C010826
:100C6000810C01087B0C0108002B25DB9FED307BFC
:100C7000E7E7BDE8F84001F03BBA9FED2F7BE0E7E6
:100C80009FED2F7BDDE72AA1D1E90001C8E7BA4239
:100C90003CD0032CABD801A151F824F0B30C0108CF
:100CA000AD0C0108810C01087B0C01089FED267B2F
:100CB000C7E79FED277BC4E79FED277BC1E730A304
:100CC000D3E90023FDF728FC1DA3D3E90023FDF79A
:100CD00023FC41EC170BB4E729A3D3E90023FDF76C
:100CE0001BFC02460B4616A1D1E90001FDF714FCDE
:100CF00041EC170BA5E701F1004141EC170BA0E710
:100D00003C32BFF67FAF0020002189E7032CABD82F
:100D1000DFE804F00B0805029FED117B91E79FEDE2
:100D2000127B8EE79FED127B8BE79FED137B88E7AD
:100D3000182D4454FB21F93F182D4454FB2109C0C0
:100D4000182D4454FB2109400000000000000080E1
:100D50000000000000000000182D4454FB21F9BFE2
:100D6000D221337F7CD902C0D221337F7CD902408B
:100D7000182D4454FB21E9BF182D4454FB21E93FB1
:100D8000075C143326A6A13C2DE9F84F55EC104B17
:100D9000B5F5801F2F4622DA25F00043234368D0A3
:100DA000002D2046294670DB00230022C4F2503378
:100DB000FDF766FD4FF6FF730F46C7F6EF739F42D0
:100DC00004460D466FF0350210DD204629462246C6
:100DD0002B46FDF7A3FB41EC100BBDE8F88F4FF657
:100DE000FF73C7F6EF7300229F42EEDC3B15A3F5BD
:100DF0007E73073B9A18D60F901927F07F47C6F5E8
:100E00007E76FDF7D7FC073627F4700747EA0655CC
:100E100045EC104B8046894601F00AFC40464946A5
:100E200021A3D3E9002355EC104BFDF729FD20A3A6
:100E3000D3E9002382468B4640464946FDF720FD14
:100E40001DA3D3E9002306460F4620462946FDF799
:100E500017FD02460B4630463946FDF75FFB02465A
:100E60000B4650465946FDF759FB41EC100BBDE8C7
:100E7000F88F00210020CCF2503100220023FDF732
:100E800029FE41EC100BBDE8F88F22462B46FDF7FA
:100E900043FB00220023FDF71DFE41EC100BBDE8D3
:100EA000F88F00BFAFF3008000609F501344D33F22
:100EB000362BF111F3FE593D0EE526157BCBDB3FBA
:100EC0002DE9F04F53EC102B42F2FB1223F00044BB
:100ED000C3F6E97294428FB01E46074640F3AA80DB
:100EE0004DF67B13C4F202039C422ADC002E51EC27
:100EF000100BDDA3D3E9002340F3CA81FDF70CFBFF
:100F000042F2FB13C3F6F9739C428046894600F017
:100F1000AA80D7A3D3E90023FDF7FEFA0D460446C5
:100F20002B462246C7E9004540464946FDF7F4FAFC
:100F3000CFA3D3E90023FDF7EFFA0125C7E90201AA
:100F400081E042F2FB13C4F239139C4240F3AA80C1
:100F50004FF6FF73C7F6EF739C4278DC4FEA245AD2
:100F6000AAF5826AAAF1060A51EC100BA4EB0A5307
:100F700019461D460446FDF71DFFFDF71BFC804684
:100F8000894642464B4620462946CDE90889FDF769
:100F9000C3FA00230022C4F27013FDF771FC0D4662
:100FA0000446FDF707FFFDF705FC8046894620460D
:100FB000294642464B46CDE90A89FDF7ADFA0023A2
:100FC0000022C4F27013FDF75BFC002204460D46BC
:100FD0000023CDE90C45FDF7BBFE002800F07B8126
:100FE0004046494600220023FDF7B2FE03240AAD25
:100FF000013C40B175E9020100220023FDF7A8FE83
:10100000013C0028F6D12346022400949E4C08A8F7
:1010100039465246019400F0ABFB002E054612DA29
:101020007A68FB6802F1004203F100437A60FB60DA
:10103000454208E00022002343EC172B87ED000B0C
:1010400080ED027B002528460FB0BDE8F08F51EC03
:10105000100B02460B46FDF75FFA0025C7E90201B7
:10106000C7E90001EFE77AA3D3E90023FDF754FABB
:1010700079A3D3E9002380468946FDF74DFA0D4652
:1010800004462B462246C7E9004540464946FDF73F
:1010900043FA71A3D3E90023FDF73EFA0125C7E91E
:1010A0000201D0E701F0E8F959EC108B6CA3D3E909
:1010B000002340464946FDF7E3FB00230022C3F628
:1010C000E073FDF72BFAFDF775FE0546FDF772FBA1
:1010D00065A3D3E90023CDE90201FDF7D1FB024668
:1010E0000B4640464946FDF717FA61A3D3E90023B2
:1010F00082468B46DDE90201FDF7C2FB1F2DCDE9DB
:101100000401504659462BDC6A1E604B53F82230CE
:10111000A34225D0DDE90423FDF7FEF902460B4684
:10112000C7E90023814688464A4643465046594609
:10113000FDF7F2F9DDE90423FDF7EEF9002E024692
:101140000B46C7E90223BFF67EAF08F1004301F169
:101150000041C7F800907B60B860F9606D4272E7AB
:10116000DDE90423FDF7D8F988462415C8F30A53AE
:10117000E31A102B8146C7E90001D5DD34A3D3E97A
:101180000023DDE90201FDF77BFB804689464246EC
:101190004B4650465946FDF7BFF9CDE90601DDE95A
:1011A000062350465946FDF7B7F942464B46FDF730
:1011B000B3F929A3D3E9002380468946DDE902017A
:1011C000FDF75EFB42464B46FDF7A6F9CDE904016B
:1011D000DDE90423DDE90601FDF79EF98846C8F341
:1011E0000A53E41A312C8146C7E9000140F3958087
:1011F00021A3D3E90023DDE90201FDF741FB80468D
:10120000894642464B46DDE90601FDF785F98246EF
:101210008B4652465B46DDE90601FDF77DF9424605
:101220004B46FDF779F916A3D3E90023804689469A
:10123000DDE90201FDF724FB42464B46FDF76CF960
:10124000CDE904015046594664E700BFAFF3008082
:101250000000601A61B4D03D7370032E8A19A33B5D
:1012600083C8C96D305FE43F00004054FB21F93F63
:101270003163621A61B4D03D0000002E8A19A33B8D
:10128000C14920259A837B39B4A1050834A10508FA
:10129000FDF744F942F2FB13C3F6F9739C42804612
:1012A00089461AD01EA3D3E90023FDF737F90D466E
:1012B00004462B462246C7E9004540464946FDF70D
:1012C0002BF917A3D3E90023FDF728F94FF0FF35D9
:1012D000C7E90201B7E6032495E613A3D3E9002387
:1012E000FDF71CF912A3D3E9002380468946FDF7D8
:1012F00015F90D4604462B462246C7E900454046EF
:101300004946FDF709F90AA3D3E90023FDF706F9D9
:101310004FF0FF35C7E9020195E6DDE906AB03E7CB
:101320003163621A61B4D03D0000601A61B4D03DEF
:101330007370032E8A19A33B2DE9F84353EC102B4D
:1013400000242546C7F6F074C7F6F0751C40AC4281
:101350002DED028BB0EE408AF0EE608A1946104601
:1013600000F0AB80002B7FDD1A1500F08980A2F51C
:101370007E7721F07F4323F47003073FD20743F4C5
:10138000801366D5C20F4FF0000C02EB43037F10B1
:101390004200654616204FF400116C18D60F9C428F
:1013A0004FEA420202DC65181B1B8C4449080138D5
:1013B00006EB4303F1D1202680464FF0004107E0C1
:1013C00043D0D40F49085200013E04EB43031BD025
:1013D000AB4208EB0104F3DD04F00049B9F1004F22
:1013E00004EB01082BD0A9469442C5EB0303C4EBE0
:1013F000020288BF013B4018D40F49085200013E49
:101400004D4604EB4303E3D11A4327D146084FEA84
:101410006C0101F17E511CF0010F01F5C00118BFF4
:1014200046F0004601EB0753324643EC182BB0EE72
:10143000480AF0EE680ABDEC028BBDE8F883B8F10B
:10144000000FD0DB05F10109CEE79442C4D91D4657
:10145000B7E7C20F02EB4303400093E7431C39D0C8
:1014600000F001031818D1E723F000441443DED044
:10147000002B36D11A46C10A153A40050029FAD088
:1014800011F4801329D149000133CC02FBD5C3F1FB
:101490000105C3F1200420FA04F4521921439840B5
:1014A000A2F57E7721F07F4323F47003073FD20734
:1014B00043F480133FF566AFCBE751EC100BFDF71B
:1014C000DFF902460B4651EC180BFDF727F841EC0B
:1014D000180BACE70CF1010C99E72024012500233F
:1014E000D9E751EC100B0B46FDF716F802460B46F8
:1014F000FDF7F0FA41EC180B99E700BF000000007F
:101500002DE9F04F5BEC10AB2DED028BB0EE418A74
:10151000F0EE618A2BF00044B4F1795F85B071DAA6
:1015200050465946FDF746FC002800F0FD80524623
:101530005B4650465946FDF7A3F981A3D3E9002342
:1015400006460F46FDF79CF97FA3D3E90023FCF77D
:10155000E5FF32463B46FDF793F97DA3D3E900232F
:10156000FCF7DAFF32463B46FDF78AF97AA3D3E966
:101570000023FCF7D3FF32463B46FDF781F978A301
:10158000D3E90023FCF7C8FF32463B46FDF778F964
:1015900075A3D3E90023FCF7C1FF32463B46FDF7B4
:1015A0006FF98046894600230022C3F6E073304677
:1015B0003946FDF765F94246CDE900014B46304614
:1015C0003946FDF75DF953EC182B04460D4650469D
:1015D0005946FDF755F902460B4620462946FCF7C9
:1015E0009BFF02460B46DDE90001FCF795FF0B4629
:1015F00000210246C3F6F0710020FCF78DFF41EC9C
:10160000100B83E052465B4650465946FDF738F9C9
:101610004BA3D3E9002306460F46FDF731F94AA351
:10162000D3E90023FCF77AFF32463B46FDF728F961
:1016300047A3D3E90023FCF76FFF32463B46FDF793
:101640001FF945A3D3E90023FCF768FF32463B4668
:10165000FDF716F942A3D3E90023FCF75DFF3246FC
:101660003B46FDF70DF940A3D3E90023FCF756FFF5
:101670003B463246FDF704F943F23233C3F6D373E7
:101680009C42804689468EDD0023C3F6E9739C4266
:1016900041DC0021A4F5001300220020C3F6F07104
:1016A00014461D46FCF738FFCDE902010023002255
:1016B000C3F6E07330463946FDF7E2F822462B4682
:1016C000FCF72AFF4246CDE900014B463046394639
:1016D000FDF7D6F853EC182B04460D4650465946F4
:1016E000FDF7CEF802460B4620462946FCF714FFCC
:1016F00002460B46DDE90001FCF70EFF02460B46F1
:10170000DDE90201FCF708FF41EC100B05B0BDEC70
:10171000028BBDE8F08F9FED067B00258DED027BEF
:101720000024C3F6D275C1E79FED030BEEE700BFBF
:10173000000000000000E73F000000000000F03F54
:10174000D43888BEE9FAA8BDC4B1B4BD9EEE213E2E
:10175000AD529C804F7E923E9015CB19A001FA3E6F
:101760007751C1166CC1563F4C5555555555A53F3F
:101770002DE9F04F4AF6AB25ADF51B7DD41EC2F620
:10178000AA2585FB0465E417A49F114E0690C4EBBF
:10179000A50424EAE47456F827600A941F46E3433C
:1017A00003EB43037C1E02EBC30314EB060809960C
:1017B00002940891079321D40A9EA599351B08F13C
:1017C00001080CAE4FEA8808002401EB85090BE004
:1017D000BCA2050859F80400FCF7ECFF04340135FD
:1017E0004445E6E9020109D0002DF3DA0434002073
:1017F000002101354445E6E90201F5D1099C002CA0
:101800002CDB099C5EAE06EBC4060DF5B87ABB4630
:101810000096029D002DC0F254820EA9069D01EB98
:10182000CB064FF000084FF00009002476E90223B0
:10183000F5E80201FDF724F802460B46404649460A
:10184000FCF76CFE0134BC4280468946EED1EAE9E1
:101850000289009DAA450BF1010BDAD1099E731E86
:101860009B0086AC9AAD04EB8604ED180B930096B2
:101870000C940D95009C009EE4009AAD2B19002E4F
:10188000049453E93C892EDD04995EAC059485AE41
:10189000651800230022C3F6706340464946FCF7F2
:1018A000EFFFFDF787FAFCF785FF00230022C4F263
:1018B000701382468B46FCF7E3FF02460B46404618
:1018C0004946FCF729FEFDF775FA044646F8044F31
:1018D00075E9020152465B46FCF720FE059CA542D5
:1018E00080468946D5D149EC108B079800F010FE50
:1018F00055EC104B00224FF07F5320462946FCF751
:10190000BFFF41EC100BFEF753FF002351EC100B0F
:101910000022C4F22003FCF7B3FF02460B46204628
:101920002946FCF7F9FD0D460446FDF743FA064645
:10193000FCF740FF02460B4620462946FCF7ECFD2B
:10194000079D002D8046894640F3C180009C9AADDA
:10195000621E05EB8202079C52F8503CC4F118004D
:1019600043FA00F101FA00F01B1AC4F117007618CF
:1019700042F8503C43FA00F5002D30DD009C013662
:10198000002C40F3B18186AA02EB840000244FF6BC
:10199000FF7352F8041BC0F2FF035B1A14B9C1F1C4
:1019A000807311B142F8043C01248242EFD10799BF
:1019B000002911DD012900F06D8102290CD1009A66
:1019C0009AA9531E01EB830353F8502C22F07F4257
:1019D00022F4400243F8502C022D00F08280404651
:1019E000494600220023FDF7B3F9002800F09C804F
:1019F000009C601E099C84420EDC009C86A901EBC1
:101A000084030C9C002253F8041DA34242EA010205
:101A1000F9D1002A40F070820D9C54F8503C002B04
:101A200040F068820B9D86AE7219012352F8041DA6
:101A300001330029FAD0009CE31804F1010A9A4509
:101A4000059341DC0A9E029D04EB060BA59C05EB69
:101A50000A0304EB8B0B049C013B0EAD5EAE05EB61
:101A6000C3053619009504965BF8040FFCF7A2FE37
:101A7000009D029EE5E90201002E00954FF000084E
:101A80004FF0000917DB0AEB07060EA9069D01EBD4
:101A9000C606002476E90223F5E80201FCF7F0FE11
:101AA00002460B4640464946FCF738FD0134BC422D
:101AB00080468946EED1049C059DE4E902890AF13D
:101AC000010AAA450494CFDD059E0096D2E640F0B7
:101AD000EF80009D9AA901EB850353F8545CED1546
:101AE0004AE7002142464B460020C3F6F071FCF75E
:101AF00013FD80468946002C3FF471AF07989FED97
:101B00008E0B00F005FD404653EC102B4946FCF7C8
:101B100003FD804689464046494600220023FDF7E2
:101B200017F900287FF464AF05960495002840F06B
:101B3000FC81079C49EC108B604200F0E9FC57ECFB
:101B4000106B0023304639460022C4F27013FDF7B3
:101B50001DF9002800F0F78100230022C3F670630E
:101B600030463946FCF78CFEFDF724F9FCF722FEDF
:101B700000230022C4F2701380468946FCF780FEE1
:101B800002460B4630463946FCF7C6FC009E9AAF2B
:101B900007EB860501360096FDF70CF99AA9034676
:101BA00001EB860445F8503C40464946FDF702F9F2
:101BB000079D44F8500C183507959FED5F0B07986B
:101BC00000F0A6FC009C002C57EC106B59DB013494
:101BD0005EAD86A95EAA069501EB840502EBC404FE
:101BE00055F8040DFCF7E6FD32463B46FCF748FE8F
:101BF000002364E90201002230463946C3F67063CF
